:020000040800F2
:10000000F0660120F1AD03081FAE030821AE03081E
:1000100023AE030825AE030827AE03080000000046
:1000200000000000000000000000000029AE0308EE
:100030002BAE0308000000002DAE0308DF180008F7
:1000400031AE030831AE030831AE030831AE030808
:1000500031AE030831AE030831AE030831AE0308F8
:1000600031AE030831AE030831AE030831AE0308E8
:100070006F86000831AE03085986000831AE0308C8
:1000800031AE03089D860008D519000831AE03087B
:100090006D71000831AE030831AE030831AE0308BC
:1000A000E775000831AE030831AE03086598000813
:1000B000273B000831AE030831AE030831AE030818
:1000C00031AE030831AE030831AE030831AE030888
:1000D00031AE030807150008792D00084315000804
:1000E000B119000831AE030831AE030831AE030880
:1000F0006319000831AE0308AB81000831AE030874
:1001000031AE0308A9190008299C000831AE030884
:100110003F2D000831AE03088D730008AD73000851
:1001200031AE030831AE030831AE030831AE030827
:1001300031AE030831AE030831AE030831AE030817
:10014000CB6D000831AE0308996E000831AE03088C
:1001500031AE030831AE030831AE0308B52D0008F7
:1001600031AE030831AE030831AE030831AE0308E7
:1001700031AE030831AE030831AE030831AE0308D7
:1001800031AE030800F002F800F058F80AA090E839
:10019000000C82448344AAF10107DA4501D100F042
:1001A0004DF8AFF2090EBAE80F0013F0010F18BFB7
:1001B000FB1A43F00103184760180400801804007C
:1001C0000A4410F8014B14F00F0508BF10F8015B4A
:1001D000240908BF10F8014B6D1E05D010F8013B33
:1001E0006D1E01F8013BF9D1641E03D0641E01F8B5
:1001F000015BFBD19142E4D370470000002300244F
:1002000000250026103A28BF78C1FBD8520728BF26
:1002100030C148BF0B607047782900F0BDA00020B6
:1002200070471FB540F090FB04000020002140F013
:1002300019FF401C60601FBD10B510BD40F0D8FE16
:100240001146FFF7EEFF00F009F840F0F6FE03B4A8
:10025000FFF7F2FF03BC40F0F7FE00001FB5624855
:10026000806840F480506049886068463BF039FA05
:100270004FF47A720198B0FBF2F1B1F1807F00D3B4
:100280001DE021F07F40401E4FF0E02250615017EA
:100290000F22002807DA13071E0E544B00F00F053B
:1002A0002D1F5E5503E013071D0E514B1D5400BF5B
:1002B00000204FF0E02290610720106100BF0DF098
:1002C00074FC05F08EFD00F045FC01F0C7F901F06B
:1002D000ABFB09F09BFD0EF071FB02F037FC07F061
:1002E00009F805F0DBFB05F0E8F80BF022F8002137
:1002F00001200BF08DF80BF0A7F80DF088FB01F052
:1003000071F911F02FFA11F079FC4FF4806139483E
:100310000BF086FB11F0D1FE0021422011F0EAFB28
:1003200053E001F07CF9012102200BF071F80AF092
:10033000C9FF0446022C07D10AF03CFD10B105F0BC
:10034000FEFC01E005F009FD2B480088012805D1DD
:100350002AA00EF035FC0020274908802848008894
:10036000042806D005280AD006280ED009281FD157
:1003700018E00020224908800FF012FD18E000204C
:100380001F4908800FF0B9FD12E00AF0DFFD18B92F
:10039000002102200BF03CF80020194908800FF0E2
:1003A00022FF05E000201649088010F0E1FB00BFA5
:1003B00000BF002011F0F7FE08B111F001FF114855
:1003C000007810B110480AF0C8FDAAE710B50F4830
:1003D00004882A2001F06CF820460EF049FC0D201C
:1003E00001F066F810BD0000002004E018ED00E008
:1003F00000E400E0822400200A0000202A310D00E1
:10040000040000202C0000207414002000FF0B08C2
:1004100000BFBFF34F8FF848006800F4E060F74971
:100420000843001DF4490860BFF34F8F00BF00BFB1
:10043000FEE710B50446022C03D10020F0490880E5
:1004400010BD032C02D10AF084FD0DE0EC480088B9
:1004500041F20E01884207D2E94801880088401C19
:10046000E74A1080E748445400BFE9E72DE9F0412E
:100470000020E449E24A128888540846057827207B
:1004800008702846392D73D008DCA0F13200052809
:100490006FD2DFE800F010D3EBF2F1005F2869D0F3
:1004A00004DC412867D0422863D1F6E2612875D088
:1004B0006228F9D1F2E2D348407830380A286ED267
:1004C000DFE800F005939798999A9B9C9DA7CD48EB
:1004D0008078382852D009DCA0F13000082822D2D8
:1004E000DFE800F01522812538394A4B462863D0D1
:1004F00006DC392843D0412842D0422873D144E059
:1005000061283ED0622841D066286CD155E02A206F
:1005100000F0CEFF0AF0B9FE064630460EF0A8FB0A
:100520000D2000F0C5FF5EE0FFF750FF5BE02A20E2
:1005300000F0BEFFB44800880EF04DFB202000F014
:10054000B7FF0EF0B9FA07460EF045FB0D2000F09C
:10055000AFFF48E047E0ADA00EF032FBAF480EF031
:100560002FFBAFA00EF02CFB0D2000F0A1FF3AE016
:1005700046E291E296E28BE235E034E033E032E0AD
:1005800000BFAAA00EF01CFB2DE000BFA948007818
:10059000012805D1A8A00EF013FB0CE079E24BE096
:1005A000A4480078022803D1A5A00EF009FB02E0C0
:1005B000A6A00EF005FB16E000BFA7A00EF000FB02
:1005C000AFA00EF0FDFAB1A00EF0FAFABAA00EF04C
:1005D000F7FABCA00EF0F4FAC1480EF049FB97A060
:1005E0000EF0EEFA00BF00BF26E00220BD490880F1
:1005F00022E021E000BF00BF00BF00BF00BF2A20F3
:1006000000F056FF05200EF0E6FA0D2000F050FF36
:1006100012E07C488078392809D12A2000F048FF70
:100620000220B14908800D2000F042FF00BF00BF4A
:100630000220AC49088000BF00BF34E27148407816
:1006400030380A2810D2DFE800F005060708090A4A
:100650000B0C0D0E08E000BF00BF00BF00BF00BFC5
:1006600000BF00BF00BF00BF00BF1CE2654840786C
:1006700030380A2816D201E063E015E0DFE800F028
:1006800005060708090A0B0C0D0E00BF00BF00BFCE
:1006900000BF00BF00BF00BF00BF00BF04209149E2
:1006A000088000BF00BFFEE15648407830380A2875
:1006B00045D2DFE800F005262728292A2B2C2D31EA
:1006C0005048807830380A2818D2DFE800F0050654
:1006D000170708090A0E121610E00FE00EE00DE0F1
:1006E0000CE001208149088008E001208049088051
:1006F00004E001207F49088000E000BF00BFBDE8A2
:10070000F08100BF00BF00BF00BF00BF00BF00BF3F
:1007100005207449088012E03A488078392809D1C8
:100720002A2000F0C5FE02206F4908800D2000F04D
:10073000BFFE00BF00BF05206A49088000BF00BFA0
:10074000DDE730484078362849D008DCA0F1300099
:10075000062845D2DFE800F010EFEEEDECEB39288B
:100760003FD004DC37283DD0382839D12CE141284E
:1007700039D06128F9D128E122488078392833D04E
:100780000ADCA0F13000092825D2DFE800F01825A6
:1007900024B5C8CCD5D9DD00612826D008DC412895
:1007A00024D0422823D0432822D0462813D1FEE06B
:1007B00062281ED063281DD066280CD1F6E02A20BE
:1007C00000F076FE0AF061FD064630460EF050FA63
:1007D0000D2000F06DFEEEE0FFF7F8FDEBE0F1E03C
:1007E0000CE1F7E0EFE0F1E0B2E0B5E0B5E0C1E048
:1007F000DBE0BEE0D8E000000CED00E00000FA0510
:100800005200002074140020020000204275696C20
:1008100064207461726765743A2000003016040821
:10082000202852656C656173652900002A43445095
:100830002B0D0000540000202A5553420D000000EB
:100840002A426C7565746F6F74680D002A556E6B63
:100850006E6F776E0D0000004461746520776865E7
:100860006E2074686520636F6D70696C6174696F68
:100870006E2077617320737461727465643A20002E
:100880004F63742032392032303135000D54696D98
:1008900065207768656E2074686520636F6D706988
:1008A0006C6174696F6E2077617320737461727408
:1008B00065643A200000000031343A32353A33336F
:1008C000000000000D56657273696F6E206F662020
:1008D00074686520636F6D70696C65723A20000002
:1008E000FA0E4D0004000020060000200800002041
:1008F0000A0000200C0000202A2000F0D9FD8248C8
:1009000000880EF068F9202000F0D2FD0EF0D4F837
:1009100007460EF060F90D2000F0CAFD4BE07B4861
:100920000EF02CFB47E001207949088043E048E0C5
:1009300046E044E042E040E00120764908803AE0A9
:1009400001207549088036E001207449088032E0B2
:100950000120734908802EE000BF2A2000F0A8FD86
:100960000DF062F807460EF083F90D2000F0A0FDAF
:1009700021E000BF2A2000F09BFD6448001FC078E2
:10098000432804D06148001FC078632804D165481B
:1009900000880EF020F903E0634800880EF01BF990
:1009A0000D2000F085FD06E000BF04E000BF5FA061
:1009B0000EF006F900BF00BFA1E600BF00BF00BFF8
:1009C00000BF00BF00BF00BF00BF00BF06205A49E4
:1009D000088013E04D48001F8078392809D12A206B
:1009E00000F066FD0220554908800D2000F060FDF2
:1009F00000BF00BF06205049088000BF00BF7EE650
:100A00004248001F407830380A283FD2DFE800F023
:100A1000051E1F202122232425293C48001F807801
:100A200030380A2810D2DFE800F005060708090A66
:100A30000B0C0D0E08E007E006E005E004E003E023
:100A400002E001E000E000BF00BF58E600BF00BFC9
:100A500000BF00BF00BF00BF00BF092036490880AB
:100A600014E02A48001F807839280AD134A00EF0FB
:100A7000A7F80AF05EFF04463249601C0AF088FFBE
:100A800000BF00BF09202C49088000BF00BF36E628
:100A900000BF41202849088005E000BF42202649C8
:100AA000088000E000BF00BF00BF28E610B5044684
:100AB0002548007818B12046FFF7BBFC19E02A2C26
:100AC00003D100202149088010BD0D2C02D1FFF771
:100AD000CDFC0EE01D48008841F20E01884208D28C
:100AE0001A4801880088401C184A10800748001FD7
:100AF000445400BFE8E70146154A1078117070476A
:100B0000134800787047000002000020781400208D
:100B10001A000020080000200A0000200C0000201D
:100B20000E00002026000020240000202A4D6169CC
:100B30006E206170700D000004000020060000208F
:100B4000A40D0000110400082C0000205200002019
:100B50005400002030B587B0012110203AF074FE17
:100B6000012188043AF05FFE0F200DF018F80128EB
:100B700001D1002071E00F200DF011F8022801D101
:100B800001206AE00F200DF00AF8042801D10220AC
:100B900063E00F200DF003F8082801D103205CE08A
:100BA0000F200CF0FCFF102801D1042055E00F208D
:100BB0000CF0F5FF202801D105204EE00F200CF0AD
:100BC000EEFF402801D1062047E00F200CF0E7FFA0
:100BD000802801D1072040E00F200CF0E0FFB0F5A5
:100BE000807F01D1082038E00F200CF0D8FFB0F54D
:100BF000007F01D1092030E00F200CF0D0FFB0F5CC
:100C0000806F01D10A2028E00F200CF0C8FFB0F55A
:100C1000006F01D10B2020E00F200CF0C0FFB0F5D9
:100C2000805F01D10C2018E00F200CF0B8FFB0F568
:100C3000005F01D10D2010E00F200CF0B0FFB0F5E7
:100C4000804F01D10E2008E00F200CF0A8FFB0F576
:100C5000004F01D10F2000E0FF2004460F200CF0D0
:100C600099FF0546072221463AF0F1F90E200CF0D3
:100C700096FF012801D1002071E00E200CF08FFFBB
:100C8000022801D101206AE00E200CF088FF042820
:100C900001D1022063E00E200CF081FF082801D171
:100CA00003205CE00E200CF07AFF102801D1042014
:100CB00055E00E200CF073FF202801D105204EE0F6
:100CC0000E200CF06CFF402801D1062047E00E20DA
:100CD0000CF065FF802801D1072040E00E200CF0C9
:100CE0005EFFB0F5807F01D1082038E00E200CF0C7
:100CF00056FFB0F5007F01D1092030E00E200CF046
:100D00004EFFB0F5806F01D10A2028E00E200CF0D4
:100D100046FFB0F5006F01D10B2020E00E200CF053
:100D20003EFFB0F5805F01D10C2018E00E200CF0E2
:100D300036FFB0F5005F01D10D2010E00E200CF061
:100D40002EFFB0F5804F01D10E2008E00E200CF0F0
:100D500026FFB0F5004F01D10F2000E0FF20044630
:100D60000E200CF017FF0546072221463AF06FF9D6
:100D70000D200CF014FF012801D1002071E00D209E
:100D80000CF00DFF022801D101206AE00D200CF0CB
:100D900006FF042801D1022063E00D200CF0FFFEC5
:100DA000082801D103205CE00D200CF0F8FE10288B
:100DB00001D1042055E00D200CF0F1FE202801D1D6
:100DC00005204EE00D200CF0EAFE402801D106205F
:100DD00047E00D200CF0E3FE802801D1072040E021
:100DE0000D200CF0DCFEB0F5807F01D1082038E04A
:100DF0000D200CF0D4FEB0F5007F01D1092030E0C9
:100E00000D200CF0CCFEB0F5806F01D10A2028E057
:100E10000D200CF0C4FEB0F5006F01D10B2020E0D6
:100E20000D200CF0BCFEB0F5805F01D10C2018E065
:100E30000D200CF0B4FEB0F5005F01D10D2010E0E4
:100E40000D200CF0ACFEB0F5804F01D10E2008E073
:100E50000D200CF0A4FEB0F5004F01D10F2000E0F2
:100E6000FF2004460D200CF095FE05460722214682
:100E70003AF0EDF80C200CF092FE012801D1002090
:100E800071E00C200CF08BFE022801D101206AE0F9
:100E90000C200CF084FE042801D1022063E00C2019
:100EA0000CF07DFE082801D103205CE00C200CF042
:100EB00076FE102801D1042055E00C200CF06FFEC6
:100EC000202801D105204EE00C200CF068FE4028BF
:100ED00001D1062047E00C200CF061FE802801D1F2
:100EE000072040E00C200CF05AFEB0F5807F01D1C5
:100EF000082038E00C200CF052FEB0F5007F01D144
:100F0000092030E00C200CF04AFEB0F5806F01D1D2
:100F10000A2028E00C200CF042FEB0F5006F01D151
:100F20000B2020E00C200CF03AFEB0F5805F01D1E0
:100F30000C2018E00C200CF032FEB0F5005F01D15F
:100F40000D2010E00C200CF02AFEB0F5804F01D1EE
:100F50000E2008E00C200CF022FEB0F5004F01D16D
:100F60000F2000E0FF2004460C200CF013FE054685
:100F7000072221463AF06BF814200CF010FE0128ED
:100F800001D1002071E014200CF009FE022801D1EB
:100F900001206AE014200CF002FE042801D1022096
:100FA00063E014200CF0FBFD082801D103205CE075
:100FB00014200CF0F4FD102801D1042055E0142079
:100FC0000CF0EDFD202801D105204EE014200CF09E
:100FD000E6FD402801D1062047E014200CF0DFFD9B
:100FE000802801D1072040E014200CF0D8FDB0F596
:100FF000807F01D1082038E014200CF0D0FDB0F53E
:10100000007F01D1092030E014200CF0C8FDB0F5BC
:10101000806F01D10A2028E014200CF0C0FDB0F54B
:10102000006F01D10B2020E014200CF0B8FDB0F5CA
:10103000805F01D10C2018E014200CF0B0FDB0F559
:10104000005F01D10D2010E014200CF0A8FDB0F5D8
:10105000804F01D10E2008E014200CF0A0FDB0F567
:10106000004F01D10F2000E0FF20044614200CF0B7
:1010700091FD05460722214639F0E9FF13200CF0C7
:101080008EFD012801D1002071E013200CF087FDB6
:10109000022801D101206AE013200CF080FD042811
:1010A00001D1022063E013200CF079FD082801D162
:1010B00003205CE013200CF072FD102801D1042005
:1010C00055E013200CF06BFD202801D105204EE0E7
:1010D00013200CF064FD402801D1062047E01320C6
:1010E0000CF05DFD802801D1072040E013200CF0BA
:1010F00056FDB0F5807F01D1082038E013200CF0B8
:101100004EFDB0F5007F01D1092030E013200CF036
:1011100046FDB0F5806F01D10A2028E013200CF0C5
:101120003EFDB0F5006F01D10B2020E013200CF044
:1011300036FDB0F5805F01D10C2018E013200CF0D3
:101140002EFDB0F5005F01D10D2010E013200CF052
:1011500026FDB0F5804F01D10E2008E013200CF0E1
:101160001EFDB0F5004F01D10F2000E0FF20044626
:1011700013200CF00FFD05460722214639F067FFCA
:1011800012200CF00CFD012801D1002071E012208A
:101190000CF005FD022801D101206AE012200CF0BC
:1011A000FEFC042801D1022063E012200CF0F7FCC1
:1011B000082801D103205CE012200CF0F0FC10287C
:1011C00001D1042055E012200CF0E9FC202801D1C7
:1011D00005204EE012200CF0E2FC402801D1062050
:1011E00047E012200CF0DBFC802801D1072040E012
:1011F00012200CF0D4FCB0F5807F01D1082038E03B
:1012000012200CF0CCFCB0F5007F01D1092030E0B9
:1012100012200CF0C4FCB0F5806F01D10A2028E048
:1012200012200CF0BCFCB0F5006F01D10B2020E0C7
:1012300012200CF0B4FCB0F5805F01D10C2018E056
:1012400012200CF0ACFCB0F5005F01D10D2010E0D5
:1012500012200CF0A4FCB0F5804F01D10E2008E064
:1012600012200CF09CFCB0F5004F01D10F2000E0E3
:10127000FF20044612200CF08DFC05460722214673
:1012800039F0E5FE11200CF08AFC012801D1002084
:1012900071E011200CF083FC022801D101206AE0EA
:1012A00011200CF07CFC042801D1022063E0112005
:1012B0000CF075FC082801D103205CE011200CF033
:1012C0006EFC102801D1042055E011200CF067FCC1
:1012D000202801D105204EE011200CF060FC4028B0
:1012E00001D1062047E011200CF059FC802801D1E3
:1012F000072040E011200CF052FCB0F5807F01D1B6
:10130000082038E011200CF04AFCB0F5007F01D134
:10131000092030E011200CF042FCB0F5806F01D1C3
:101320000A2028E011200CF03AFCB0F5006F01D142
:101330000B2020E011200CF032FCB0F5805F01D1D1
:101340000C2018E011200CF02AFCB0F5005F01D150
:101350000D2010E011200CF022FCB0F5804F01D1DF
:101360000E2008E011200CF01AFCB0F5004F01D15E
:101370000F2000E0FF20044611200CF00BFC054676
:101380000722214639F063FE02208DF808008DF80F
:10139000090000208DF80A0001208DF80B000F20B5
:1013A0000CF0FDFB01900F200CF0F4FB044601A9AA
:1013B00039F0CAFD14200CF0F2FB019014200CF05F
:1013C000E9FB044601A939F0BFFD0E200CF0E7FB54
:1013D00001900E200CF0DEFB044601A939F0B4FDAB
:1013E00013200CF0DCFB019013200CF0D3FB04461F
:1013F00001A939F0A9FD0D200CF0D1FB01900D20C1
:101400000CF0C8FB044601A939F09EFD12200CF037
:10141000C6FB019012200CF0BDFB044601A939F077
:1014200093FD0C200CF0BBFB01900C200CF0B2FBE8
:10143000044601A939F088FD11200CF0B0FB0190A1
:1014400011200CF0A7FB044601A939F07DFD4FF4F3
:101450008050ADF810008010ADF814004FF4E1306A
:1014600003900020ADF812000C20ADF816008001AA
:10147000ADF8180003A9564839F06CFE03A9554889
:1014800039F068FE0121524839F0ECFE0121514843
:1014900039F0E8FE012240F225514D4839F0EEFEC8
:1014A000012240F225514B4839F0E8FE07B030BD2B
:1014B00010B5044610F065F947480078022802D0BC
:1014C0000CF00EFA58B100BF8021424839F0A5FF58
:1014D0000028F9D021463F4839F031FF12E03E485C
:1014E0000078032803D1204609F0A2FD0AE000BFDE
:1014F0008021374839F091FF0028F9D0214634483F
:1015000039F01DFF10BD10B50821314839F085FFB5
:101510002F4839F018FFC4B240F225512C4839F059
:10152000C9FF2D480078032803D109F00FFD00B151
:1015300010BD0120284908702046FFF7B7FA00BF08
:10154000F6E710B50821234839F067FF214839F044
:10155000FAFEC4B240F225511E4839F0ABFF1F48D5
:10156000007830B11E48007810B901201C4908707D
:1015700010BD00201A4908700CF0B2F918B12046CD
:101580000CF011FAF4E714480078032803D109F0AD
:10159000DDFC00B1ECE702200F4908702046FFF7A0
:1015A00085FA00BFE4E710B5402010F0CFFA18B17B
:1015B0003F2010F0CBFA08B9012010BD0020FCE755
:1015C00008B9012100E00021044A117070470000B1
:1015D0000010014000480040540000205500002049
:1015E0005600002010B57D2039F099FF20B10EA0E3
:1015F00009F048FD3AF017FA45F255503EF068FE02
:1016000002203EF068FE4FF448603EF067FE002086
:101610003EF05EFE3EF065FE3EF068FE10BD10B589
:101620003EF05FFE10BD00005761746368646F6731
:101630003A643D31362C6F3D352C623D3136303ABF
:10164000612C702C672C702C612C702C652C702CEC
:10165000632C702C652C702C3861340008B54FF465
:1016600040703AF0EFFA25208DF800000F208DF839
:10167000010000208DF8020001208DF8030068466B
:101680003AF0E5FA27208DF800000C208DF80100D3
:1016900000208DF8020001208DF8030068463AF022
:1016A000D6FA34208DF800000A208DF801000020C1
:1016B0008DF8020001208DF8030068463AF0C7FA61
:1016C00026208DF800000A208DF8010000208DF8FA
:1016D000020001208DF8030068463AF0B8FA47206E
:1016E0008DF800000A208DF8010000208DF802001E
:1016F00001208DF8030068463AF0A9FA2E208DF8F3
:10170000000008208DF8010000208DF80200012063
:101710008DF8030068463AF09AFA1B208DF8000015
:1017200008208DF8010000208DF8020001208DF8BE
:10173000030068463AF08BFA32208DF8000008204A
:101740008DF8010000208DF8020001208DF80300C3
:1017500068463AF07CFA0E208DF8000009208DF8DA
:10176000010000208DF8020001208DF8030068467A
:101770003AF06DFA0C208DF8000009208DF8010078
:1017800000208DF8020001208DF8030068463AF031
:101790005EFA11208DF8000009208DF8010000206C
:1017A0008DF8020001208DF8030068463AF04FFAE8
:1017B00040208DF800000B208DF8010000208DF8EE
:1017C000020001208DF8030068463AF040FA4220FA
:1017D0008DF800000B208DF8010000208DF802002C
:1017E00001208DF8030068463AF031FA36208DF872
:1017F000000005208DF8010000208DF80200012076
:101800008DF8030068463AF022FA37208DF8000080
:1018100004208DF8010000208DF8020001208DF8D1
:10182000030068463AF013FA18208DF800000320F0
:101830008DF8010000208DF8020001208DF80300D2
:1018400068463AF004FA28208DF800000F208DF841
:10185000010000208DF8020001208DF80300684689
:101860003AF0F5F912208DF800000E208DF80100F5
:1018700000208DF8020001208DF8030068463AF040
:10188000E6F92C208DF800000F208DF801000020D3
:101890008DF8020001208DF8030068463AF0D7F970
:1018A00031208DF800000A208DF8010000208DF80D
:1018B000020001208DF8030068463AF0C8F91C20A8
:1018C0008DF800000C208DF8010000208DF802003A
:1018D00001208DF8030068463AF0B9F908BD10B54B
:1018E00047480068401C4649086046480068401C5C
:1018F0004449086044480068401C43490860434824
:101900000068401C4149086041480068401C40494B
:10191000086040480088401C3E49088004F0EAFA0C
:101920003B4800680A21B0FBF1F201FB120030B91C
:1019300039480088401C3849088003F0CCFF3448FF
:1019400000681E21B0FBF1F201FB1200042801D156
:101950000DF076F809F013FD09F0E5FF09F0ECFF52
:1019600010BD10B501212D483BF076FB38B10121A7
:101970002A483BF07AFB012128483BF08AFB0121F1
:1019800027483BF069FB70B103F08AFD18B903F0FA
:10199000B0FF04F038FA012121483BF066FB012139
:1019A0001F483BF076FB10BD10B53EF02AF810BD85
:1019B00010B54FF400503EF0B0F938B14FF400507C
:1019C0003EF0B6F94FF400503EF0C7F910BD104894
:1019D0000068704710B540F2052112483EF060FCE7
:1019E00060B110483EF06DFB044640F205210D4801
:1019F0003EF069FC20460DF09BF800BF10BD0000D2
:101A0000380000203C00002044000020400000205E
:101A1000580000201E000020100000200018004088
:101A2000001C00400020014030B587B001210803B0
:101A300039F00AFF23200CF0B2F8012801D1002070
:101A400071E023200CF0ABF8022801D101206AE0FC
:101A500023200CF0A4F8042801D1022063E0232005
:101A60000CF09DF8082801D103205CE023200CF045
:101A700096F8102801D1042055E023200CF08FF8AF
:101A8000202801D105204EE023200CF088F84028C2
:101A900001D1062047E023200CF081F8802801D1F5
:101AA000072040E023200CF07AF8B0F5807F01D1C8
:101AB000082038E023200CF072F8B0F5007F01D147
:101AC000092030E023200CF06AF8B0F5806F01D1D6
:101AD0000A2028E023200CF062F8B0F5006F01D155
:101AE0000B2020E023200CF05AF8B0F5805F01D1E4
:101AF0000C2018E023200CF052F8B0F5005F01D163
:101B00000D2010E023200CF04AF8B0F5804F01D1F1
:101B10000E2008E023200CF042F8B0F5004F01D170
:101B20000F2000E0FF20044623200CF033F8054688
:101B30000522214639F08BFA24200CF030F80128D8
:101B400001D1002071E024200CF029F8022801D1F5
:101B500001206AE024200CF022F8042801D10220A0
:101B600063E024200CF01BF8082801D103205CE07E
:101B700024200CF014F8102801D1042055E0242072
:101B80000CF00DF8202801D105204EE024200CF0A7
:101B900006F8402801D1062047E024200BF0FFFF83
:101BA000802801D1072040E024200BF0F8FFB0F599
:101BB000807F01D1082038E024200BF0F0FFB0F541
:101BC000007F01D1092030E024200BF0E8FFB0F5C0
:101BD000806F01D10A2028E024200BF0E0FFB0F54F
:101BE000006F01D10B2020E024200BF0D8FFB0F5CE
:101BF000805F01D10C2018E024200BF0D0FFB0F55D
:101C0000005F01D10D2010E024200BF0C8FFB0F5DB
:101C1000804F01D10E2008E024200BF0C0FFB0F56A
:101C2000004F01D10F2000E0FF20044624200BF0DC
:101C3000B1FF05460522214639F009FA25200BF0AF
:101C4000AEFF012801D1002071E025200BF0A7FF95
:101C5000022801D101206AE025200BF0A0FF042812
:101C600001D1022063E025200BF099FF082801D163
:101C700003205CE025200BF092FF102801D1042006
:101C800055E025200BF08BFF202801D105204EE0E8
:101C900025200BF084FF402801D1062047E02520B5
:101CA0000BF07DFF802801D1072040E025200BF0BC
:101CB00076FFB0F5807F01D1082038E025200BF0B9
:101CC0006EFFB0F5007F01D1092030E025200BF038
:101CD00066FFB0F5806F01D10A2028E025200BF0C7
:101CE0005EFFB0F5006F01D10B2020E025200BF046
:101CF00056FFB0F5805F01D10C2018E025200BF0D5
:101D00004EFFB0F5005F01D10D2010E025200BF053
:101D100046FFB0F5804F01D10E2008E025200BF0E2
:101D20003EFFB0F5004F01D10F2000E0FF20044638
:101D300025200BF02FFF05460522214639F087F9B3
:101D400002208DF818008DF8190000208DF81A0077
:101D50008DF81B0023200BF022FF059023200BF0B1
:101D600019FF044605A939F0EFF824200BF017FFFE
:101D7000059024200BF00EFF044605A939F0E4F885
:101D800025200BF00CFF059025200BF003FF0446E7
:101D900005A939F0D9F801208DF8180002208DF836
:101DA000190000208DF81A008DF81B0044200BF05C
:101DB000F6FE059044200BF0EDFE044605A939F02F
:101DC000C3F83D200BF0EBFE05903D200BF0E2FE4A
:101DD000044605A939F0B8F826200BF0E0FE05907E
:101DE00026200BF0D7FE044605A939F0ADF80121F5
:101DF00044200FF07FFE01213D200FF07BFE0121EA
:101E000026200FF077FE4FF44040ADF800004FF46D
:101E10008270ADF802000020ADF80400ADF80600B5
:101E2000ADF808004FF40070ADF80A003820ADF8A6
:101E30000C000020ADF80E00ADF810006946FE4819
:101E400039F094FF0121FC483AF093F807B030BD17
:101E50002DE9F04105460F461646072D06D1F748F5
:101E6000007840F01000F5490870AEE10020F44918
:101E70000870F4490870F148007800F01000EF494C
:101E800008700C2D55D2DFE805F006310E15232A17
:101E900038541C3F464D0020E9490870E949087054
:101EA000E649087049E0E648007840F02000E4493F
:101EB000087042E0E248007840F00200E049087013
:101EC0003BE0DF48007840F00200DD49087034E074
:101ED000DB48007840F00400D94908702DE0D8486C
:101EE000007840F00800D649087026E0D448007811
:101EF00040F00100D24908701FE0D148007840F05E
:101F00001000CF49087018E0CC48007840F020005D
:101F1000CA49087011E0C948007840F04000C7493C
:101F200008700AE0C548007840F08000C349087096
:101F300003E00020C249087000BF00BF102F77D215
:101F4000DFE807F096080910171819252C384455B2
:101F50005C6977898DE0BB48007840F00800B9499A
:101F6000087086E0B748007840F00200B549087074
:101F70007FE07EE07DE0B348007840F00200B149A8
:101F800008700846007840F00800087071E0AD481D
:101F9000007840F00100AB4908706AE0A948007879
:101FA00040F00100A74908700846007840F0100092
:101FB00008705EE0A348007840F00100A149087075
:101FC0000846007840F00200087052E09D48007812
:101FD00040F001009B4908700846007840F002007C
:101FE00008700846007840F01000087041E09448FE
:101FF000007840F04000924908703AE0904800783C
:1020000040F040008E4908708E48007840F0200073
:102010008C4908702DE08A48007840F040008849DB
:1020200008708848007840F004008649087020E075
:102030001EE08348007840F04000814908708148E4
:10204000007840F004007F4908700846007840F0AE
:10205000200008700DE07A48007840F04000784990
:1020600008707848007840F001007649087000E078
:1020700000BF00BF102E7AD2DFE806F099080910E1
:10208000171819262D3A46585F6C7A8C9CE06B48DD
:10209000007840F002006949087095E069480078CE
:1020A00040F08000674908708EE08DE08CE0654864
:1020B000007840F08000634908706048007840F084
:1020C00002005E4908707FE05E48007840F0400002
:1020D0005C49087078E05B48007840F0400059495E
:1020E00008705648007840F00400544908706BE0CE
:1020F0005448007840F04000524908700846007883
:1021000040F0800008705FE04E48007840F04000EA
:102110004C4908700846007840F080000870474835
:10212000007840F00400454908704DE044480078CC
:1021300040F080004249087046E04148007840F095
:1021400080003F4908703D48007840F008003B4956
:10215000087039E03A48007840F08000384908704B
:102160003648007840F00100344908702CE01EE049
:102170003348007840F08000314908702F480078DB
:1021800040F001002D4908700846007840F0080032
:10219000087019E02A48007840F08000284908704B
:1021A0002848007840F04000264908700CE0244898
:1021B000007840F08000224908702248007840F002
:1021C00040002049087000BF00BF05200DF082FDCF
:1021D0001A480178184839F009FF002144200FF00F
:1021E00089FC05200DF076FD1748046800BF022128
:1021F000114839F04EFF20B913480068001B3228FF
:10220000F5D31148046800BF02210B4839F041FFA3
:1022100020B90D480068001B3228F5D305200DF0C9
:1022200059FD08480178044839F0E0FE0648046882
:1022300000BF0221004809E0003001405E0000209C
:102240005C0000205D0000203800002039F021FFF4
:1022500020B914480068001B3228EAD305200DF08D
:1022600039FD11480178114839F0C0FE0D48046865
:1022700000BF02210D4839F00CFF20B90948006861
:10228000001B3228F5D305200DF024FD0121442048
:102290000FF030FC1EB9012145200FF02BFCBDE8EA
:1022A000F0810000380000205C0000200030014078
:1022B00010B5F748007868B90CF030FC012804D15B
:1022C00000214B200FF016FC15E001214B200FF0F0
:1022D00011FC10E0EE480078012804D100214B20C9
:1022E0000FF008FC07E0EA480078022803D101213A
:1022F0004B200FF0FFFB10BD30B587B00121C804A3
:1023000039F091FA0121480439F08DFA0121202099
:1023100039F09AFA22200BF042FC012801D100206A
:1023200071E022200BF03BFC022801D101206AE081
:1023300022200BF034FC042801D1022063E022208B
:102340000BF02DFC082801D103205CE022200BF0CB
:1023500026FC102801D1042055E022200BF01FFCA0
:10236000202801D105204EE022200BF018FC402847
:1023700001D1062047E022200BF011FC802801D17A
:10238000072040E022200BF00AFCB0F5807F01D14D
:10239000082038E022200BF002FCB0F5007F01D1CC
:1023A000092030E022200BF0FAFBB0F5806F01D15C
:1023B0000A2028E022200BF0F2FBB0F5006F01D1DB
:1023C0000B2020E022200BF0EAFBB0F5805F01D16A
:1023D0000C2018E022200BF0E2FBB0F5005F01D1E9
:1023E0000D2010E022200BF0DAFBB0F5804F01D178
:1023F0000E2008E022200BF0D2FBB0F5004F01D1F7
:102400000F2000E0FF20044622200BF0C3FB05460E
:102410000822214638F01BFE21200BF0C0FB0128CA
:1024200001D1002071E021200BF0B9FB022801D17D
:1024300001206AE021200BF0B2FB042801D1022028
:1024400063E021200BF0ABFB082801D103205CE006
:1024500021200BF0A4FB102801D1042055E02120FD
:102460000BF09DFB202801D105204EE021200BF030
:1024700096FB402801D1062047E021200BF08FFB7E
:10248000802801D1072040E021200BF088FBB0F527
:10249000807F01D1082038E021200BF080FBB0F5CF
:1024A000007F01D1092030E021200BF078FBB0F54E
:1024B000806F01D10A2028E021200BF070FBB0F5DD
:1024C000006F01D10B2020E021200BF068FBB0F55C
:1024D000805F01D10C2018E021200BF060FBB0F5EB
:1024E000005F01D10D2010E021200BF058FBB0F56A
:1024F000804F01D10E2008E021200BF050FBB0F5F9
:10250000004F01D10F2000E0FF20044621200BF0F6
:1025100041FB05460822214638F099FD20200BF0AA
:102520003EFB012801D1002071E020200BF037FB99
:10253000022801D101206AE020200BF030FB0428A2
:1025400001D1022063E020200BF029FB082801D1F3
:1025500003205CE020200BF022FB102801D1042096
:1025600055E020200BF01BFB202801D105204EE078
:1025700020200BF014FB402801D1062047E020204A
:102580000BF00DFB802801D1072040E020200BF04C
:1025900006FBB0F5807F01D1082038E020200BF049
:1025A000FEFAB0F5007F01D1092030E020200BF0C9
:1025B000F6FAB0F5806F01D10A2028E020200BF058
:1025C000EEFAB0F5006F01D10B2020E020200BF0D7
:1025D000E6FAB0F5805F01D10C2018E020200BF066
:1025E000DEFAB0F5005F01D10D2010E020200BF0E5
:1025F000D6FAB0F5804F01D10E2008E020200BF074
:10260000CEFAB0F5004F01D10F2000E0FF200446C4
:1026100020200BF0BFFA05460722214638F017FDAF
:102620001F200BF0BCFA012801D1002073E01F200D
:102630000BF0B5FA022801D101206CE01F200BF04D
:10264000AEFA042801D1022065E01F200BF0A7FAA2
:10265000082801D103205EE01F200BF0A0FA10280B
:1026600001D1042057E01F200BF099FA202801D156
:10267000052050E01F200BF092FA402801D10620DF
:1026800049E01F200BF08BFA802803D1072042E09D
:10269000720000201F200BF082FAB0F5807F01D17C
:1026A000082038E01F200BF07AFAB0F5007F01D146
:1026B000092030E01F200BF072FAB0F5806F01D1D5
:1026C0000A2028E01F200BF06AFAB0F5006F01D154
:1026D0000B2020E01F200BF062FAB0F5805F01D1E3
:1026E0000C2018E01F200BF05AFAB0F5005F01D162
:1026F0000D2010E01F200BF052FAB0F5804F01D1F1
:102700000E2008E01F200BF04AFAB0F5004F01D16F
:102710000F2000E0FF2004461F200BF03BFA054687
:102720000722214638F093FC1E200BF038FA0128CE
:1027300001D1002071E01E200BF031FA022801D1F6
:1027400001206AE01E200BF02AFA042801D10220A1
:1027500063E01E200BF023FA082801D103205CE07F
:102760001E200BF01CFA102801D1042055E01E2079
:102770000BF015FA202801D105204EE01E200BF0A9
:102780000EFA402801D1062047E01E200BF007FA80
:10279000802801D1072040E01E200BF000FAB0F5A0
:1027A000807F01D1082038E01E200BF0F8F9B0F549
:1027B000007F01D1092030E01E200BF0F0F9B0F5C8
:1027C000806F01D10A2028E01E200BF0E8F9B0F557
:1027D000006F01D10B2020E01E200BF0E0F9B0F5D6
:1027E000805F01D10C2018E01E200BF0D8F9B0F565
:1027F000005F01D10D2010E01E200BF0D0F9B0F5E4
:10280000804F01D10E2008E01E200BF0C8F9B0F572
:10281000004F01D10F2000E0FF2004461E200BF0E6
:10282000B9F905460822214638F011FC1D200BF0AD
:10283000B6F9012801D1002071E01D200BF0AFF99D
:10284000022801D101206AE01D200BF0A8F904281C
:1028500001D1022063E01D200BF0A1F9082801D16D
:1028600003205CE01D200BF09AF9102801D1042010
:1028700055E01D200BF093F9202801D105204EE0F2
:102880001D200BF08CF9402801D1062047E01D20C7
:102890000BF085F9802801D1072040E01D200BF0C6
:1028A0007EF9B0F5807F01D1082038E01D200BF0C3
:1028B00076F9B0F5007F01D1092030E01D200BF042
:1028C0006EF9B0F5806F01D10A2028E01D200BF0D1
:1028D00066F9B0F5006F01D10B2020E01D200BF050
:1028E0005EF9B0F5805F01D10C2018E01D200BF0DF
:1028F00056F9B0F5005F01D10D2010E01D200BF05E
:102900004EF9B0F5804F01D10E2008E01D200BF0EC
:1029100046F9B0F5004F01D10F2000E0FF2004463A
:102920001D200BF037F905460822214638F08FFBB1
:1029300050200BF034F9012801D1002071E0502023
:102940000BF02DF9022801D101206AE050200BF094
:1029500026F9042801D1022063E050200BF01FF972
:10296000082801D103205CE050200BF018F9102852
:1029700001D1042055E050200BF011F9202801D19D
:1029800005204EE050200BF00AF9402801D1062026
:1029900047E050200BF003F9802801D1072040E0E8
:1029A00050200BF0FCF8B0F5807F01D1082038E012
:1029B00050200BF0F4F8B0F5007F01D1092030E091
:1029C00050200BF0ECF8B0F5806F01D10A2028E020
:1029D00050200BF0E4F8B0F5006F01D10B2020E09F
:1029E00050200BF0DCF8B0F5805F01D10C2018E02E
:1029F00050200BF0D4F8B0F5005F01D10D2010E0AD
:102A000050200BF0CCF8B0F5804F01D10E2008E03B
:102A100050200BF0C4F8B0F5004F01D10F2000E0BA
:102A2000FF20044650200BF0B5F80546032221464E
:102A300038F00DFB02208DF808008DF80900002009
:102A40008DF80A0001208DF80B0022200BF0A7F86A
:102A5000019022200BF09EF8044601A938F074FA88
:102A600021200BF09CF8019021200BF093F80446F4
:102A700001A938F069FA02208DF808008DF80900E4
:102A800000208DF80A0001208DF80B0020200BF0AB
:102A900086F8019020200BF07DF8044601A938F05B
:102AA00053FA1F200BF07BF801901F200BF072F8F7
:102AB000044601A938F048FA02208DF808008DF884
:102AC000090000208DF80A0001208DF80B001D2060
:102AD0000BF065F801901D200BF05CF8044601A98D
:102AE00038F032FA1E200BF05AF801901E200BF03D
:102AF00051F8044601A938F027FA50200BF04FF89E
:102B0000019050200BF046F8044601A938F01CFA59
:102B100042F6A00003900020ADF81000ADF81200BE
:102B2000ADF814000C20ADF816000020ADF8180028
:102B300003A9FE4838F00EFB03A9FD4838F00AFB54
:102B400003A9FC4838F006FB07B030BD1CB5472090
:102B50000BF025F8009001208DF8040002208DF87C
:102B6000050000208DF806008DF8070047200BF0C7
:102B700011F80446694638F0E7F948200BF00FF8E1
:102B8000009048200BF006F80446694638F0DCF95E
:102B900049200BF004F8009001208DF80400022079
:102BA0008DF8050000208DF806008DF807004920FB
:102BB0000AF0F0FF0446694638F0C6F94A200AF0E8
:102BC000EEFF00904A200AF0E5FF0446694638F01F
:102BD000BBF94B200AF0E3FF009001208DF80400C0
:102BE00002208DF8050000208DF806008DF8070002
:102BF0004B200AF0CFFF0446694638F0A5F94C2077
:102C00000AF0CDFF00904C200AF0C4FF044669464C
:102C100038F09AF94D200AF0C2FF00904D200AF0DA
:102C2000B9FF0446694638F08FF946200AF0B7FF2D
:102C3000009001208DF8060046200AF0ABFF044604
:102C4000694638F081F945200AF0A9FF0090452037
:102C50000AF0A0FF0446694638F076F94E200AF0E3
:102C60009EFF009000208DF8040002208DF80500E2
:102C700000208DF806008DF807004E200AF08AFF2C
:102C80000446694638F060F9012146200EF032FF13
:102C9000012145200EF02EFF01200DF01BF801212F
:102CA00046200EF027FF01200DF014F800214620E9
:102CB0000EF020FF012145200EF01CFF01200DF039
:102CC00009F8002145200EF015FF01214B200EF0E0
:102CD00011FF002098490870FFF70EFB1CBD70B56E
:102CE00004460D46042D04D0052D1AD0062D24D1FE
:102CF0000BE000BF80218E4838F08FFB0028F9D010
:102D0000A1B28B4838F01BFB17E000BF8021894837
:102D100038F083FB0028F9D0A1B2864838F00FFBC9
:102D20000BE000BF8021814838F077FB0028F9D004
:102D3000A1B27E4838F003FB00BF00BF70BD10B5E4
:102D400040F225517A4838F0B5FB0821784838F030
:102D500064FB774838F0F7FA7849794A128821F805
:102D6000120077480088B0F57A7F04D27448008852
:102D7000401C7349088010BD10B540F225516D48C4
:102D800038F098FB08216B4838F047FB694838F069
:102D9000DAFAC0B269496A4A128821F81200684812
:102DA0000088B0F57A7F04D265480088401C6449E9
:102DB000088010BD10B540F225515C4838F07AFB10
:102DC00008215A4838F029FB584838F0BCFA044624
:102DD0005C48007818B95C48007800287ED05B48D1
:102DE00000885B490988401A80B225283DDD554896
:102DF0000078C8B355480088554908805548007880
:102E0000401C544908700020097801EB410202EB94
:102E1000C101514A02F811004E48007800EB40020F
:102E200002EBC0004C4A02EB40024A48007800EB3B
:102E3000400303EBC000484B13F81000401C14542F
:102E40004448007800EB400101EBC000194611F83E
:102E50001000401C3F49097801EB410202EBC1011F
:102E60001A4602F811009DE0FFE73848008838490B
:102E70000988401A80B228283FDD334800780128AD
:102E80003BD1324800883249088032480078401CE3
:102E9000304908700020097801EB410202EBC101C2
:102EA0002D4A02F811002B48007800EB400202EB9B
:102EB000C000294A02EB40022648007800EB40039C
:102EC00003EBC000244B13F81000401C145421489D
:102ED000007800EB400101EBC00000E052E0194631
:102EE00011F81000401C1B49097801EB410202EB6C
:102EF000C1011A4602F8110054E014480088144930
:102F000008801448007800EB400101EBC000124932
:102F100001EB40010F48007800EB400303EBC000D9
:102F20000D4B13F81000401C0C5417E00014014026
:102F3000004C0040004400407200002004080020C3
:102F4000160000202D0000202E0000209C000020F4
:102F50009C02002097020020393B0120FE480078A7
:102F600000EB400101EBC000194611F81000401CB5
:102F7000F949097801EB410202EBC1011A4602F856
:102F800011000FE0E0B2F549F54A128821F812006D
:102F9000F3480088B0F57A7F04D2F1480088401CDD
:102FA000EF49088010BD10B504460CB1012000E0C7
:102FB00000200146EB4838F055F90CB1012000E043
:102FC00000200146E84838F04DF90CB1012000E03E
:102FD00000200146E54838F045F910BD7FB50646AA
:102FE0000C461546FFF788F90020FFF7DCFF009636
:102FF000092C03D14FF48050ADF80400082C02D105
:103000000020ADF804000020ADF806000DB9ADF8C1
:103010000800012D0DD14FF4C060ADF80800072C59
:1030200002D10020ADF80400082C02D16002ADF8F6
:103030000400022D0CD16802ADF80800072C02D163
:103040000020ADF80400082C02D16002ADF80400A5
:10305000032D0BD10020ADF80800072C01D1ADF8ED
:103060000400082C02D16002ADF80400042D0BD13D
:103070000020ADF80800072C01D1ADF80400082CA1
:1030800002D16002ADF804000C20ADF80A00002067
:10309000ADF80C006946B34838F05CF86946B248B0
:1030A00038F058F86946B14838F054F80120FFF775
:1030B0007AFF7FBD1CB501208DF8040002208DF839
:1030C000050000208DF806008DF8070022200AF088
:1030D00066FD009022200AF05DFD0446694637F047
:1030E00033FF21200AF05BFD009002208DF80400E0
:1030F00021200AF04FFD0446694637F025FF1CBD2C
:10310000F0B587B004460D4699480480994805807B
:1031100000220421080739F022FD0021914838F0EF
:10312000A1F80021904838F09DF800218F4838F030
:1031300099F8FFF7BFFF0121084638F074FB212002
:103140000AF02DFD012801D1002071E021200AF0B4
:1031500026FD022801D101206AE021200AF01FFD8E
:10316000042801D1022063E021200AF018FD08287C
:1031700001D103205CE021200AF011FD102801D1CB
:10318000042055E021200AF00AFD202801D1052065
:103190004EE021200AF003FD402801D1062047E03F
:1031A00021200AF0FCFC802801D1072040E02120EA
:1031B0000AF0F5FCB0F5807F01D1082038E021202D
:1031C0000AF0EDFCB0F5007F01D1092030E02120AC
:1031D0000AF0E5FCB0F5806F01D10A2028E021203B
:1031E0000AF0DDFCB0F5006F01D10B2020E02120BA
:1031F0000AF0D5FCB0F5805F01D10C2018E0212049
:103200000AF0CDFCB0F5005F01D10D2010E02120C7
:103210000AF0C5FCB0F5804F01D10E2008E0212056
:103220000AF0BDFCB0F5004F01D10F2000E0FF20F7
:10323000064621200AF0AEFC07460122314637F04F
:1032400006FF3C20ADF810000020ADF812004A48FF
:10325000B0FBF4F005900020ADF8180004A94FF081
:10326000804039F0D8F90420ADF8040041480088C6
:10327000012803D10A20ADF8060002E00220ADF8D3
:1032800006000120ADF808000020ADF80A00ADF8F6
:103290000C0001A94FF0804039F09DFB4FF0FF3149
:1032A0004FF0804039F0B5FE0421080739F0DDFE0B
:1032B0000421080739F0EDFE01220421080739F046
:1032C0004EFC07B0F0BD10B500214FF0804039F042
:1032D0002CFC00220421080739F041FC00220421C3
:1032E000080739F006FE10BD10B5044600214FF066
:1032F000804039F088FE0121880739F0CAFE1F4856
:10330000048008201E49088000201E4908800021F2
:1033100022200EF0EFFB01221146900739F01FFC2E
:103320000121880739F001FC10BD10B5044604F0F6
:10333000E6F910BD7CB50446072C42D2DFE804F064
:1033400004425580B8CBDE00FEF7B2FF00214920D1
:103350000EF0D0FB002117E09702002004080020A7
:1033600016000020004C00400014014000440040C2
:10337000680000206C00002040420F006A0000201E
:1033800064000020620000204A200EF0B3FB0122FE
:1033900040F22551FB4837F071FF002240F22551E1
:1033A000F94837F06BFF002240F22551F74837F01B
:1033B00065FF002149200EF09DFB00214A200EF000
:1033C00099FBD9E0002240F22551EE4837F056FF34
:1033D000012240F22551EC4837F050FF002240F224
:1033E0002551EA4837F04AFFC6E0002149200EF097
:1033F00081FB00214A200EF07DFB01214C200EF0C4
:1034000079FB00214D200EF075FB012147200EF0C5
:1034100071FB012148200EF06DFB002240F2255186
:10342000D84837F02BFF002240F22551D64837F01C
:1034300025FF012240F22551D44837F01FFF9BE0C1
:1034400001208DF8040002208DF8050000208DF881
:10345000060001208DF8070022200AF0A0FB009052
:1034600022200AF097FB0546694637F06DFD0121E1
:1034700022200EF03FFBFEF71BFF002149200EF03B
:1034800039FB00214A200EF035FB012240F2255184
:10349000BC4837F0F3FE002240F22551BA4837F01D
:1034A000EDFE002240F22551B84837F0E7FE63E018
:1034B000012240F22551B34837F0E0FE002240F2ED
:1034C0002551B14837F0DAFE002240F22551AF48CD
:1034D00037F0D4FE50E0012240F22551A94837F0E0
:1034E000CDFE002240F22551A74837F0C7FE00224A
:1034F00040F22551A54837F0C1FE3DE00021A34828
:1035000037F0B0FE01208DF8040002208DF8050090
:1035100000208DF8060001208DF8070020200AF019
:103520003EFB009020200AF035FB0546694637F047
:103530000BFD002149200EF0DDFA00214A200EF09B
:10354000D9FA012120200EF0D5FA012148200EF0F1
:10355000D1FA002240F225518A4837F08FFE00222E
:1035600040F22551884837F089FE002240F225516B
:10357000864837F083FE00BF00BF7CBD2DE9FC41CB
:1035800007460E46154601208DF8040002208DF8EE
:10359000050000208DF8060001208DF807000DB110
:1035A000681E85B2042F04D0052F2DD0062F7DD1A3
:1035B00055E022200AF0F3FA009022200AF0EAFAFD
:1035C0008046694637F0C0FC012122200EF092FAB5
:1035D00001200CF07FFB002122200EF08BFA6C48BA
:1035E000046800BF6A480068001BB042FAD301219A
:1035F00022200EF07FFA6648046800BF6448006825
:10360000001BA842FAD35BE01E200AF0C8FA009023
:103610001E200AF0BFFA8046694637F095FC01216A
:103620001E200EF067FA01200CF054FB00211E2032
:103630000EF060FA5648046800BF55480068001B49
:10364000B042FAD301211E200EF054FA504804680B
:1036500000BF4F480068001BA842FAD330E020208A
:103660000AF09DFA009020200AF094FA80466946FC
:1036700037F06AFC012120200EF03CFA01200CF00A
:1036800029FB002120200EF035FA4148046800BFD4
:103690003F480068001BB042FAD3012120200EF001
:1036A00029FA3B48046800BF394800E004E000689C
:1036B000001BA842F8D303E036A00BF081FA00BF4C
:1036C00000BFBDE8FC812DE9F04F8BB080468946F4
:1036D00016469A46159C00250027AB464FF4A0508D
:1036E00037F09DFF012211022F4839F0C0FA41F254
:1036F0008831149891FBF0F02C49088027462C481B
:103700000680072E02D14FF0800B06E0082E02D172
:103710004FF4807B01E04FF0000B03E0781E074080
:10372000681C85B2002FF9D1284605EBD0714910ED
:10373000A5EB41018DB2B9F1000F06D0B9F1010F2F
:1037400006D0B9F1020F3AD110E01A48048037E0F0
:1037500017480088401C1649088025B904EB0B0067
:103760001449088001E01348048029E010480088CB
:10377000401C0F49088025B104EB0B000D4908805F
:103780001CE019E0004C00400014014000440040DF
:10379000380000204E6F7420696D706C656D656E29
:1037A000746564210D000000001C004066000020CC
:1037B0006400002060000020F948048000E000BFA1
:1037C00000BFB8F1040F06D0B8F1050F64D0B8F10E
:1037D000060F7DD1C3E00121082038F024F8F1481C
:1037E00039F0D6F9012122200EF084F901208DF85C
:1037F000280002208DF8290000208DF82A008DF87D
:103800002B0022200AF0CBF9099022200AF0C2F9FD
:1038100009A9009037F098FB0A200CF05BFA42F6F9
:10382000E060ADF818000020ADF81A004FF6FF7008
:1038300007900020ADF8200006A9DA4838F0EBFE2A
:103840000020ADF804004FF6FF70039001A9D548A1
:1038500038F013FFD34839F0F6FBD3490988084400
:1038600001460090CF4839F0D6FB0821CD4839F009
:1038700010FC01220821CB4839F071F901220821FE
:10388000C84839F036FB002122200EF033F901211F
:10389000C44839F04AF964E00121082037F0C3FF39
:1038A000C04839F075F901208DF8280002208DF804
:1038B000290000208DF82A008DF82B001E200AF028
:1038C0006EF9099001211E200EF014F91E2000E06F
:1038D00046E00AF05FF909A9009037F035FB0A20AD
:1038E0000CF0F8F942F6E060ADF818000020ADF8F1
:1038F0001A004FF6FF7007900020ADF8200006A9CF
:10390000A84838F088FE0020ADF804004FF6FF709C
:10391000039001A9A34838F0B0FEA24839F093FB08
:10392000A14909880844014600909E4839F073FB7C
:1039300008219C4839F0ADFB01220821994839F053
:103940000EF901220821974839F0D3FA00211E20F0
:103950000EF0D0F80121934839F0E7F801E000E0DB
:1039600000BF00BF00209149088000BF9048008838
:1039700050448E4909888842F8DC0A200CF0AAF9E4
:103980000BB0BDE8F08F10B5FDF749FE8748017810
:103990000120884082490988084028B98348008866
:1039A00083490988884208D1012122200EF0A2F81B
:1039B00001211E200EF09EF807E0002122200EF0CB
:1039C00099F800211E200EF095F878480088401CD8
:1039D000764908800846008875490988884212DDC2
:1039E000012122200EF086F801211E200EF082F81F
:1039F000002208216B4839F0B2F8002208216948FA
:103A000039F077FA0DE0674839F017FB6649098805
:103A100044182146634839F0FEFA0821614839F01C
:103A200038FB10BD10B563480088B0F57A7F04D22A
:103A300060480088401C5F4908800421080739F06D
:103A400014FB0421080739F024FB01220421080794
:103A500039F085F810BD10B521200EF077F840B18F
:103A60005548017801208840544909880843534942
:103A7000088051480088401C4F490880084600884B
:103A8000062819DD4D4801884D484A4A128820F819
:103A900012100020494908804749088007F049FF73
:103AA000484909884FF4FA6292FBF1F144184649FB
:103AB000204607F06DFF0CE007F03BFF4149098805
:103AC0004FF47A7292FBF1F144184049204607F016
:103AD0005FFF10BD10B50421080739F0BDFA78B9B1
:103AE00000203549088007F024FF364909884FF443
:103AF000FA7292FBF1F144183449204607F048FF6E
:103B00000421080739F0B1FA0421080739F0C1FA95
:103B100001220421080739F022F8012204210807B4
:103B200039F0E7F910BD10B50121880739F0A0FA86
:103B300001284FD1FDF773FD1C4801780120884012
:103B400023490988084020B1012122200DF0D2FF2D
:103B500003E0002122200DF0CDFF14480088401C16
:103B600012490880084600881149098888420EDDFC
:103B7000012122200DF0BEFF00220121880738F02C
:103B8000EEFF00214FF0804038F0CFFF03E001212D
:103B9000880739F07EFA0121880739F07AFA57E070
:103BA00060000020000C0040660000206200002041
:103BB00064000020160000206E000020700000202D
:103BC0000408002068000020253A0008573A000841
:103BD0006A0000200421080739F04AFA012835D18B
:103BE00021200DF0B3FF40BB00220421080738F06C
:103BF000B6FF002018490880184908801848008836
:103C000001280DD107F095FE164909884FF47A7204
:103C100092FBF1F144181449204607F0B9FE0CE07C
:103C200007F087FE0F49098840F2DC5292FBF1F160
:103C300044180E49204607F0ABFE0421080739F06E
:103C400014FA0421080739F024FA01E0FDF7E7FC33
:103C500010BD0749087070476E00002070000020FA
:103C60006C00002068000020D53A0008573A000890
:103C70007200002010B5F84801780078401EF64A1E
:103C8000107049B1FDF7CBFC07F053FE0446F34931
:103C900004F5FA7007F07CFE10BD70B52A240025EB
:103CA00000BF3AF033FD0446681CC5B22A2C01D08F
:103CB000032DF6DB2A2C01D1012070BD0020FCE78A
:103CC00070B594B02A24002568463AF099F9044664
:103CD0002A2C20D12820E049087007F02AFE064649
:103CE000DE4906F5FA7007F053FE00BF1198411E39
:103CF00000203BF007FD0446681CC5B22A2C01D009
:103D0000032DF3DB0020D44908702A2C01D014B015
:103D100070BD0120FBE70020F9E710B53AF06CFD1B
:103D2000012800D110BD0020FCE770B594B02A2610
:103D3000CBA00AF045FF68463AF062F90646CCA0EF
:103D40000AF03EFF0C9C200E45B2E8B2FDF7B0FB36
:103D5000200C45B2E8B2FDF7ABFB200A45B2E8B251
:103D6000FDF7A6FB65B2E8B2FDF7A2FBBFA00AF023
:103D700027FFC3A00AF024FF11980AF079FFC4A01E
:103D80000AF01EFF12980AF073FFC6A00AF018FF8F
:103D90009DF808000AF01FFFC6A00AF011FF9DF869
:103DA0001F000AF018FFB1A00AF00AFFC6A00AF02F
:103DB00007FF30460AF00FFFACA00AF001FF14B075
:103DC00070BD7CB504460025C1A00AF0F9FE20466E
:103DD0000BF024F8A5A00AF0F3FE07F077FC0190A1
:103DE0002146019807F03FFD002824D000BF10E0D5
:103DF00001226946019807F0B6FC48B1B6A00AF066
:103E0000DFFE9DF800000AF0B1FFA9A00AF0D8FE7D
:103E10006D1CB5F5007FEBDB94A00AF0D1FEAAA0E3
:103E20000AF0CEFE019807F01BFD06460AF0D3FE0D
:103E30008EA00AF0C5FE01A807F07DFC7CBD77B519
:103E400081B004460D46002607F040FC0090611941
:103E5000009807F008FD48B1012203A9009807F077
:103E6000C5FC18B1009807F0B2FC0646684607F09A
:103E700062FC304604B070BD2DE9F84305460E469D
:103E800017461C464FF0000807F020FC009029461A
:103E9000009807F0E8FC70B13A463146009807F008
:103EA000A5FC40B11CB1009807F0F5FC206000981B
:103EB00007F08DFC8046684607F03DFC4046BDE8B3
:103EC000F8837CB52C2009F06AFE012801D100207E
:103ED00071E02C2009F063FE022801D101206AE084
:103EE0002C2009F05CFE042801D1022063E02C2084
:103EF00009F055FE082801D103205CE02C2009F0D0
:103F00004EFE102801D1042055E02C2009F047FE78
:103F1000202801D105204EE02C2009F040FE402849
:103F200001D1062047E02C2009F039FE802801D17C
:103F3000072040E02C2009F032FEB0F5807F01D14F
:103F4000082038E02C2009F02AFEB0F5007F01D1CE
:103F5000092030E02C2009F022FEB0F5806F01D15D
:103F60000A2028E02C2009F01AFEB0F5006F01D1DC
:103F70000B2020E02C2009F012FEB0F5805F01D16B
:103F80000C2018E02C2009F00AFEB0F5005F01D1EA
:103F90000D2010E02C2009F002FEB0F5804F01D179
:103FA0000E2008E02C2009F0FAFDB0F5004F01D1F9
:103FB0000F2000E0FF2004462C2009F0EBFD054611
:103FC0000C22214637F043F82B2009F0E8FD0128A8
:103FD00001D10020B3E02B2009F0E1FD022801D13E
:103FE0000120ACE02B2009F0DAFD042801D10220E9
:103FF000A5E02B2009F0D3FD082801D103209EE085
:104000002B2009F0CCFD102801D1042097E02B20B3
:1040100009F0C5FD202801D1052090E02B2009F0F2
:10402000BEFD402801D1062089E02B2009F0B7FD14
:10403000802801D1072082E02B2009F0B0FDB0F5E7
:10404000807F01D108207AE02B2009F0A8FDB0F58F
:10405000007F43D1092072E073000020753C000806
:104060004765742043617264696E666F0D000000DD
:1040700050726F644E616D6531203D20000000007C
:104080004361726443617061636974793D2000002B
:104090000D43617264426C6F636B53697A653D20B6
:1040A000000000000D5264426C6F636B4C656E3D06
:1040B000200000000D4D61785772426C6F636B4CAD
:1040C000656E3D20000000005374617475733D00FF
:1040D0005265616420534420307800002B2009F0A1
:1040E0005EFDB0F5806F01D10A2028E02B2009F099
:1040F00056FDB0F5006F01D10B2020E02B2009F018
:104100004EFDB0F5805F01D10C2018E02B2009F0A6
:1041100046FDB0F5005F01D10D2010E02B2009F025
:104120003EFDB0F5804F01D10E2008E02B2009F0B4
:1041300036FDB0F5004F01D10F2000E0FF2004460E
:104140002B2009F027FD05460C22214636F07FFF83
:104150002A2009F024FD012801D1002071E02A2045
:1041600009F01DFD022801D101206AE02A2009F092
:1041700016FD042801D1022063E02A2009F00FFD7A
:10418000082801D103205CE02A2009F008FD10284E
:1041900001D1042055E02A2009F001FD202801D199
:1041A00005204EE02A2009F0FAFC402801D1062023
:1041B00047E02A2009F0F3FC802801D1072040E0E5
:1041C0002A2009F0ECFCB0F5807F01D1082038E00E
:1041D0002A2009F0E4FCB0F5007F01D1092030E08D
:1041E0002A2009F0DCFCB0F5806F01D10A2028E01C
:1041F0002A2009F0D4FCB0F5006F01D10B2020E09B
:104200002A2009F0CCFCB0F5805F01D10C2018E029
:104210002A2009F0C4FCB0F5005F01D10D2010E0A8
:104220002A2009F0BCFCB0F5804F01D10E2008E037
:104230002A2009F0B4FCB0F5004F01D10F2000E0B6
:10424000FF2004462A2009F0A5FC05460C22214641
:1042500036F0FDFE292009F0A2FC012801D1002042
:1042600071E0292009F09BFC022801D101206AE0BD
:10427000292009F094FC042801D1022063E02920C0
:1042800009F08DFC082801D103205CE0292009F009
:1042900086FC102801D1042055E0292009F07FFC7C
:1042A000202801D105204EE0292009F078FC402883
:1042B00001D1062047E0292009F071FC802801D1B6
:1042C000072040E0292009F06AFCB0F5807F01D189
:1042D000082038E0292009F062FCB0F5007F01D108
:1042E000092030E0292009F05AFCB0F5806F01D197
:1042F0000A2028E0292009F052FCB0F5006F01D116
:104300000B2020E0292009F04AFCB0F5805F01D1A4
:104310000C2018E0292009F042FCB0F5005F01D123
:104320000D2010E0292009F03AFCB0F5804F01D1B2
:104330000E2008E0292009F032FCB0F5004F01D131
:104340000F2000E0FF200446292009F023FC054649
:104350000C22214636F07BFE282009F020FC0128A3
:1043600001D1002071E0282009F019FC022801D1B8
:1043700001206AE0282009F012FC042801D1022063
:1043800063E0282009F00BFC082801D103205CE041
:10439000282009F004FC102801D1042055E0282031
:1043A00009F0FDFB202801D105204EE0282009F06E
:1043B000F6FB402801D1062047E0282009F0EFFB5A
:1043C000802801D1072040E0282009F0E8FBB0F563
:1043D000807F01D1082038E0282009F0E0FBB0F50B
:1043E000007F01D1092030E0282009F0D8FBB0F58A
:1043F000806F01D10A2028E0282009F0D0FBB0F519
:10440000006F01D10B2020E0282009F0C8FBB0F597
:10441000805F01D10C2018E0282009F0C0FBB0F526
:10442000005F01D10D2010E0282009F0B8FBB0F5A5
:10443000804F01D10E2008E0282009F0B0FBB0F534
:10444000004F01D10F2000E0FF200446282009F092
:10445000A1FB05460C22214636F0F9FD272009F084
:104460009EFB012801D1002071E0272009F097FB75
:10447000022801D101206AE0272009F090FB0428DE
:1044800001D1022063E0272009F089FB082801D12F
:1044900003205CE0272009F082FB102801D10420D2
:1044A00055E0272009F07BFB202801D105204EE0B4
:1044B000272009F074FB402801D1062047E027207F
:1044C00009F06DFB802801D1072040E0272009F08A
:1044D00066FBB0F5807F01D1082038E0272009F085
:1044E0005EFBB0F5007F01D1092030E0272009F004
:1044F00056FBB0F5806F01D10A2028E0272009F093
:104500004EFBB0F5006F01D10B2020E0272009F011
:1045100046FBB0F5805F01D10C2018E0272009F0A0
:104520003EFBB0F5005F01D10D2010E0272009F01F
:1045300036FBB0F5804F01D10E2008E0272009F0AE
:104540002EFBB0F5004F01D10F2000E0FF20044604
:10455000272009F01FFB05460C22214636F077FD87
:1045600003208DF8050002208DF8040000208DF84E
:10457000060001208DF807002C2009F010FB0090A8
:104580002C2009F007FB0446694636F0DDFC2B20A1
:1045900009F005FB00902B2009F0FCFA044669465F
:1045A00036F0D2FC2A2009F0FAFA00902A2009F00D
:1045B000F1FA0446694636F0C7FC292009F0EFFA03
:1045C0000090292009F0E6FA0446694636F0BCFC62
:1045D000272009F0E4FA0090272009F0DBFA0446CE
:1045E000694636F0B1FC282009F0D9FA0090002085
:1045F0008DF80700282009F0CDFA0446694636F008
:10460000A3FC00208DF8040001208DF80700412054
:1046100009F0C5FA0090412009F0BCFA0446694649
:1046200036F092FC0121C80237F00EF9012188050D
:1046300037F0C6F87CBD7CB5002039F0A9F9002020
:1046400039F0A9F939F07CF900214FF4006037F016
:10465000FBF82C2009F0A3FA012801D1002071E019
:104660002C2009F09CFA022801D101206AE02C20BC
:1046700009F095FA042801D1022063E02C2009F00A
:104680008EFA082801D103205CE02C2009F087FA7B
:10469000102801D1042055E02C2009F080FA2028B0
:1046A00001D105204EE02C2009F079FA402801D1F3
:1046B000062047E02C2009F072FA802801D107205B
:1046C00040E02C2009F06BFAB0F5807F01D1082082
:1046D00038E02C2009F063FAB0F5007F01D1092001
:1046E00030E02C2009F05BFAB0F5806F01D10A2090
:1046F00028E02C2009F053FAB0F5006F01D10B200F
:1047000020E02C2009F04BFAB0F5805F01D10C209D
:1047100018E02C2009F043FAB0F5005F01D10D201C
:1047200010E02C2009F03BFAB0F5804F01D10E20AB
:1047300008E02C2009F033FAB0F5004F01D10F202A
:1047400000E0FF2004462C2009F024FA0546002250
:10475000214636F07CFC2B2009F021FA012801D1FA
:10476000002071E02B2009F01AFA022801D1012063
:104770006AE02B2009F013FA042801D1022063E03B
:104780002B2009F00CFA082801D103205CE02B2033
:1047900009F005FA102801D1042055E02B2009F07A
:1047A000FEF9202801D105204EE02B2009F0F7F971
:1047B000402801D1062047E02B2009F0F0F980289D
:1047C00001D1072040E02B2009F0E9F9B0F5807F06
:1047D00001D1082038E02B2009F0E1F9B0F5007F85
:1047E00001D1092030E02B2009F0D9F9B0F5806F14
:1047F00001D10A2028E02B2009F0D1F9B0F5006F93
:1048000001D10B2020E02B2009F0C9F9B0F5805F21
:1048100001D10C2018E02B2009F0C1F9B0F5005FA0
:1048200001D10D2010E02B2009F0B9F9B0F5804F2F
:1048300001D10E2008E02B2009F0B1F9B0F5004FAE
:1048400001D10F2000E0FF2004462B2009F0A2F93F
:1048500005460022214636F0FAFB2A2009F09FF98E
:10486000012801D1002071E02A2009F098F90228DE
:1048700001D101206AE02A2009F091F9042801D130
:10488000022063E02A2009F08AF9082801D10320D8
:104890005CE02A2009F083F9102801D1042055E0BA
:1048A0002A2009F07CF9202801D105204EE02A2099
:1048B00009F075F9402801D1062047E02A2009F0C7
:1048C0006EF9802801D1072040E02A2009F067F91D
:1048D000B0F5807F01D1082038E02A2009F05FF987
:1048E000B0F5007F01D1092030E02A2009F057F906
:1048F000B0F5806F01D10A2028E02A2009F04FF995
:10490000B0F5006F01D10B2020E02A2009F047F913
:10491000B0F5805F01D10C2018E02A2009F03FF9A2
:10492000B0F5005F01D10D2010E02A2009F037F921
:10493000B0F5804F01D10E2008E02A2009F02FF9B0
:10494000B0F5004F01D10F2000E0FF2004462A20DF
:1049500009F020F905460022214636F078FB29208F
:1049600009F01DF9012801D1002071E0292009F08A
:1049700016F9022801D101206AE0292009F00FF977
:10498000042801D1022063E0292009F008F9082851
:1049900001D103205CE0292009F001F9102801D1A0
:1049A000042055E0292009F0FAF8202801D105203B
:1049B0004EE0292009F0F3F8402801D1062047E015
:1049C000292009F0ECF8802801D1072040E02920B7
:1049D00009F0E5F8B0F5807F01D1082038E0292002
:1049E00009F0DDF8B0F5007F01D1092030E0292081
:1049F00009F0D5F8B0F5806F01D10A2028E0292010
:104A000009F0CDF8B0F5006F01D10B2020E029208E
:104A100009F0C5F8B0F5805F01D10C2018E029201D
:104A200009F0BDF8B0F5005F01D10D2010E029209C
:104A300009F0B5F8B0F5804F01D10E2008E029202B
:104A400009F0ADF8B0F5004F01D10F2000E0FF20D4
:104A50000446292009F09EF805460022214636F03A
:104A6000F6FA282009F09BF8012801D1002071E016
:104A7000282009F094F8022801D101206AE02820BA
:104A800009F08DF8042801D1022063E0282009F004
:104A900086F8082801D103205CE0282009F07FF87F
:104AA000102801D1042055E0282009F078F82028AA
:104AB00001D105204EE0282009F071F8402801D1ED
:104AC000062047E0282009F06AF8802801D1072055
:104AD00040E0282009F063F8B0F5807F01D108207C
:104AE00038E0282009F05BF8B0F5007F01D10920FB
:104AF00030E0282009F053F8B0F5806F01D10A208A
:104B000028E0282009F04BF8B0F5006F01D10B2008
:104B100020E0282009F043F8B0F5805F01D10C2097
:104B200018E0282009F03BF8B0F5005F01D10D2016
:104B300010E0282009F033F8B0F5804F01D10E20A5
:104B400008E0282009F02BF8B0F5004F01D10F2024
:104B500000E0FF200446282009F01CF8054600224A
:104B6000214636F074FA272009F019F8012801D1FE
:104B7000002071E0272009F012F8022801D101205D
:104B80006AE0272009F00BF8042801D1022063E035
:104B9000272009F004F8082801D103205CE0272031
:104BA00008F0FDFF102801D1042055E0272008F06F
:104BB000F6FF202801D105204EE0272008F0EFFF66
:104BC000402801D1062047E0272008F0E8FF802890
:104BD00001D1072040E0272008F0E1FFB0F5807FF9
:104BE00001D1082038E0272008F0D9FFB0F5007F78
:104BF00001D1092030E0272008F0D1FFB0F5806F07
:104C000001D10A2028E0272008F0C9FFB0F5006F85
:104C100001D10B2020E0272008F0C1FFB0F5805F14
:104C200001D10C2018E0272008F0B9FFB0F5005F93
:104C300001D10D2010E0272008F0B1FFB0F5804F22
:104C400001D10E2008E0272008F0A9FFB0F5004FA1
:104C500001D10F2000E0FF200446272008F09AFF32
:104C600005460022214636F0F2F900208DF80400B6
:104C70008DF807002C2008F092FF00902C2008F0FF
:104C800089FF0446694636F05FF92B2008F087FF5C
:104C900000902B2008F07EFF0446694636F054F958
:104CA0002A2008F07CFF00902A2008F073FF0446B9
:104CB000694636F049F9292008F071FF0090292053
:104CC00008F068FF0446694636F03EF9272008F0F0
:104CD00066FF0090272008F05DFF0446694636F025
:104CE00033F9282008F05BFF0090282008F052FFDD
:104CF0000446694636F028F97CBD30B58FB00446CD
:104D00000D464FF0FA513E4837F076FB00213C4803
:104D100037F0DCFA3A4837F0FBF94FF000600090CA
:104D200038480190029440200390002004900590A0
:104D30004FF480600690800007908000089000206B
:104D400009904FF440300A9004200B9003200C90FF
:104D50004FF400000D9080100E906946284837F0FF
:104D600079FA2021264837F0EFFA0121244837F05C
:104D7000ADFA0FB030BD30B58FB004460D464FF0E0
:104D8000FA511F4837F038FB00211D4837F09EFAD2
:104D90001B4837F0BDF94FF00060009019480190B2
:104DA000029400200390049005904FF480600690D8
:104DB0008000079080000890002009904FF4403058
:104DC0000A9004200B9003200C904FF400000D90EB
:104DD00080100E9069460A4837F03CFA20210848B6
:104DE00037F0B2FA0121064837F070FA0FB030BD43
:104DF00010B54FF0C051024837F0E2FA10BD000084
:104E000058640240802C014010B504462146FE48FB
:104E100038F001F910BD10B504462146FA4838F0C3
:104E2000FCF810BD10B504462146F74838F0F1F8FB
:104E300010BD10B50024F5480078F449497888423F
:104E400021D0F248007800F00100E8B1EF48007886
:104E500000F03E00C0B91E20ED49088000BF08E008
:104E60000620EC4901F814000F2001EB44014870C2
:104E7000641C282CF4D300F0B4FF00F0B9FFE34821
:104E80000078E2494870D7E2E048007800F003007B
:104E900003281DD1DD48007800F03C00C0B91E2079
:104EA000DB490880002408E00320DA4901F81400F7
:104EB0000F2001EB44014870641C282CF4D300F04F
:104EC00090FF00F095FFD1480078D0494870B3E2D8
:104ED000CE48007800F0050005281DD1CB480078A9
:104EE00000F02800C0B91E20C9490880002408E04D
:104EF0000520C84901F814000F2001EB4401487057
:104F0000641C282CF4D300F06CFF00F071FFBF4844
:104F10000078BE4948708FE2BC48007800F00D0070
:104F20000D2837D1B948007800F0200088BBFF2059
:104F3000B7490880002404E00520B64901F81400B0
:104F4000641C282CF8D3002418E008222046641C96
:104F5000B04901EB4000427004222046641C01EB82
:104F60004000427002222046641C01EB4000427067
:104F700001222046641C01EB40004270282CE4D33F
:104F800000F02FFF00F034FFA04800789F494870E0
:104F900052E2FFE79D48007800F01300132843D148
:104FA0009A48007800F02C0000283DD14FF47A7028
:104FB00097490880002422E002222046641C95497B
:104FC00001F810202046641C01F810202046641CC3
:104FD00001F810202046641C01F81020032220460E
:104FE000641C01F810202046641C01F810202046A3
:104FF000641C01F810202046641C01F81020282CA5
:10500000DAD3002405E00F20824901EB4401487007
:10501000641C282CF7D300F0E4FE00F0E9FE7B4886
:1050200000787A49487007E27848007800F031004B
:10503000312845D17548007800F00E0000283FD196
:10504000002408E00220734901F814000F2001EB4E
:1050500044014870641C282CF4D300206D498870EA
:1050600001200871002088710120087200208872D8
:1050700001200873002088730120087400208874C0
:1050800081F82800032081F82A0081F82C000020F4
:1050900081F82E0081F83000032081F8320081F879
:1050A0003400002081F8360000F065FE00F083FE39
:1050B0000020594908705548007854494870BBE1B0
:1050C0005248007800F01100112833D14F48007881
:1050D00000F02E0070BB002408E002204D4901F8CA
:1050E00014000F2001EB44014870641C282CF4D3F9
:1050F0000020484981F82800032081F82A0081F81F
:105100002C00002081F82E0081F83000032081F867
:10511000320081F83400002081F8360000F04BFEA8
:1051200000F05FFE00203C4908703848007837499D
:10513000487081E13548007800F02100212830D105
:105140003248007800F01E0058BB002408E006201A
:10515000304901F814000F2001EB44014870641C31
:10516000282CF4D300202B498870012008710020DE
:1051700088710120087200208872012008730020C5
:105180008873012008740020887400F0F4FD00F09A
:105190002FFE0020204908701C4800781B494870E9
:1051A0004AE11A48007800F0310031283CD1174814
:1051B000007800F00E0088BB002408E002201549AA
:1051C00001F814000F2001EB44014870641C282CE6
:1051D000F4D300200F4988700120087100208871E5
:1051E0000120087200208872012008730020887353
:1051F000012008740020887400F0BDFD00F0F8FD67
:105200000020054908700AE00004004084000020E6
:1052100080000020822800208300002004E0F7485E
:105220000078F649487007E1F448007800F0330050
:10523000332855D1F148007800F00C0000284FD1F8
:10524000002422E002222046641CED4901F81020CF
:105250002046641C01F810202046641C01F8102030
:105260002046641C01F8102003222046641C01F82B
:1052700010202046641C01F810202046641C01F810
:1052800010202046641C01F81020282CDAD30024BA
:1052900005E00F20DA4901EB44014870641C282C1A
:1052A000F7D30020D649887001200871002088714A
:1052B0000120087200208872012008730020887382
:1052C000012008740020887400F055FD00F090FD66
:1052D0000020CC490870C9480078C8494870ABE044
:1052E000C648007800F02300232831D1C348007855
:1052F00000F01C0060BB002400BF08E00320C04990
:1053000001F814000F2001EB44014870641C282CA4
:10531000F4D30020BA4988700120087100208871F8
:105320000120087200208872012008730020887311
:10533000012008740020887400F01DFD00F058FD65
:105340000020B0490870AD480078AC49487073E05F
:10535000AA48007800F02500252858D1FF20AA4946
:105360000880002405E005222046641CA44901F8B9
:105370001020282CF7D3002418E008222046641CB3
:105380009F4901EB4000427004222046641C01EB5F
:105390004000427002222046641C01EB4000427033
:1053A00001222046641C01EB40004270282CE4D30B
:1053B000002093498870012008710F2190484171A5
:1053C00000208F498871012008720F218C4841729A
:1053D00000208B498872012008730F21884841738F
:1053E000002087498873012008740F218448417484
:1053F00000208349887400F0BEFC00F0F9FC002016
:10540000804908707D4800787C49487014E0002489
:1054100008E000207A4901F814000F2001EB440154
:105420004870641C282CF4D300F0DBFC00F0E0FC96
:10543000724800787149487010BD10B5044604F0F8
:10544000080020B1012108460CF054FB03E00021C4
:1054500001200CF04FFB04F0040020B101210220D8
:105460000CF048FB03E0002102200CF043FB04F0A9
:10547000020020B1012103200CF03CFB03E00021DD
:1054800003200CF037FB04F0010020B101210420BF
:105490000CF030FB03E0002104200CF02BFB10BDCE
:1054A0005A4800787047594908707047584B18801F
:1054B000584B1A80584B1980704770B588B000243B
:1054C00001204E4908700020487054490880504916
:1054D00008805349088050490880524908804D4946
:1054E00008801E2048490880002046490870464828
:1054F0000088454908804A4800884949088047484B
:1055000000884649088047480088464908800020AE
:105510003E4908700121022036F085F9052008F087
:105520003EFB012801D1002087E0052008F037FB71
:10553000022801D1012080E0052008F030FB04287A
:1055400001D1022079E0052008F029FB082801D1CB
:10555000032072E0052008F022FB102801D104206E
:105560006BE0052008F01BFB202801D1052064E03A
:10557000052008F014FB402801D106205DE005203D
:1055800008F00DFB802801D1072056E0052008F027
:1055900006FBB0F5807F01D108204EE0052008F021
:1055A000FEFAB0F5007F01D1092046E0052008F0A1
:1055B000F6FAB0F5806F01D10A203EE0052008F030
:1055C000EEFAB0F5006F01D10B2036E0052008F0AF
:1055D000E6FAB0F5805F01D10C202EE0052008F03E
:1055E000DEFAB0F5005F01D10D2026E0052008F0BD
:1055F000D6FAB0F5804F17D10E201EE084000020AF
:1056000082280020830000208000002082000020EB
:105610007A0000207E0000207C0000207400002022
:105620007600002078000020052008F0B8FAB0F5D8
:10563000004F01D10F2000E0FF200546052008F0B3
:10564000A9FA06460222294635F001FD062008F097
:10565000A6FA012801D1002071E0062008F09FFA87
:10566000022801D101206AE0062008F098FA0428F7
:1056700001D1022063E0062008F091FA082801D148
:1056800003205CE0062008F08AFA102801D10420EB
:1056900055E0062008F083FA202801D105204EE0CD
:1056A000062008F07CFA402801D1062047E00620B9
:1056B00008F075FA802801D1072040E0062008F0A4
:1056C0006EFAB0F5807F01D1082038E0062008F09E
:1056D00066FAB0F5007F01D1092030E0062008F01D
:1056E0005EFAB0F5806F01D10A2028E0062008F0AC
:1056F00056FAB0F5006F01D10B2020E0062008F02B
:105700004EFAB0F5805F01D10C2018E0062008F0B9
:1057100046FAB0F5005F01D10D2010E0062008F038
:105720003EFAB0F5804F01D10E2008E0062008F0C7
:1057300036FAB0F5004F01D10F2000E0FF200546FA
:10574000062008F027FA06460222294635F07FFC9B
:10575000072008F024FA012801D1002071E0072079
:1057600008F01DFA022801D101206AE0072008F0A4
:1057700016FA042801D1022063E0072008F00FFA8E
:10578000082801D103205CE0072008F008FA10285F
:1057900001D1042055E0072008F001FA202801D1AA
:1057A00005204EE0072008F0FAF9402801D1062034
:1057B00047E0072008F0F3F9802801D1072040E0F6
:1057C000072008F0ECF9B0F5807F01D1082038E01F
:1057D000072008F0E4F9B0F5007F01D1092030E09E
:1057E000072008F0DCF9B0F5806F01D10A2028E02D
:1057F000072008F0D4F9B0F5006F01D10B2020E0AC
:10580000072008F0CCF9B0F5805F01D10C2018E03A
:10581000072008F0C4F9B0F5005F01D10D2010E0B9
:10582000072008F0BCF9B0F5804F01D10E2008E048
:10583000072008F0B4F9B0F5004F01D10F2000E0C7
:10584000FF200546072008F0A5F906460222294652
:1058500035F0FDFB714800687149B0FBF1F0401E66
:1058600084B24FF47A700690ADF814400020ADF881
:105870001C00ADF8160005A96A4836F0CCFE602081
:10588000ADF800000120ADF8020000200290ADF854
:105890000C006946634836F023FF0821614837F061
:1058A0006CFA0020029069465E4836F05EFF0821DF
:1058B0005C4837F06EFA002002906946594836F08D
:1058C00097FF0821574837F06CFA0121554837F007
:1058D0002CF908B070BD10B553480088FFF7A2FA44
:1058E00052480088FFF797FA51480088FFF78CFA72
:1058F00010BD10B5FBF757FE30B14E48007840F0B0
:1059000002004C49087005E04A48007820F0020087
:105910004849087009F0EDF830B14648007840F089
:1059200020004449087005E04248007820F020003B
:10593000404908704048007830B13E48007840F057
:1059400010003C49087005E03A48007820F010004B
:1059500038490870FFF76DFA38483949097810F866
:105960001100072837D2DFE800F0040A11181F26BB
:105970002E00002211461046FFF798FD2BE0002272
:1059800011464FF47A70FFF791FD24E000224FF4A6
:105990007A711046FFF78AFD1DE04FF47A720021FC
:1059A0000846FFF783FD16E04FF47A720021104697
:1059B000FFF77CFD0FE000224FF47A714FF42F7057
:1059C000FFF774FD07E04FF416724FF47A7110463A
:1059D000FFF76CFD00BF00BF1849194A127801EBB0
:1059E00042014878FFF729FD15480078401C14490A
:1059F000087008460078282801D30020087010BDE0
:105A000029B10C4A127802430A4B1A7004E0094A81
:105A100012788243074B1A70704700001803002069
:105A200080841E00000400407A0000207C000020DA
:105A30007E000020840000205100002082280020E9
:105A40008300002010B504462146FE4837F0DFFAF7
:105A500010BD10B50446A1B20122FA4837F007F98B
:105A600010BD70B504460D468020FFF7EBFFF648E9
:105A700090FBF4F63046FFF7ECFFF448058070BD6C
:105A800010B5F348008840B1F1480188F14800881A
:105A9000FFF7E7FF0020EE49088010BD30B589B060
:105AA0000020ED4908700121080235F0BCFE3C20C1
:105AB00008F075F8012801D1002071E03C2008F0C1
:105AC0006EF8022801D101206AE03C2008F067F856
:105AD000042801D1022063E03C2008F060F8082887
:105AE00001D103205CE03C2008F059F8102801D1D6
:105AF000042055E03C2008F052F8202801D1052070
:105B00004EE03C2008F04BF8402801D1062047E049
:105B10003C2008F044F8802801D1072040E03C20D8
:105B200008F03DF8B0F5807F01D1082038E03C2036
:105B300008F035F8B0F5007F01D1092030E03C20B5
:105B400008F02DF8B0F5806F01D10A2028E03C2044
:105B500008F025F8B0F5006F01D10B2020E03C20C3
:105B600008F01DF8B0F5805F01D10C2018E03C2052
:105B700008F015F8B0F5005F01D10D2010E03C20D1
:105B800008F00DF8B0F5804F01D10E2008E03C2060
:105B900008F005F8B0F5004F01D10F2000E0FF201C
:105BA00004463C2007F0F6FF05460922214635F061
:105BB0004EFA3B20ADF81800FF2007900020ADF80A
:105BC0002000ADF81A0006A99E4836F024FD60209A
:105BD000ADF804000120ADF8060000200390ADF8F8
:105BE000100001A9974836F048FD0821954837F084
:105BF000BCF80121934836F098FF0020FFF722FF00
:105C000009B030BD9148008810B99148008808B1AA
:105C1000012070470020FCE78D4A11808D4A1080DA
:105C2000704710B50F2140F2DC50FFF71AFF322009
:105C30000AF050F80F214FF4D460FFF712FF19203B
:105C40000AF048F80F2140F29E70FFF70AFF192072
:105C50000AF040F80F2140F67700FFF702FF192005
:105C60000AF038F80F2140F68510FFF7FAFE1920E8
:105C70000AF030F80F2140F6E220FFF7F2FE19207B
:105C80000AF028F80F2140F6B240FFF7EAFE19208B
:105C90000AF020F80F2140F63C70FFF7E2FE10BD3D
:105CA00010B56EA005F0EEF964219620FFF7D9FE3D
:105CB00064200AF00FF8C8217320FFF7D2FE10BD50
:105CC00010B50F2140F63C70FFF7CBFE32200AF0F2
:105CD00001F80F2140F6B240FFF7C3FE192009F08A
:105CE000F9FF0F2140F6E220FFF7BBFE192009F073
:105CF000F1FF0F2140F68510FFF7B3FE192009F0E0
:105D0000E9FF0F2140F69500FFF7ABFE192009F0DF
:105D1000E1FF0F2140F29E70FFF7A3FE192009F06A
:105D2000D9FF0F214FF4D460FFF79BFE192009F033
:105D3000D1FF0F2140F2DC50FFF793FE10BD10B5EC
:105D400000BFFFF75FFF0028FBD14FF4487009F058
:105D5000C1FF4DA005F096F910BD10B500BFFFF7CB
:105D600051FF0028FBD14FF4487009F0B3FF50A059
:105D700005F088F910BD32205C4908814FF45C7150
:105D80005A4841813220594908824FF45C71574882
:105D900041823220554908834FF45C715348418356
:105DA0003220524908844FF45C71504841840020ED
:105DB00029490870704764204C49A1F854004FF4F9
:105DC000DC614A48A0F8561064204849A1F86400F4
:105DD0004FF4DC614548A0F8661000201E490870A9
:105DE0007047002041490881088208830884704771
:105DF00000203E49A1F85400A1F85C00A1F864001D
:105E0000A1F86C00704710B538481349097830F88C
:105E1000210000280BDD354A0F4B1B7832F8231088
:105E20000D4B1B7802EB83025088FFF71AFE0A48DD
:105E30000078401C0849087008460078282858D384
:105E4000002055E000200040109203008600002052
:105E5000880000208A0000208C0000205553423A20
:105E6000643D382C6F3D352C623D3136303A313649
:105E7000612C3136672C3136612C313661232C632D
:105E8000362C6336000000004672656353746172FD
:105E9000743A643D382C6F3D362C623D3136303AD1
:105EA000632C642C6123352C642C326600000000C6
:105EB000467265634661696C65643A643D382C6F6F
:105EC0003D362C623D3136303A632C642C612335EB
:105ED0002C642C702C63342C702C63342C702C6349
:105EE000342C702C63342C702C633400D2280020A6
:105EF000087010BD10B50948008800280ADD074861
:105F00000088401E80B20549088028B90020FFF7AC
:105F100099FD01E0FFF7B4FD10BD000086000020F0
:105F200010B586B0FBF77BFB01A9012000F0C4FD92
:105F3000FE48007808B1032400E008249DF804001E
:105F40004FF60C7108408DF804009DF8040040EAFB
:105F50000410C0B28DF8040030208DF80C00F44815
:105F600001788DF80D10F34801788DF80E1000219E
:105F70008DF80F108DF810108DF811108DF812108B
:105F80008DF8131001A9012000F0F1FC4FF4967078
:105F900009F0AEFE0121084600F0BEFE06B010BDBD
:105FA0002DE9FC4105460F461446681EC6B20B2D6E
:105FB00002D00E2D64D11CE00821DF4837F0D7FB5A
:105FC00058B10822DD4928460BF0CCFE28460BF0DC
:105FD000E5FE0220DA4908700AE028460BF038FE98
:105FE0003A46214628460BF0BDFE0220D4490870EF
:105FF000CBE00821D04837F0BAFB58B10822CF498E
:1060000028460BF0AFFE28460BF0C8FE0220CD4913
:10601000087034E001A9601C14F044FD8046B8F11A
:10602000000F07D09DF80400782803D10020C6494E
:10603000086023E0002000900822214628460BF04B
:1060400091FE18B1694628460BF0CDFE9DF8000080
:10605000812806D10120BB4908700020BA49086098
:1060600002E00220B7490870607830B9A07820B902
:10607000E07810B90220B349087000BF00BF84E087
:106080000821AD4837F073FB40B10722AB492846E1
:106090000BF068FE28460BF081FE75E0207800F0DA
:1060A000F000202822D1A9480088401CA749088078
:1060B0000722611C28460BF02BFE022804D1A049C0
:1060C0000870A34988555FE09948007800285BDD97
:1060D0009E48008896490978884255DBFFF720FFE3
:1060E00000209A4908809B4908604DE0207800F024
:1060F000F000A0B9207800F00F0828460BF0A8FDAA
:106100004346621C414628460BF0C7FD601C14F054
:10611000C2FC02208E4988558949087034E02078F5
:1061200000F0F00010281CD16078217801F00F01F8
:1061300000EB012800208549088028460BF088FDE7
:1061400041460623A21C28460BF0A7FD01208049EA
:1061500088557B490870FFF7E3FE00207D49086001
:1061600012E0207800F0F00030280DD101207A49AB
:106170000870207800F00F0078490870607878493E
:106180000870A0787749087000BF00BFBDE8FC81A7
:1061900010B586B0FBF743FA01A9012000F08CFC92
:1061A0006248007808B1042400E008249DF8040047
:1061B0004FF60C7108408DF804009DF8040040EA89
:1061C0000410C0B28DF80400674800788DF80C0008
:1061D00030218DF80D10564801788DF80E10554875
:1061E00001788DF80F1000218DF810108DF8111026
:1061F0008DF812108DF8131001A9012000F0B7FBE3
:106200000121084600F088FD06B010BD2DE9F041DF
:10621000064688461446701EC5B20821464837F027
:10622000A6FA40B10722454930460BF09BFD3046A7
:106230000BF0B4FD9BE0607800F0F000202826D140
:1062400042480088401C414908800622A11C304673
:106250000BF05EFD022804D1394908703C494855CD
:1062600085E033480078002810DD38480088304940
:10627000097888427BDB4FF4167009F039FDFFF78F
:1062800087FF002031490880324908606FE060785C
:1062900000F0F000A0B9607800F00F0730460BF076
:1062A000D7FC3B46A21C394630460BF0F6FCA01C3E
:1062B00014F0F1FB0220264948552149087056E0A8
:1062C000607800F0F00010281DD1A078617801F00E
:1062D0000F0100EB012700201C49088030460BF01D
:1062E000B7FC39460523E21C30460BF0D6FC0120F2
:1062F00017494855124908704FF4167009F0F8FC18
:10630000FFF746FF33E0607800F0F00030282ED130
:10631000012011490870607800F00F000F490870E3
:10632000A0780F490870E0780E491FE00C020020A9
:10633000BA010020BB0100200068004035160408A7
:10634000B801002000020020380000208E0000204C
:106350005C24012044000020FC010020FD010020FD
:10636000FE010020FF010020060200200870BDE8A9
:10637000F08170B504460E461546022C1FD1082147
:10638000FE4837F0F4F958B120460BF061FC0822C2
:10639000FB4920460BF0E6FC20460BF0FFFC0DE02D
:1063A0000822294620460BF0DDFC38B920460BF0C8
:1063B0004FFC0822294620460BF0D4FC00E000BF29
:1063C00000BF70BD2DE9FC4105460F461446102D57
:1063D00070D2DFE805F0E8090A2D77E8E80B2E789F
:1063E000E8E8E8E8E808DFE0DEE000BF0821E3488D
:1063F00037F0BDF928B1FF20E2494880012008802C
:1064000015E02078DF49488060788880A078C880CF
:10641000E07808812079488160798881A079C881F5
:10642000E0790882082008800220D7490870BBE084
:1064300000BF0821D14837F09AF928B1FF20D1498F
:106440004880012008803CE02078102825D1617820
:10645000A07801EB0020CD490880E078CC49087095
:106460000020CC490870032D0AD1FF2000900123A1
:106470000190C748027811210D2027F0E1F820E0B3
:10648000082D1ED1FF20009001230190C048027802
:1064900011210E2027F0D4F813E0207811280AD11A
:1064A0000120BD4908706078BC490870A078BC49DB
:1064B000087006E077E02078132802D10120B9495E
:1064C000087071E000BF0821AC4837F050F900288F
:1064D00068D16178AB480088401CAA4A22F81010A5
:1064E000A17810460088801C22F81010E178104630
:1064F0000088C01C22F81010217910460088001D69
:1065000022F81010617910460088401D22F8101002
:10651000A17910460088801D22F81010E1791046FC
:106520000088C01D22F8101010460088C01D1146BA
:10653000088098480078401C964908700846007802
:106540009349097888422DD1042D11D1FF2091491A
:106550000978CDE900108D480678F01706EB106039
:1065600003128A48027813210D2027F069F812E0FF
:10657000092D10D1FF2087490978CDE90010834803
:106580000678F01706EB106003128048027813219A
:106590000E2027F055F802207B4908707B480088C0
:1065A0007849088000E000BF00BFBDE8FC8170476B
:1065B00070471CB5FBF733F830208DF800007A489F
:1065C00000788DF80100794800788DF802000020ED
:1065D0008DF803008DF804008DF805008DF8060095
:1065E0008DF807006946012000F03FFB012000F014
:1065F000CCFB1CBD2DE9F84305460F461446681E2A
:10660000C6B20B2D02D00E2D52D11CE008215B48E2
:1066100037F0ADF858B10822594928460BF0A2FBD3
:1066200028460BF0BBFB0220574908700AE02846B9
:106630000BF00EFB3A46214628460BF093FB022056
:1066400051490870C3E008214C4837F090F858B120
:1066500008224B4928460BF085FB28460BF09EFB91
:1066600002205349087022E00020009008222146B1
:1066700028460BF077FB694628460BF0B4FB9DF8E3
:106680000000812806D101204949087000204949AD
:10669000086002E0022046490870607830B9A078AE
:1066A00020B9E07810B902204149087000BF8EE09F
:1066B0000821324837F05BF840B1072230492846BC
:1066C0000BF050FB28460BF069FB7FE0207800F0D0
:1066D000F00020280BD10722611C28460BF018FB84
:1066E000022873D128490870334988556EE0207814
:1066F00000F0F000A0B9207800F00F0828460BF059
:10670000A7FA4346621C414628460BF0C6FA601CB5
:1067100014F0C1F90220284988551B49087055E03A
:10672000207800F0F000102816D16078217801F070
:106730000F0100EB012828460BF08AFA4146062398
:10674000A21C28460BF0A9FA01201B4988550E49C6
:106750000870FFF72EFF39E0207800F0F0003028B5
:1067600034D1012015490870207800F00F00144939
:106770000870607813490870A07825E00068004030
:106780003516040854030020B8010020B20200208E
:10679000B4020020BA020020BB020020B502002093
:1067A000B6020020BC020020BA010020BB0100207C
:1067B00000020020380000205C240120FC010020A1
:1067C000FD010020FE0100200249087000BF00BF4B
:1067D000BDE8F883FF01002000228A71CA710A72A5
:1067E0004A728A720122CA7200228A707D2828D0D9
:1067F00006DC21280AD0322811D05F283CD117E0CE
:10680000FA2827D0B0F5FA7F36D12CE00022CA70E2
:1068100004220A7103224A715A220A8035E00022BA
:10682000CA7005220A7102224A713C220A802CE0B9
:106830000022CA7006220A7103224A711A220A80B3
:1068400023E00022CA7005220A7102224A7118222E
:106850000A801AE00022CA7005220A7102224A71D7
:106860000C220A8011E00022CA7005220A7102225D
:106870004A7106220A8008E00022CA7005220A71C5
:1068800002224A7106220A8000BF00BF70473EB54F
:1068900005460C4605B93EBD0020FE49087000F0D3
:1068A00095FC07F008FDFC4836F0F6FB0A2036F0B0
:1068B00027FD69462846FFF78FFF6946F64836F000
:1068C00004FC0CB1F548046001220221F24836F0C4
:1068D0002FFD01220821F04836F02AFD0122D103C4
:1068E000ED4836F025FD0122D102EB4836F020FDBF
:1068F00001221102E84836F01BFD00BFCBE73EB590
:1069000005460C4605B93EBD0120E249087000F07D
:106910005DFC07F019FEE04836F0BEFB0A2036F0B9
:10692000EFFC69462846FFF757FF6946DA4836F01C
:10693000CCFB0CB1DA48046001220221D64836F0C3
:10694000F7FC01220821D44836F0F2FC0122D103E1
:10695000D14836F0EDFC0122D102CF4836F0E8FCF8
:1069600001221102CC4836F0E3FC00BFCBE77FB533
:1069700005460C46207800F00800E0B3207800F0CF
:10698000040078B10421681E00EB8000C54A02EBC8
:1069900080000172681E00EB800002EB80006168DD
:1069A00041600DE00021681E00EB8000BD4A02EB53
:1069B00080000172681E00EB8000616842F82010C0
:1069C00000260CE004F10800815D681E00EB8000E9
:1069D000B44A02EB80000B308155701CC6B220789F
:1069E000B6EB101FEEDB681E00EB8000AD4901EB3B
:1069F0008000867257E0FFE705F10900C0B28DF80C
:106A00000A0001208DF80B00207800F00400F8B196
:106A100001208DF80C006068C0F34F30ADF8000025
:106A20004FF6FF71606801EAC000001DADF802007A
:106A30000421681E00EB80009B4A02EB800001727B
:106A4000681E00EB800002EB8000616841601BE083
:106A500000208DF80C004FF6FF70ADF800004FF6E7
:106A6000FF71606801EA4010ADF802000021681E65
:106A700000EB80008C4A02EB80000172681E00EB84
:106A80008000616842F820104FF6FF70ADF80400F6
:106A9000ADF806000020ADF8080001208DF80D00CB
:106AA000684636F09CFB7FBD70B504460D4629460E
:106AB0002046FFF75CFF70BD30B5431E03EB830338
:106AC000784C04EB83035B68002B4DD1431E03EB32
:106AD000830354F82330002B46D10B70431E03EB85
:106AE0008303714C04EB83031B7A042B0BD10B78CB
:106AF00043F004030B70431E03EB830304EB830397
:106B00005B684B600AE00B7823F007030B70431EB1
:106B100003EB8303644C54F823304B6000220CE0F9
:106B2000431E03EB8303604C04EB83030B339C5C39
:106B300001F108039C54531CDAB2431E03EB830398
:106B4000594C04EB83039B7A9342E9DC0B780F24C6
:106B50002340441E04EB8404534D05EB8404A47AC3
:106B600043EA04130B7046E008230B70431E03EB4B
:106B700083034C4C04EB83031B7A042B0BD10B785F
:106B800043F004030B70431E03EB830304EB830306
:106B90005B684B600AE00B7823F007030B70431E21
:106BA00003EB83033F4C54F823304B6000220CE08E
:106BB000431E03EB83033B4C04EB83030B339C5CCE
:106BC00001F108039C54531CDAB2431E03EB830308
:106BD000344C04EB83039B7A9342E9DC0B780F245B
:106BE0002340441E04EB84042E4D05EB8404A47A58
:106BF00043EA04130B7030BD30B504460D462946F8
:106C00002046FFF759FF30BD01460120704701467D
:106C1000012070471FB50446601E00EB800021492B
:106C200001EB80004068E8B9601E00EB800051F87D
:106C30002000B8B904F10900C0B28DF80A000020A4
:106C40008DF80D00684636F0CAFA0021601E00EB90
:106C50008000154A42F82010601E00EB800002EB15
:106C600080004160012004B010BD30B50246002014
:106C70000AE00C5C531E03EB83030A4D05EB830310
:106C80000B331C54431CD8B2531E03EB8303054C37
:106C90000CE00000900000200068004094000020FC
:106CA00098000020A02A00207429002004EB830310
:106CB0009B7A8342DDDC30BD2DE9F04104460D4670
:106CC0002146B54836F03DFB0746042F22D10DB3CF
:106CD000B248066812E00021AF4836F0C5FB022832
:106CE0000BD10121AC4836F0BFFB022805D10221AF
:106CF000A94836F0B9FB022800D004E0A748006894
:106D0000801BC828E7D300BF2146A34836F019FBF3
:106D1000074600BFBDE8F08170B504460D46611E10
:106D200001EB81019E4A02EB81002946FFF7C4FF77
:106D300070BD70B504462146974836F002FB064602
:106D4000042E21D19548056812E00021924836F0C2
:106D50008BFB02280BD101218F4836F085FB0228DE
:106D600005D102218C4836F07FFB022800D004E0D8
:106D70008A480068401BC828E7D300BF21468648E0
:106D800036F0DFFA064600BF70BD10B50446611E3E
:106D900001EB8101824A02EB8100FFF7CAFF10BDBF
:106DA0007D48006840F001007B49086000BF7A48D8
:106DB000001D006800F001000028F8D07648006847
:106DC00020F0010074490860704770B586B07548BE
:106DD000007840B101AA00216F4836F0C2FB01A83B
:106DE00014F008F856E0FF2501206F490870801E56
:106DF0000190029001AA0021674836F0B2FB0024FE
:106E00001FE004EB8400694901EB8000007A50B96F
:106E100004EB840051F82000019988420FD1E01C56
:106E2000C5B20F240BE004EB8400604901EB800045
:106E300040680299884202D1E01CC5B20F24601C50
:106E400084B20F2CDDDBFF2D23DA284600F076F824
:106E50000646EEB1711E01EB8101544A02EB81003E
:106E6000142201A939F0F2FC5148007840B19DF894
:106E70000E100DF10F0230464E4B1B68984707E08D
:106E80009DF80E100DF10F0230464B4B1B689847D2
:106E900000BF00BF06B070BD10B53F481830046891
:106EA00004F0700070B300203F49087004F07000D7
:106EB000302816D04148007898B941480078401CE5
:106EC0003F4908700021344836F019FB012132484F
:106ED00036F015FB0221304836F011FBFFF760FF5A
:106EE00004E038480078401C364908702A481830B9
:106EF000006820F07000284918310860C91426483D
:106F000036F0C8FC04F0010050B12E48007838B9C2
:106F10002A48007820B94FF480711F4836F0BAFC37
:106F200004F0020020B14FF400711B4836F0B2FCAF
:106F30004FF40041184836F0ADFC10BD0146C81EA4
:106F40000F2827D2DFE800F0080A0C0E10121416E2
:106F5000181A1C1E20222400012070470220FCE782
:106F60000320FAE70420F8E70520F6E70620F4E717
:106F70000720F2E70820F0E70920EEE70A20ECE717
:106F80000B20EAE70C20E8E70D20E6E70E20E4E717
:106F90000F20E2E70020E0E7006800403800002012
:106FA000A02A0020150200204C0000207429002097
:106FB0009000002098000020940000204D00002048
:106FC000B9010020BC0100203EB5044604B93EBD15
:106FD00000F0FCF807F06EF9794836F05DF8694684
:106FE0002046FFF7F9FB6946754836F06EF8012236
:106FF0000221734836F09CF90122D103704836F023
:1070000097F90122D1026E4836F092F9012211025D
:107010006B4836F08DF900BFD9E77FB505460C46C1
:10702000207800F00800E0B3207800F0040078B188
:107030000421681E00EB8000624A02EB80000172AE
:10704000681E00EB800002EB8000616841600DE08B
:107050000021681E00EB80005A4A02EB800001729A
:10706000681E00EB8000616842F8201000260CE0EA
:1070700004F10800815D681E00EB8000514A02EBBC
:1070800080000B308155701CC6B22078B6EB101F03
:10709000EEDB681E00EB80004A4901EB800086723F
:1070A00057E0FFE7681EC0B28DF80A0001208DF896
:1070B0000B00207800F0040000B301208DF80C00D4
:1070C0006068000C4FF6FF7101EAC000ADF80000E7
:1070D000606801EAC000001DADF802000421681ECE
:1070E00000EB8000384A02EB80000172681E00EB62
:1070F000800002EB8000616841601BE000208DF899
:107100000C004FF6FF70ADF800004FF6FF7160689D
:1071100001EA4010ADF802000021681E00EB80007B
:10712000294A02EB80000172681E00EB8000616852
:1071300042F820104FF6FF70ADF80400ADF80600DD
:107140000020ADF8080001208DF80D00684636F0EB
:1071500046F87FBD10B50446601E00EB8000194A5A
:1071600002EB8001164836F0ECF810BD00B585B092
:107170006A460021124836F0F4F99DF80B0007F03A
:10718000F5FD9DF80C0007F0F1FD9DF80D0007F0EE
:10719000EDFD9DF80E0007F0E9FD9DF80F0007F0EA
:1071A000E5FD9DF8100007F0E1FD9DF8110007F0E6
:1071B000DDFD9DF8120007F0D9FD05B000BD00000F
:1071C00000640040A02A00207429002010B500208F
:1071D0004EE0002200EB8003274C44F8232000EB14
:1071E000800304EB83035A6000EB800304EB83030A
:1071F0001A7200EB800304EB83035A7200EB8003E6
:1072000004EB83039A7200EB80031C4C44F82320A8
:1072100000EB800304EB83035A6000EB800304EB74
:1072200083031A7200EB800304EB83035A7200EBB2
:10723000800304EB83039A7200EB800304EB830367
:10724000DA74002110E0002300EB80020A4C04EB0A
:1072500082020B32535400EB8002084C04EB820292
:107260000B3253544A1C91B20829ECD3411C88B20A
:107270000F28AED310BD0000A02A002074290020E2
:107280000021FA4A1170FA4A1180002008E000211A
:10729000F84A22F81010F84A22F81010411C88B25F
:1072A0000528F4DB704730B50246F048007890427C
:1072B0001EDDEE48007888421ADDEE4830F81100F5
:1072C000EC4B33F81230984211DBEB4830F81200E7
:1072D000E84D35F8125040EA0543E74830F8110010
:1072E000E44D35F8115040EA0544E01A30BD00BFC6
:1072F0000020FBE710B50121102034F094FA0122A0
:107300001821DE4835F0B3FC7F21DC4835F07DFEE6
:107310000021DA4835F077FE01221146D74835F0D2
:107320001EFC0121202034F07EFA01224FF4C061BE
:10733000D34835F09CFC4FF6FF71D14835F065FE1F
:107340000021CF4835F05FFE01221146CC4835F0D0
:1073500006FC0121802034F066FA01221102C9489E
:1073600035F085FC45F63231C64835F04EFE45F61F
:107370003231C44835F047FE01221146C14835F08C
:10738000EEFB0121BF4835F0D0FB10BD10B5012147
:10739000BA4835F07EFEBC480088401CBA490880D7
:1073A000BA480088401CB949088010BD10B5B848DB
:1073B000007878B1B7480088401CB6490880B648C4
:1073C0000088098888427ADC0DF091F90020B149E3
:1073D000088074E0B148007801283FD1B0480078B7
:1073E00000283BD1AF480078AF490978884207DBD5
:1073F000AC480078AC490978401AAC49087007E0FD
:10740000A94800784042A74909780844A74908706C
:10741000A7480078002852D10120A649087010E042
:10742000FAF7FDF8A0480178A34814F0E9FD9E485A
:107430000078401C9C4908709C480078401E9B497D
:1074400008709A4800780028EADC974801789A4842
:1074500014F0D6FD00209749087030E0904800787D
:1074600068B39048007890490978884207DB8D48D6
:1074700000788D490978401A8C49087007E08A48DD
:10748000007840428749097808448849087012E02A
:10749000FAF7C5F884480078401CC1B2864833F03A
:1074A00088F881480078401C7F4908707F48007840
:1074B000401E7E4908707D4800780028E8DC0121E4
:1074C0006F4835F0E6FD10BD2DE9FF41002600278D
:1074D00000244FF010080025684634F002F900201F
:1074E000FBF761FDFFF7CCFE01221146734835F032
:1074F00036FB002072490880039F7248066818E036
:10750000FAF78DF86F480068801B40F6C411884276
:1075100001D2012000E0002058B90120684908800C
:1075200000220121654835F01AFB002004B0BDE8B7
:10753000F0814E4800780528E2DB002201215F48F7
:1075400035F00DFB01210020FFF7ADFE054647F2A7
:107550003050854207D901210020FFF7A4FE0546DF
:107560004FF0040812E043F69820854207D9022123
:107570000020FFF798FE05464FF0080806E00421BA
:107580000020FFF790FE05464FF0100808FB07F0BB
:1075900005EB450101EB0511B0FBF1F4B4F5C87F33
:1075A0000BD24FF4C05034F03AF8F9F7D3FA012275
:1075B0008021344835F05BFB08E04FF4A05034F0F4
:1075C0002EF8012211022F4835F051FBFFF758FE2B
:1075D00000213A4835F0A9FA002208212046FBF79D
:1075E000FDFC20B2A2E710B50121344835F040FD82
:1075F00040B10121314835F04CFD1D480088401C48
:107600001B49088002212D4835F032FDD8B10221F6
:107610002A4835F03EFD15480078042813DC14484C
:1076200000881449114A127821F81200234835F0D5
:10763000FEFC11490D4A127821F812000B4800781F
:10764000401C0A49087004211C4835F011FDD8B3CC
:1076500004211A4835F01DFD1048007810B9104873
:10766000007890B300200949088047E0A40000207A
:10767000A2000020D62B0020CC2B002000100040C0
:1076800000140040001C00409C0000209E000020D0
:107690004E000020A0000020220000202D0000202D
:1076A0002E0000209702002098020020990200205E
:1076B0009B0200209A020020393B0120004001403B
:1076C000120000203800002018E0FFE7CE480078C4
:1076D000042813DCCD480188CD48CB4A127820F825
:1076E0001210CC4835F0A6FCCB49C74A127821F8D5
:1076F0001200C5480078401CC349087010BD30B561
:1077000089B00121080434F09FF84F2006F047FAB1
:10771000012801D1002071E04F2006F040FA022834
:1077200001D101206AE04F2006F039FA042801D186
:10773000022063E04F2006F032FA082801D103202E
:107740005CE04F2006F02BFA102801D1042055E010
:107750004F2006F024FA202801D105204EE04F20CA
:1077600006F01DFA402801D1062047E04F2006F020
:1077700016FA802801D1072040E04F2006F00FFACA
:10778000B0F5807F01D1082038E04F2006F007FADD
:10779000B0F5007F01D1092030E04F2006F0FFF95D
:1077A000B0F5806F01D10A2028E04F2006F0F7F9EC
:1077B000B0F5006F01D10B2020E04F2006F0EFF96B
:1077C000B0F5805F01D10C2018E04F2006F0E7F9FA
:1077D000B0F5005F01D10D2010E04F2006F0DFF979
:1077E000B0F5804F01D10E2008E04F2006F0D7F908
:1077F000B0F5004F01D10F2000E0FF2004464F20DC
:1078000006F0C8F905460322214633F020FC50203B
:1078100006F0C5F9012801D1002071E0502006F0E2
:10782000BEF9022801D101206AE0502006F0B7F924
:10783000042801D1022063E0502006F0B0F90828A6
:1078400001D103205CE0502006F0A9F9102801D1F5
:10785000042055E0502006F0A2F9202801D105208F
:107860004EE0502006F09BF9402801D1062047E069
:10787000502006F094F9802801D1072040E05020E4
:1078800006F08DF9B0F5807F01D1082038E0502056
:1078900006F085F9B0F5007F01D1092030E05020D5
:1078A00006F07DF9B0F5806F01D10A2028E0502064
:1078B00006F075F9B0F5006F01D10B2020E05020E3
:1078C00006F06DF9B0F5805F01D10C2018E0502072
:1078D00006F065F9B0F5005F01D10D2010E05020F1
:1078E00006F05DF9B0F5804F01D10E2008E0502080
:1078F00006F055F9B0F5004F01D10F2000E0FF2050
:107900000446502006F046F905460322214633F08E
:107910009EFB02208DF820008DF8210000208DF8BC
:1079200022008DF823004F2006F039F907904F20F0
:1079300006F030F9044607A933F006FB502006F0A4
:107940002EF90790502006F025F9044607A933F0D8
:10795000FBFA304835F01CF900202E49088212202D
:10796000ADF804000020ADF806004FF6FF7002905D
:107970000020ADF80C0001A9264834F04CFE002090
:10798000ADF81000ADF812000120ADF81400002091
:10799000ADF81600ADF8180004A91E4835F01BF824
:1079A0000420ADF810000020ADF812000120ADF861
:1079B00014000020ADF81600ADF8180004A9154811
:1079C00035F009F80221134835F063FB0421114812
:1079D00035F05FFB012202210E4835F0C0F801228C
:1079E00004210C4835F0BBF801220021094835F08C
:1079F00080FA01220421074835F07BFA012105486D
:107A000035F093F809B030BDA4000020A20000209A
:107A1000D62B002000400140CC2B00202DE9F04364
:107A2000A1B00120FE4908600020FE490880102016
:107A3000FD4908600020FD490860FD490860F52007
:107A4000FC4908706A20FC4908706B2048706C2063
:107A500088706D20C87014200871002507E0002090
:107A6000F64941F82500F64941F825006D1C202D06
:107A7000F5D30120F1490860F1490860002500268E
:107A8000012443E0C6F107010120884000F0F5071A
:107A9000EFB1601EE94951F82000083041F8240098
:107AA000601EE74951F82000C01C41F82400641C06
:107AB000601EE24951F82000103041F82400601E99
:107AC000DF4951F82000153041F824001CE0601E09
:107AD000DA4951F82000103041F82400601ED849DE
:107AE00051F820000B3041F82400641C601ED3497B
:107AF00051F82000083041F82400601ED04951F8A8
:107B000020000D3041F82400761C641C082EB9D3E7
:107B10000121042033F087FE0121022033F094FE7E
:107B20000121480533F04CFE1C2006F038F80128EE
:107B300001D1002071E01C2006F031F8022801D1AB
:107B400001206AE01C2006F02AF8042801D1022056
:107B500063E01C2006F023F8082801D103205CE034
:107B60001C2006F01CF8102801D1042055E01C2030
:107B700006F015F8202801D105204EE01C2006F063
:107B80000EF8402801D1062047E01C2006F007F837
:107B9000802801D1072040E01C2006F000F8B0F555
:107BA000807F01D1082038E01C2005F0F8FFB0F5F7
:107BB000007F01D1092030E01C2005F0F0FFB0F576
:107BC000806F01D10A2028E01C2005F0E8FFB0F505
:107BD000006F01D10B2020E01C2005F0E0FFB0F584
:107BE000805F01D10C2018E01C2005F0D8FFB0F513
:107BF000005F01D10D2010E01C2005F0D0FFB0F592
:107C0000804F01D10E2008E01C2005F0C8FFB0F520
:107C1000004F01D10F2000E0FF2080461C2005F01E
:107C2000B9FF81460222414633F011FA1B2005F0CC
:107C3000B6FF012801D1002071E01B2005F0AFFF45
:107C4000022801D101206AE01B2005F0A8FF0428CA
:107C500001D1022063E01B2005F0A1FF082801D11B
:107C600003205CE01B2005F09AFF102801D10420BE
:107C700055E01B2005F093FF202801D105204EE0A0
:107C80001B2005F08CFF402801D1062047E01B2077
:107C900005F085FF802801D1072040E01B2005F07A
:107CA0007EFFB0F5807F01D1082038E01B2005F071
:107CB00076FFB0F5007F01D1092030E01B2005F0F0
:107CC0006EFFB0F5806F01D10A2028E01B2005F07F
:107CD00066FFB0F5006F01D10B2020E01B2005F0FE
:107CE0005EFFB0F5805F01D10C2018E01B2005F08D
:107CF00056FFB0F5005F01D10D2010E01B2005F00C
:107D00004EFFB0F5804F01D10E2008E01B2005F09A
:107D100046FFB0F5004F01D10F2000E0FF20804664
:107D20001B2005F037FF81460322414633F08FF9CF
:107D300002208DF880008DF8810000208DF88200EF
:107D40008DF883001C2005F02AFF1F901C2005F0F1
:107D500021FF80461FA933F0F7F800211C2009F00D
:107D6000C9FE1B2005F01BFF1F901B2005F012FF12
:107D700080461FA933F0E8F8324834F009FF324852
:107D800034F006FF00202F49103108804FF6FF71B4
:107D90002C4835F03EF93B20ADF800000020ADF84E
:107DA00002004FF6FF7001900020ADF80800694610
:107DB000244834F030FC7720ADF8000069462248B2
:107DC00034F029FC3020ADF868000120ADF86A00DD
:107DD0004FF6FF701C900020ADF874001AA91948E6
:107DE00034F07EFC00220E21164834F0C3FE01223E
:107DF0009102144834F0C3FE4FF0806003901148A4
:107E00003830049040200690002008904FF48060A5
:107E1000099080000A9080000B9000200C9015E0E3
:107E2000D8000020CC000020B4000020BC000020BE
:107E3000C0000020CF000020D0000020F03900203A
:107E4000703A002000080040000401404FF48030E8
:107E50000D9000200E900F901090119003A9FE48F5
:107E600034F0F8F901221021FB4834F044FA0020E4
:107E7000ADF85C000A20ADF85E000120ADF86000AE
:107E80000020ADF86200ADF8640017A9F34834F0A3
:107E9000A2FD0020ADF848004FF6FF70149012A923
:107EA000EE4834F01DFC01220221EC4834F057FE6C
:107EB00001220421E94834F052FE0121E74834F060
:107EC00034FE012021B0BDE8F083F0B502460B4638
:107ED000FF210026154625E04FF0000C80271BE00F
:107EE0002888384058B101F0800008B1012400E032
:107EF0001C24012000EB41006040C1B207E00024D7
:107F000001F0800000B11D2484EA4100C1B20CF1EF
:107F1000010000F0FF0C7F10BCF1080FE0DB701CCB
:107F2000C6B2AD1C9E42D7DBC843C0B2F0BD2DE93E
:107F3000FF4F8BB082460120C9490860804600206F
:107F4000C8490860C84908600AF0FF060C9880B26A
:107F5000ADF804000D9880B2ADF806000E9880B21E
:107F6000ADF80800189880B2ADF80A00199880B2F0
:107F7000ADF80C001A9880B2ADF80E001B9880B2D4
:107F8000ADF810001C9880B2ADF812001D9880B2B8
:107F9000ADF814001E9880B2ADF816001F9880B29C
:107FA000ADF81800002404E00020B04921F81400C6
:107FB000641CFF2CF8D9314601A8FFF786FF8146E3
:107FC00001A820F81690701CC6B2C820A849086005
:107FD000002464E0002700255EE001A830F81400CA
:107FE000C7F107020121914000EA010BBBF1000F2C
:107FF00024D0B8F1000F10D0012000EBC4002844B9
:10800000401E9B4951F820007E30012101EBC40144
:108010002944974A42F8210034E0012000EBC400D3
:108020002844401E924951F820004030012101EBC4
:10803000C40129448E4A42F8210023E0B8F1000F20
:1080400010D0012000EBC4002844401E884951F89C
:1080500020004030012101EBC4012944844A42F848
:1080600021000FE0012000EBC4002844401E80499D
:1080700051F820007E30012101EBC40129447C4AE3
:1080800042F821007F1C6D1CB8F1000F02D04FF0A8
:10809000000801E04FF00108082F9ED3641CB44291
:1080A00098D3012101EB0610401E714951F82000C0
:1080B0006430012202EB06116D4A42F821000521CD
:1080C0006C4834F0A6FF6A48634958394866022074
:1080D00000EBC600C86501215F4834F0F7F80120C5
:1080E000654908800020654908800121614834F015
:1080F0008AFF00BF624800680028FBD10120604968
:10810000086001215B4834F010FD01200FB0BDE88C
:10811000F08F30B50120012200235A4C23805A4CA5
:10812000238000BF431E594CE15C012807D1CBB22C
:10813000574C2478A34202D00123534C23800228B9
:1081400007D1CBB2524C6478A34202D001234E4CEB
:108150002380504B1B780BB1032810DD4D4B1B784F
:10816000012B05D1042803D1D21E0023494C2370D2
:10817000CBB2494C24881444474D25F81430401C98
:10818000521C0E2804DA454B1B789B1C9842C9DB15
:108190003D4B1B8843B901233E4C23703E4B1B884B
:1081A00013449B1E3C4C238030BD2DE9F04186B02A
:1081B00002212A4834F05CFF012875D11B2009F008
:1081C000C5FC0746254834F032FF84B20FB1E01FEA
:1081D00084B22B48006801287ED12949086004F543
:1081E0008C711E4834F015FF2448008801286DDD8D
:1081F0002B480088201A85B220480088401E1C4960
:1082000031F820101D480088801E194A32F82000DD
:10821000081A86B219480088801E224941F8206059
:1082200016480088401E41F8205006F10F00854294
:1082300002DC1E38A84249DD1020114908600021E7
:108240000C4834F072FC0021034834F03FF8402120
:10825000084834F03EFD29E0586002400004014027
:10826000D8000020BC000020B8000020F03700201B
:10827000E02B002000080040B0000020E8000020B3
:10828000B40000201C00002012000020E037002075
:10829000A8000020AB00002054030020DF000020D5
:1082A000CC000020F03A00200FE115E03020ADF8BE
:1082B00004000120ADF806004FF6FF700390002087
:1082C000ADF8100001A9FE4834F00AFAFD48008814
:1082D000401CFC490880E8E0FB480068042805D100
:1082E00004F58C71F94834F094FEDEE0F64800683D
:1082F000022803D0F448006800287DD1F4480088A3
:10830000201AF449F44A127821F81200F249087848
:10831000C11700EB5171C910F04A1170002F4DD1F7
:10832000EC48ED49097830F81100602818DCEC4879
:1083300011460978405C11460978E74A1278A2EBA9
:10834000C101C1F10702012191400843E449E34A18
:1083500012788854E0480078401CDF49087069E0D2
:10836000DC48DD49097830F81100A32819DCDC4825
:10837000DA490978405CD9490978D74A1278A2EBE2
:10838000C101C1F107026FF0010191400840D449D9
:10839000D24A12788854D0480078401CCE490870E0
:1083A00048E004F59671C94834F033FE0020CA490C
:1083B0000870CC490870C94908703BE0C548C649F7
:1083C000097830F8110060281BDAC548C3490978DC
:1083D000405CC2490978C04A1278A2EBC101C1F1E0
:1083E00007026FF0010191400840BD49BB4A127875
:1083F0008854B948007800E040E0401CB649087055
:1084000018E0B748B5490978405CB4490978B24AE0
:108410001278A2EBC101C1F107020121914008438A
:10842000C1B2AF48AD4A12788154AB480078401CC5
:10843000A9490870A4480068022804D104F1C801C1
:10844000A24834F0E6FD02209F490860A248007867
:1084500009282AD10846007800F0010028BB002036
:10846000A1490870A14908609D480078A049097891
:1084700088421AD101209D49086016E092480068A0
:10848000082809D1914834F0D2FD00F1C8084146CE
:108490008E4834F0BEFD08E08C4834F0C8FD00F58D
:1084A00096784146894834F0B4FD89480480042117
:1084B000864834F0EEFD01220421844834F04FFB5D
:1084C0000221824834F0E5FD00BF04217F4834F0EA
:1084D000CFFD012821D1002204217C4834F03FFB4C
:1084E00004217A4834F0D5FD77480068012815D179
:1084F000764834F09FFD00F164073946734834F044
:1085000088FD1020704908600421704834F0C1FDD6
:10851000012204216D4834F022FB9AE06A48006889
:10852000042828D1102068490860684834F07FFD8D
:1085300000F596773946654834F06BFD0122042139
:10854000624834F00CFB6648007830B16648007829
:1085500018B10120674908607BE06348007830B1BA
:1085600000206149087002206249086071E0012022
:10857000604908606DE054480068022831D15348D2
:1085800034F055FD00F58C773946504834F041FD04
:10859000012204214D4834F0E2FA08204A490860DB
:1085A00051480078012854D100204F490870052116
:1085B000434834F02EFD5048504948660720C865AE
:1085C00001214E48583033F081FE01204C4908808B
:1085D00001213B4834F017FD0121394834F0A5FA58
:1085E00037E039480068082811D110203649086062
:1085F000364834F01CFD00F596773946334834F0A0
:1086000008FD01220421314834F0A9FA21E00020BC
:108610002D49086031480078002817DD324800787D
:10862000A0B932480068012810D12C48007835499B
:1086300008700020284908702A49087027490870E6
:1086400001203149088000201F4908600020274987
:10865000086006B0BDE8F08110B52C4927485830B5
:1086600033F008FF0021164834F05FFA10BD10B552
:1086700027492248283033F0FDFE2648008838B9C3
:1086800000214FF0804034F050FA04200E49086079
:108690001B480088401E1A49088010BD10B51E49AD
:1086A0001648A03033F0E6FE1548008838B900219E
:1086B0004FF0804034F039FA0420034908602DE07F
:1086C00000080040E8000020B40000200004014041
:1086D000CC000020F0370020DC000020DE0000206D
:1086E000E0370020DD000020CE000020EC0000205C
:1086F000A8000020BC000020E02B00200060024009
:10870000B0000020DF0000201C00002000800018C6
:1087100000880010B200002000802020044800885B
:10872000401E0349088010BD02460120704700002A
:10873000B20000202DE9F043A1B00020F7490880E5
:10874000F7490860F7490860F7490860F749887BEE
:1087500006F0D6FB8046F549487B06F0D1FB08EBD6
:108760000010F3490870F149C87A06F0C9FB804649
:10877000EE49887A06F0C4FB08EB0010ED4908705A
:108780006B20487000208870C8700871002507E0D1
:108790000020E94941F82500E84941F825006D1C11
:1087A000202DF5D30120E4490860E4490860002544
:1087B0000026012443E0C6F107010120884000F0B3
:1087C000F507EFB1601EDC4951F82000083041F890
:1087D0002400601ED94951F82000083041F82400D7
:1087E000641C601ED44951F82000103041F8240068
:1087F000601ED24951F82000103041F824001CE0DE
:10880000601ECD4951F82000103041F82400601E50
:10881000CA4951F82000103041F82400641C601E41
:10882000C54951F82000083041F82400601EC349B2
:1088300051F82000083041F82400761C641C082EF2
:10884000B9D30121084632F0FFFF0121084632F07A
:10885000EAFF0121082032F0E6FF0121480532F04D
:10886000AFFF192005F09BF9012801D1002071E02C
:10887000192005F094F9022801D101206AE019209D
:1088800005F08DF9042801D1022063E0192005F0DC
:1088900086F9082801D103205CE0192005F07FF952
:1088A000102801D1042055E0192005F078F920287E
:1088B00001D105204EE0192005F071F9402801D1C1
:1088C000062047E0192005F06AF9802801D1072029
:1088D00040E0192005F063F9B0F5807F01D1082050
:1088E00038E0192005F05BF9B0F5007F01D10920CF
:1088F00030E0192005F053F9B0F5806F01D10A205E
:1089000028E0192005F04BF9B0F5006F01D10B20DC
:1089100020E0192005F043F9B0F5805F01D10C206B
:1089200018E0192005F03BF9B0F5005F01D10D20EA
:1089300010E0192005F033F9B0F5804F01D10E2079
:1089400008E0192005F02BF9B0F5004F01D10F20F8
:1089500000E0FF208046192005F01CF98146012225
:10896000414632F074FB1A2005F019F9012801D1B3
:10897000002071E01A2005F012F9022801D101202F
:108980006AE01A2005F00BF9042801D1022063E007
:108990001A2005F004F9082801D103205CE01A2010
:1089A00005F0FDF8102801D1042055E01A2005F04B
:1089B000F6F8202801D105204EE01A2005F0EFF846
:1089C000402801D1062047E01A2005F0E8F8802869
:1089D00001D1072040E01A2005F0E1F8B0F5807FD2
:1089E00001D1082038E01A2005F0D9F8B0F5007F51
:1089F00001D1092030E01A2005F0D1F8B0F5806FE0
:108A000001D10A2028E01A2005F0C9F8B0F5006F5E
:108A100001D10B2020E01A2005F0C1F8B0F5805FED
:108A200001D10C2018E01A2005F0B9F8B0F5005F6C
:108A300001D10D2010E01A2005F0B1F8B0F5804FFB
:108A400001D10E2008E01A2005F0A9F8B0F5004F7A
:108A500001D10F2000E0FF2080461A2005F09AF88F
:108A600081460122414632F0F2FA152005F097F8CE
:108A7000012801D1002084E0152005F090F802289B
:108A800001D101207DE0152005F089F8042801D1ED
:108A9000022076E0152005F082F8082801D1032095
:108AA0006FE0152005F07BF8102801D1042068E064
:108AB000152005F074F8202801D1052061E015206B
:108AC00005F06DF8402801D106205AE0152005F088
:108AD00066F8802801D1072053E0152005F05FF8E3
:108AE000B0F5807F01D108204BE0152005F057F844
:108AF000B0F5007F01D1092043E0152005F04FF8C3
:108B0000B0F5806F01D10A203BE0152005F047F851
:108B1000B0F5006F14D10B2033E00000CC00002032
:108B2000B4000020BC000020C0000020741400200D
:108B3000CF000020D0000020F0390020703A002043
:108B4000152005F02CF8B0F5805F01D10C2018E05D
:108B5000152005F024F8B0F5005F01D10D2010E0DC
:108B6000152005F01CF8B0F5804F01D10E2008E06B
:108B7000152005F014F8B0F5004F01D10F2000E0EA
:108B8000FF208046152005F005F881460122414668
:108B900032F05DFA162005F002F8012801D100201C
:108BA00071E0162004F0FBFF022801D101206AE0E9
:108BB000162004F0F4FF042801D1022063E01620FF
:108BC00004F0EDFF082801D103205CE0162004F03A
:108BD000E6FF102801D1042055E0162004F0DFFF45
:108BE000202801D105204EE0162004F0D8FF4028AF
:108BF00001D1062047E0162004F0D1FF802801D1E2
:108C0000072040E0162004F0CAFFB0F5807F01D1B4
:108C1000082038E0162004F0C2FFB0F5007F01D133
:108C2000092030E0162004F0BAFFB0F5806F01D1C2
:108C30000A2028E0162004F0B2FFB0F5006F01D141
:108C40000B2020E0162004F0AAFFB0F5805F01D1D0
:108C50000C2018E0162004F0A2FFB0F5005F01D14F
:108C60000D2010E0162004F09AFFB0F5804F01D1DE
:108C70000E2008E0162004F092FFB0F5004F01D15D
:108C80000F2000E0FF208046162004F083FF81467D
:108C90000122414632F0DBF9182004F080FF012860
:108CA00001D1002071E0182004F079FF022801D1E1
:108CB00001206AE0182004F072FF042801D102208C
:108CC00063E0182004F06BFF082801D103205CE06A
:108CD000182004F064FF102801D1042055E018206A
:108CE00004F05DFF202801D105204EE0182004F09B
:108CF00056FF402801D1062047E0182004F04FFF1E
:108D0000802801D1072040E0182004F048FFB0F58A
:108D1000807F01D1082038E0182004F040FFB0F532
:108D2000007F01D1092030E0182004F038FFB0F5B1
:108D3000806F01D10A2028E0182004F030FFB0F540
:108D4000006F01D10B2020E0182004F028FFB0F5BF
:108D5000805F01D10C2018E0182004F020FFB0F54E
:108D6000005F01D10D2010E0182004F018FFB0F5CD
:108D7000804F01D10E2008E0182004F010FFB0F55C
:108D8000004F01D10F2000E0FF208046182004F0A2
:108D900001FF81460122414632F059F9172004F0C3
:108DA000FEFE012801D1002071E0172004F0F7FE3B
:108DB000022801D101206AE0172004F0F0FE042807
:108DC00001D1022063E0172004F0E9FE082801D158
:108DD00003205CE0172004F0E2FE102801D10420FB
:108DE00055E0172004F0DBFE202801D105204EE0DD
:108DF000172004F0D4FE402801D1062047E01720B8
:108E000004F0CDFE802801D1072040E0172004F0B7
:108E1000C6FEB0F5807F01D1082038E0172004F0AD
:108E2000BEFEB0F5007F01D1092030E0172004F02C
:108E3000B6FEB0F5806F01D10A2028E0172004F0BB
:108E4000AEFEB0F5006F01D10B2020E0172004F03A
:108E5000A6FEB0F5805F01D10C2018E0172004F0C9
:108E60009EFEB0F5005F01D10D2010E0172004F048
:108E700096FEB0F5804F01D10E2008E0172004F0D7
:108E80008EFEB0F5004F01D10F2000E0FF2080469C
:108E9000172004F07FFE81460122414632F0D7F8C8
:108EA00002208DF880008DF8810000208DF882006E
:108EB00002208DF88300182004F071FE1F90182006
:108EC00004F068FE80461FA932F03EF8172004F037
:108ED00066FE1F90172004F05DFE80461FA932F049
:108EE00033F8192004F05BFE1F90192004F052FEA5
:108EF00080461FA932F028F81A2004F050FE1F9077
:108F00001A2004F047FE80461FA932F01DF81520F4
:108F100004F045FE1F90152004F03CFE80461FA97A
:108F200032F012F8162004F03AFE1F90162004F0DA
:108F300031FE80461FA932F007F8FE4833F028FEC4
:108F40004FF0804033F024FEFB4833F021FE002038
:108F50004FF0804108824FF6FF714FF0804034F0AF
:108F600056F84FF6FF714FF0804034F052F84FF64C
:108F7000FF71F14834F04BF83B20ADF800000020C1
:108F8000ADF802004FF6FF7001900020ADF8080028
:108F900069464FF0804033F03EFB3B20ADF80000C7
:108FA0006946E54833F037FB7720ADF80000002034
:108FB000ADF802004FF6FF7001900020ADF80800F8
:108FC0006946DC4833F027FB3020ADF8680001200B
:108FD000ADF86A004FF6FF701C900220ADF87400E7
:108FE0001AA9400733F0C1FB0020ADF874001AA99C
:108FF0004FF0804033F0FCFB0020ADF84800401EED
:10900000149012A9CC4833F038FB00221146CA480C
:1090100033F06FFF00220F214FF0804033F0AAFDA4
:1090200000221021880633F0A5FD0122D102C804D8
:1090300033F0A5FD01221103880433F0A0FD4FF0A9
:10904000C0600390BD480490402006900020089026
:109050004FF48060099080000A9080000B900020FF
:109060000C904FF480300D9000200E900F901090D7
:10907000119003A9B24833F0EDF84FF0C0600390AF
:10908000AE48001D049003A9AD48783033F0E2F8F3
:1090900001221021AA4833F02EF901221021A848FC
:1090A000783033F028F90020ADF85C00ADF85E00B0
:1090B0000120ADF860000020ADF86200ADF864005A
:1090C00017A99C4833F087FC0C20ADF85C00002009
:1090D000ADF85E0017A9974833F07DFC0420ADF889
:1090E0005C000220ADF85E0017A9924833F073FCD3
:1090F0000820ADF85C000220ADF85E0017A98D488D
:1091000033F069FC00218B4833F07DFF00218A4851
:1091100033F079FF0121874833F007FD01218648AC
:1091200033F003FD01220021824833F0E2FE0122E8
:109130000421804833F0DDFE012202217D4833F016
:109140000EFD21B0BDE8F0832DE9F14F8AB04FF05C
:10915000040820200190002600BF7A4A08F101018E
:10916000505C05F0CDFE8346764911F8080005F005
:10917000C7FE0BEB001002A921F81600F8F74FFA12
:10918000701CC6B26F4908F10200085C019008F13A
:10919000030801980028E0D1C87A05F0B1FE8346A3
:1091A0006849887A05F0ACFE0BEB00106649087040
:1091B00001206649086066490860002400270125EF
:1091C00045E0C7F107010120884000F0F509B9F139
:1091D000000F1DD0681E5D4951F82000801D41F828
:1091E0002500681E5A4951F82000001D41F825004D
:1091F0006D1C681E554951F82000123041F82500B9
:10920000681E534951F82000143041F825001CE035
:10921000681E4E4951F820000E3041F82500681EA6
:109220004B4951F820000C3041F825006D1C681E98
:10923000464951F820000A3041F82500681E44498B
:1092400051F820000C3041F825007F1C6D1C082FC0
:10925000B7D3F8F7E4F90A9860B93A49C87A05F043
:109260004FFE83463749887A05F04AFE0BEB001023
:1092700038490870002038490860002404E00020C4
:10928000364921F81400641CFF2CF8D9314602A895
:10929000FEF71BFE824602A921F816A0701CC6B27A
:1092A0001E202F49086008460068123048601C20C4
:1092B0002C49086008460068143048600024B2E079
:1092C00000270025ABE002A830F81400C7F1070220
:1092D0000121914000EA0109B9F1000F5CD00220A0
:1092E00000EB04102844401E1D4951F82000801D49
:1092F000022101EB04112944194A42F821000220FD
:1093000000EB04102844401E164951F82000001DAF
:10931000022101EB04112944124A42F821006D1C7C
:10932000022000EB04102844401E0D4951F8200093
:10933000123019E000000140000C00403C000040E9
:109340002860024074140020CF000020F039002073
:10935000703A0020D0000020B8000020F037002034
:10936000E02B0020E02F0020022101EB0411294412
:10937000F84A42F82100022000EB04102844401E65
:10938000F54951F820001430022101EB0411294461
:10939000F14A42F8210040E0022000EB041028448A
:1093A000401EEC4951F820000E30022101EB04115F
:1093B0002944E84A42F82100022000EB0410284426
:1093C000401EE54951F820000C30022101EB041148
:1093D0002944E14A42F821006D1C022000EB0410F0
:1093E0002844401EDB4951F820000A30022101EBDD
:1093F00004112944D74A42F82100022000EB04104E
:109400002844401ED44951F820000C30022101EBC1
:1094100004112944D04A42F821007F1C6D1C082FFA
:10942000FFF451AF641CB442FFF44AAF012101EBD9
:109430000610401EC74951F820006430012202EB9B
:109440000611C44A42F82100012101EB0610401E1A
:10945000C14951F820006430012202EB0611BE4AD6
:1094600042F821000121880733F0D5FD012188074A
:1094700033F0D3FDB748B9494863B748B749AC3171
:109480000860022101EB0610B449C862022101EB19
:109490000610B249C1F8A4000121B048283032F0CA
:1094A00015FF0121AD48A03032F010FF0120AC497A
:1094B0000880AC4908800020AB49088000214FF0AB
:1094C000804033F0A0FD00BFA84800680028FBD111
:1094D0000120A64908600121800733F026FBF8F738
:1094E0009EF80020A249086008460068192803D3A6
:1094F0000120A049088001E0F8F791F80BB0BDE821
:10950000F08F2DE9F047064600209B4908600024B3
:1095100004E00020994921F81400641CFF2CF8D9BC
:10952000F1B29748FEF7D1FC8046954820F81680A6
:10953000761C1E2087490860084600681230486083
:109540001C208549086008460068143048600024E3
:1095500097E00027002590E0894830F81400C7F113
:1095600007020121914000EA0109B9F1000F41D041
:10957000022000EB04102844401E764951F82000D8
:10958000801D022101EB04112944724A42F8210096
:10959000022000EB04102844401E6F4951F82000BF
:1095A000001D022101EB041129446B4A42F82100FD
:1095B0006D1C022000EB04102844401E654951F840
:1095C00020001230022101EB04112944614A42F8C3
:1095D0002100022000EB04102844401E5E4951F88F
:1095E00020001430022101EB041129445A4A42F8A8
:1095F000210040E0022000EB04102844401E5549A1
:1096000051F820000E30022101EB04112944514A87
:1096100042F82100022000EB04102844401E4E496D
:1096200051F820000C30022101EB041129444A4A70
:1096300042F821006D1C022000EB04102844401E5B
:10964000444951F820000A30022101EB0411294459
:10965000404A42F82100022000EB04102844401E3A
:109660003D4951F820000C30022101EB041129443E
:10967000394A42F821007F1C6D1C082FFFF46CAFA3
:10968000641CB442FFF465AF012101EB0610401EDB
:10969000304951F820006430012202EB06112D4AB6
:1096A00042F82100012101EB0610401E2A4951F821
:1096B00020006430012202EB0611274A42F8210003
:1096C0000121880733F0A7FC0121880733F0A5FCAE
:1096D00020482249486320482049AC3108600221D3
:1096E00001EB06101D49C862022101EB06101B495F
:1096F000C1F8A40001211948283032F0E7FD01210A
:109700001648A03032F0E2FD0120154908801549C5
:10971000088000201449088000214FF0804033F079
:1097200072FC00BF114800680028FBD101200F49DE
:1097300008600121800733F0F8F9F7F770FF002087
:109740000B4908600846006819281BD30120094905
:10975000088019E0E02B0020E02F0020006002408C
:10976000B0000020B2000020E8000020B40000207B
:109770003800002012000020B8000020F037002040
:10978000F8120020F7F74BFFBDE8F0872DE9F0470E
:1097900005460E460027B846B94601240020FE497A
:1097A0000880FE49088000BF0020FD49086000BF16
:1097B000F7F735FFFB48008818B9F948006885427B
:1097C000F6D2F7480068854202D80120F2490880A5
:1097D000F148008898BBB8F1010F0BDB012E02D0D5
:1097E0004FF0030906E040F2E730EC4921F814009D
:1097F000601C04B2EC4890F800A0012E03D10AF1DD
:1098000001000FFA80FA0020E649088000270CE0EA
:1098100007EB0900E549085CE04921F81400F7F777
:10982000FEFE601C04B2781C07B2AAEB0900B84225
:10983000EEDCF7F7F4FE08F101000FFA80F8D648E5
:1098400000880028B0D0D4480088012805D1B8F19C
:10985000010F02DB0020D0490880601ECF4908803C
:10986000BDE8F08770B586B000221146D04833F0CD
:1098700040FB0021CE4833F0C6FBCD4824300068C1
:10988000CC490860CC4833F0D2FBCC490860CA48C8
:1098900033F0D0FBCA490860CA48006801285ED18D
:1098A000C8490860C34801683031C14833F0AFFB94
:1098B000C548008802284CDDC1480068C3490988B2
:1098C000451AC1480088801EC14951F82010BE4881
:1098D0000088C01EBE4A52F820000E1A301D854274
:1098E00002D8301FA84234D91020B64908600021A0
:1098F000800633F01AF90021B64832F0E7FC002167
:10990000B448783032F0E2FC0020B3490880B34913
:1099100008804021080633F0E8F94021080633F0BA
:10992000ECF93020ADF804000120ADF806004FF648
:10993000FF7003900220ADF8100001A9400732F03B
:1099400014FF0020ADF8100001A94FF0804032F064
:109950004FFF9D480088801C9B49088011E1994871
:109960000068042806D1934801684831904833F0D4
:109970004EFB06E193480068022803D09148006836
:1099800000287DD18E4800889549964A127821F8A2
:1099900012008B4800888D490988401A9249914AE3
:1099A000127821F812008F490878C11700EB517125
:1099B000C9108E4A11708C488A49097830F8110014
:1099C0000D2818DA794811460978405C1146097863
:1099D000844A1278A2EBC101C1F107020121914032
:1099E00008437249814A127888547E480078401CA6
:1099F0007C4908702DE07C487A49097830F81100DC
:109A0000182819DA694879490978405C7749097852
:109A1000744A1278A2EBC101C1F107026FF0010193
:109A2000914008406149714A127888546D48007825
:109A3000401C6C4908700CE05E48016860315C486D
:109A400033F0E5FA002067490870694908706749F2
:109A500008705C480068022806D15648006800F18A
:109A60002801534833F0D3FA0220564908605D4874
:109A70000078092832D10846007800F0010000E0A3
:109A80006DE038BB4948007800F0080018BB474833
:109A9000007800F00700052818D2DFE800F003077F
:109AA0000B0F130002205349087013E001205149A5
:109AB00008700FE002204F4908700BE003204D4969
:109AC000087007E001204B49087003E00020494975
:109AD000087000BF02E00020464908704148007845
:109AE00012284ED13748007800F00100002848D1F4
:109AF0002E48407800F0040098B12C4840783E4948
:109B00000978884209D000203A49087010202D4970
:109B1000086000203949086033E0012037490860B7
:109B20002FE0002035490860002409E01F484078F4
:109B30003349095D884202D1012030490860641C24
:109B40002F48005D08B1052CF0D32C480068C0B93F
:109B500000202849087010201A49086011E01948AF
:109B60000068082806D1134801683031104833F0E6
:109B70004EFA06E00F48006800F15B010C4833F034
:109B800046FA0E480088114908800221084833F03F
:109B900080FA0122022135E0120000205403002047
:109BA0003800002020000020DF000020E0370020E7
:109BB000000C0040F400002000000140E000002004
:109BC000E4000020B4000020E8000020CC000020C9
:109BD000E02B002028600240B0000020B2000020EE
:109BE000E0350020DC000020F0370020DE000020FF
:109BF000DD000020CE000020CF000020F00000207B
:109C0000D0000020714832F0AAFF012200216F48E5
:109C100033F06FF902216E4833F03BFA08216C48AB
:109C200033F037FA06B070BD10B50221674833F043
:109C30001FFA012826D100220221644832F08FFF4A
:109C400000221146614833F054F902215F4833F095
:109C500020FA60480068012815D15C4833F0E7F924
:109C600000F130042146594833F0D1F91020594908
:109C700008600221554833F00CFA012202215348B2
:109C800032F06DFF99E053480068042812D110208B
:109C9000504908605048016860314C4833F0B7F9CA
:109CA00002214A4833F0F5F901220221474832F0F7
:109CB00056FF82E04748006802284BD1434833F002
:109CC000B6F900F148042146404833F0A0F90221DA
:109CD0003E4833F0DEF9012202213C4832F03FFFDA
:109CE00008203C4908603D480078012865D13C487F
:109CF0000068012861D100203849087001218807D7
:109D000033F089F90121880733F087F9354836495E
:109D1000486336483449AC31086010203249C86283
:109D2000C1F8A40001213048283032F0CFFA0121D7
:109D30002D48A03032F0CAFA01202D4908802D4963
:109D400008800021800733F05EF90121880732F096
:109D5000ECFE32E01F480068082812D110201D498F
:109D600008601D4801686031184833F050F902213D
:109D7000164833F08EF901220221144832F0EFFE2A
:109D80001BE00020134908601B480078002814DD00
:109D900013480068012810D1184908801648007837
:109DA00017490870002017490870174908701249B0
:109DB0000870084908600A4908600821034833F020
:109DC00057F9012801D1F9F7DEFD10BD000C004064
:109DD00000000140B4000020F4000020CE0000206C
:109DE000F0000020F439002000600240743A0020A6
:109DF000B0000020B2000020DE0000202000002083
:109E0000DF000020DC000020DD00002010B5012173
:109E1000402031F0E6FC012035F0E8FF10BD2DE9CF
:109E2000F04105460E46174600BF00BF012035F041
:109E3000FFFF0028FAD035F0F7FF00EA0704AC4234
:109E4000F3D3B442F1D82046BDE8F08110B5FD4906
:109E50000B880988491CFB4C2180FB49C85410BD64
:109E6000FA490880704710B501F02CFA0446012C1D
:109E700002D0022C12D103E00120F54908700EE057
:109E8000F448407930B14FF4FA714FF49670FBF713
:109E9000C3FE02E00120F049087000E000BF00BFEF
:109EA00010BD10B5ED48008870B12A20F6F7FEFD10
:109EB0003620F6F7FBFD3020F6F7F8FD3720F6F7F1
:109EC000F5FD0D20F6F7F2FD00210820FBF798FDC7
:109ED00010BD10B5FFF7E5FFE1480078FF2806D078
:109EE000DF48007801F07FFDFF20DD490870DD4884
:109EF0000078FF2806D0DB48007801F074FDFF20D1
:109F0000D8490870D8480078FF2806D0D64800788D
:109F100001F069FDFF20D449087000210820FBF7FB
:109F20006FFD00210420FBF76BFD0021012001F0F3
:109F30006FFA0020C8490870C5490870CB490870FD
:109F400010BD2DE9F04104464EF66020B4FBF0F65A
:109F5000B4FBF0F100FB11454FF47A70B5FBF0F75C
:109F6000B5FBF0F100FB1158B0B204F034FE5F20F5
:109F7000F7F79EFAB8B204F02EFE5F20F7F798FAD2
:109F80001FFA88F004F027FEBDE8F08110B5FF202D
:109F9000B3490870FFF767FFAF48007810B1FFF7CB
:109FA00098FF0EE0B148007858B100210820FBF777
:109FB00027FDC8214FF4FA70FBF753FD002000F095
:109FC00001F810BDF8B50446002734B9C821A848E7
:109FD00036F090FC0020A749088001F077FB009044
:109FE000C4EBC4004FF4A05202EB4021009801F0F2
:109FF0003AFC002843D040F648429F49009801F0BF
:10A00000B2FB002838D02A20F6F750FD3620F6F7AC
:10A010004DFD002606E03146721C96B2974A505C10
:10A02000F6F744FD9548805D0028F4D10320F6F74B
:10A0300062FD0D20F6F73AFD91480470007840B2B9
:10A04000FFF704FF3D20F7F733FA012701F071FC19
:10A05000054644B98B4944F62060284401F098FC39
:10A060007F4908700DE0874941F28830284401F0AB
:10A070008FFC7B49087004E0FFF72BFF01E0FFF73E
:10A0800028FF684601F057FB3846F8BD0146CAB2C2
:10A09000C2F500700844704738B501F017FB009016
:10A0A00000240021009801F0DEFB30B10C22694948
:10A0B000009801F058FB00B10124684601F03BFB19
:10A0C000204638BD2DE9FF4107460C4616460025BF
:10A0D00000208DF80000208080463CE0012203A98A
:10A0E000384601F040FB78B39DF80C0030280BDBBC
:10A0F0009DF80C00392807DC9DF80C202846691CC7
:10A10000CDB20DF8002022E0C5B12088B0F5007F67
:10A1100010DA00222846691CCDB20DF800206846EE
:10A1200036F0C6FA218826F811002088401C2080CD
:10A13000002503E0002004B0BDE8F0819DF80C008C
:10A140000D2802D10120F6E700E000E004E008F16C
:10A1500001001FFA80F8C1E700BF0020EBE72DE9FE
:10A16000F04180460D461646002700241CE035F8D5
:10A170001400FF2807DA781C87B29EB115F8140086
:10A18000F7F796F90EE0F81C87B25EB1FF20F7F7FB
:10A190008FF935F81410080AF7F78AF915F8140042
:10A1A000F7F786F9601C84B24445E0DB3846BDE829
:10A1B000F0817CB5054600260024012201A928462D
:10A1C00001F0D1FA48B3304A69462846FFF77AFFD2
:10A1D00018B300222C49BDF80000FFF7C0FF044669
:10A1E000601C84B2200AF7F763F9E0B2F7F760F970
:10A1F00004EB1421C1F1FF01C8B2F7F759F99DF83A
:10A200000400F7F755F901221F49BDF80000FFF7D8
:10A21000A6FF401CA04200D1012630467CBD10B5EF
:10A220001A4801880088401E184A108049B1F7F783
:10A23000F6F901F07EFB0446154904F57A7001F049
:10A24000A7FB10BDF8000020444B002010010020A7
:10A2500006010020384B00200501002002000020EC
:10A2600008010020090100200A010020040100204B
:10A27000445300200C010020F03E0020F446002052
:10A28000FA0000208D9F0008444F00200E0100209E
:10A290001FA200087CB5054601F018FA0090C5EB36
:10A2A000C5004FF4A05202EB4021009801F0DBFA08
:10A2B00050B1012201A9009801F055FA10B19DF8A2
:10A2C000044002E0312400E03124684601F033FA12
:10A2D00020467CBD2DE9FC4105460C46681E042144
:10A2E00001EBC00086B20027200E8DF80400200C80
:10A2F0008DF80500200A8DF80600E0B28DF8070001
:10A3000001F0E4F9009006F55C21009801F0ABFA49
:10A3100048B1042201A9009801F068FA18B1009828
:10A3200001F055FA0746684601F005FA3846BDE8DF
:10A33000FC8138B501F0CAF9009000240021009892
:10A3400001F091FA48B10C22FE49009801F04EFA52
:10A3500018B1009801F03BFA0446684601F0EBF9A9
:10A36000204638BD10B5FF20F7490870F5488178C0
:10A37000F6480078401C81420CD101210820FBF7EF
:10A380003FFB0121084601F043F8EE484078EF49D1
:10A3900008701EE0EB484178EC480078401C814290
:10A3A00017DD00BFE9490978491CC8B2FFF772FF01
:10A3B0000446322C04D1E5480078401CE34908707B
:10A3C000322C06D1DF484178E0480078401C8142B9
:10A3D000E8DCDC484178DD480078401C814248DCFC
:10A3E000DB48007830B10020D9490870001FFFF722
:10A3F0002DFD03E06FF00400FFF728FD3D20F7F787
:10A4000057F82A20F7F754F8D2480068FFF799FD6B
:10A410000D20FFF71BFDD04BD0480288D0491846CD
:10A420000068F9F729FD08B30020CC490880CD4821
:10A430000068401CCB490860C2490879C9490968CD
:10A44000FFF748FFC4480068BE498860FFF771FF06
:10A45000C548007838B1C548007820B9B94988782E
:10A46000FFF7B0FD0EE0FFF734FD0BE0FFF731FD25
:10A4700008E0BD48007828B1B4490978491CC8B241
:10A48000FFF7A0FD10BD10B5FF20B9490870FFF718
:10A49000EAFCB648007810B1FFF71BFD09E0B248AE
:10A4A000007830B100210820FBF7AAFA0020FFF75E
:10A4B00089FD10BD03E0AF49884200D303E010F8E6
:10A4C000012B202AF7D100BF70472DE9FE43074634
:10A4D0000C469046002600208DF800002080814622
:10A4E0002CE017F80950302D07DB392D05DC3046FC
:10A4F000711CCEB20DF800501CE0BEB12088B0F542
:10A50000007F10DA00223046711CCEB20DF8002018
:10A51000684636F0CDF8218828F811002088401CC4
:10A520002080002602E00120BDE8FE830D2D01D130
:10A530000120F9E709F101001FFA80F9D1E72DE9BF
:10A54000FC4100278C4C2046FFF7B4FF0446204610
:10A55000FFF7B0FF04462046FFF7ACFF0446204655
:10A56000FFF7A8FF04462046FFF7A4FF0446204655
:10A5700036F09EF8C5B2012D02DA0120BDE8FC815B
:10A580002046FFF797FF044621467C4801F0B2FAC7
:10A59000E8B17B4A69467248401CFFF796FF0028E5
:10A5A0006BD0BDF80000A84267DB09E0681E744963
:10A5B00031F81000BDF80410884201D1012705E0F0
:10A5C00001A96E4801F0C3FA0028EFD155E06A49AD
:10A5D000091F91F8050C04F093FC80466649091F99
:10A5E00091F8040C04F08CFC08EB0010C5B2002DAF
:10A5F00042D0634A69465A48401CFFF766FFB8B329
:10A60000BDF80000A84238DB5E4C04F1400630E0A3
:10A6100014F8010B04F074FC4FF6FF7101EA0030EE
:10A62000019014F8010B04F06BFCBDF8041001EB71
:10A63000002080B2019014F8010B04F061FCBDF819
:10A64000041001EB001080B2019014F8010B04F02B
:10A6500057FCBDF80410084480B20190681E4849B8
:10A6600031F81000BDF80410884202D1012702E041
:10A6700003E0B442CCD300E0012727BB3348007885
:10A68000C82819D2404831490978405C401CC1B201
:10A690003D482E4A127881542C490978405C0A289A
:10A6A0000ADB4FF4FA714FF49670FBF7DAF90021E8
:10A6B0003548264A1278815434480088401C334972
:10A6C000088000205AE721480078C82804D20020DA
:10A6D0002D491E4A1278885400202C4908800120F8
:10A6E0004CE770B5FFF7BFFB29480078FF287DD005
:10A6F0002748007801F077F9FF2025490870164BAC
:10A7000016480288164918460068F9F7B5FB002874
:10A710006DD0FFF714FF054600201049088011484E
:10A720000068401C0F490860A5BB064880780749AF
:10A73000097888423CDDFFF7B4FB01F0FAF80446E3
:10A74000C82128E0384B002009010020FA00002031
:10A75000060100204000002000010020F800002039
:10A76000444B0020FC0000200401002005010020D3
:10A770000A010020F4460020F43E00200C54002082
:10A78000444F0020F84A0020445300200C010020D0
:10A79000080100202CE04FF4FA70FBF762F9FE4943
:10A7A00041F28830204401F0F3F8FC49087070BD94
:10A7B000FB48C07800EB4000FA490988884217DA64
:10A7C0000020F8490880FFF76CFB01F0B2F804465E
:10A7D000C8214FF4FA70FBF744F9EF4941F2883091
:10A7E000204401F0D5F8ED490870E0E71AE016E0E2
:10A7F00001F09FF80446EC48007838B9EB4904F6BC
:10A80000B83001F0C5F8EA49087013E0E949098851
:10A810006018E64901F0BCF8E54908700AE0FFF766
:10A8200058FB07E00021E448E44A128881540020E4
:10A83000E249088000BFBAE72DE9FC410546002641
:10A840000024002700F042FF0090C5EBC5004FF444
:10A85000A05202EB4021009801F005F800282DD00D
:10A860000220F6F725FE00BF13E0012201A900989F
:10A8700000F079FF48B101279DF80400F6F718FEB3
:10A880009DF804002044C4B201E0002705E0701CDC
:10A8900086B240F648408642E7D300BF47B184F015
:10A8A000FF04204604F062FA0320F6F701FE05E0FB
:10A8B0003020F6F7FDFD0320F6F7FAFD684600F0BC
:10A8C0003AFFBDE8FC812DE9F84304460026254601
:10A8D000002741F20101085D04F012FB81464FF4AC
:10A8E0008051085D04F00CFB09EB001000F0FF083C
:10A8F00000BF05E015F8011B8819C6B2781C87B2A5
:10A90000B7F5805FF6DB86F0FF0646451FD100F005
:10A91000DDFE00904FF40071009800F0A4FF48B1F4
:10A920004FF480522146009800F060FF10B100986B
:10A9300000F04DFF684600F0FEFE0220F6F7B8FD7D
:10A940003120F6F7B5FD0320F6F7B2FD08E002204E
:10A95000F6F7AEFD3020F6F7ABFD0320F6F7A8FDC5
:10A96000BDE8F88310B5F9F7ABF90446012C09D11D
:10A970000220F6F79DFD3120F6F79AFD0320F6F749
:10A9800097FD08E00220F6F793FD3020F6F790FDE2
:10A990000320F6F78DFD10BD38B50024FFF77CFBD2
:10A9A00000285AD07E48407818B17D484078FF286A
:10A9B0004ED100207A498870C8704870487100F004
:10A9C00085FE009000BFC4EBC4004FF4A05202EB20
:10A9D0004021009800F047FF40F64842784900982F
:10A9E00000F0C1FE28B37648007830280ED16C48BC
:10A9F0008078401C6A49887008464078401C48703E
:10AA00006F48407800F00100487110E06C48007811
:10AA1000312803D06A480078322808D16048C078CD
:10AA2000401C5F49C87008464078401C4870601C54
:10AA3000C4B2634800783028C5D061480078312816
:10AA4000C1D05F4800783228BDD0684600F073FE60
:10AA5000FFF76FFC08B1012038BD0020FCE710B5FE
:10AA6000F9F75BF958B1F9F718F930B1FFF714FBB2
:10AA700008B1012010BD0520FCE70320FAE7022001
:10AA8000F8E710B5FFF7EBFF012805D1FFF784FFCA
:10AA900010B14348407810BD0020FCE72DE9FC418F
:10AAA00005460C46681E4FF6FF7101EAC0060027F6
:10AAB000200E8DF80400200C8DF80500200A8DF87A
:10AAC0000600E0B28DF8070000F000FE009006F5E9
:10AAD0005C21009800F0C7FE48B1042201A900984B
:10AAE00000F084FE18B1009800F071FE0746684639
:10AAF00000F021FE3846BDE8FC8110B5FFF7AFFF3E
:10AB000001280AD126480079FF2803D100202449D2
:10AB1000087110BD22480079FBE70020F9E77CB5F9
:10AB200004460025E60000F0D1FD009006F55C210A
:10AB3000009800F098FEB0B1042201A9009800F03E
:10AB400012FE68B19DF8040000069DF8051000EBA8
:10AB500001409DF8061000EB01209DF807104518F4
:10AB6000684600F0E8FD28467CBD7CB5044604201C
:10AB700000EBC405002600F0A9FD009005F55C215E
:10AB8000009800F070FE58B3042201A9009800F06C
:10AB9000EAFD28B316E0000087A400080A0100209F
:10ABA000384B00200C010020FA00002065A30008AB
:10ABB0000901002010010020444B0020F800002073
:10ABC000F03E00209DF8040000069DF8051000EB03
:10ABD00001409DF8061000EB01209DF80710461873
:10ABE000684600F0A8FD30467CBD2DE9FC5F0446B8
:10ABF0000026B046271DE01C0090207804F080F964
:10AC0000642100FB01FB607804F07AF900EB80001E
:10AC10000BEB400BA07804F073F9584400F0FF09E7
:10AC200094F84D0C04F06CF9834694F84C0C04F045
:10AC300067F90BEB001000F0FF0A0098407801283C
:10AC400002D10020401C00BF00F040FD0190C9EB84
:10AC5000C9004FF4A05202EB4021019800F003FE1E
:10AC6000F8B1002511E001223946019800F0BEFD3F
:10AC700010B14FF0010802E04FF0000809E0387809
:10AC80003044C6B2681C85B27F1C40F648408542FD
:10AC9000E9D300BFB8F1000F03D0019800F097FD91
:10ACA000804601A800F047FD86F0FF06B8F1000FCE
:10ACB0000BD0564509D10220F6F7FAFB3120F6F702
:10ACC000F7FB0320F6F7F4FB08E00220F6F7F0FBB1
:10ACD0003020F6F7EDFB0320F6F7EAFBBDE8FC9F1A
:10ACE0007CB50024002600F0F1FC01904FF40071C7
:10ACF000019800F0B8FD28B30220F6F7D9FB002533
:10AD000013E001226946019800F02DFD48B10126AB
:10AD10009DF80000F6F7CCFB9DF800002044C4B27B
:10AD200001E0002604E0681C85B2B5F5805FE8DB31
:10AD300000BF46B184F0FF04204604F017F803205A
:10AD4000F6F7B6FB05E03020F6F7B2FB0320F6F786
:10AD5000AFFB01A800F0EFFC7CBD10B5FFF79CF93C
:10AD60000120BB490870FFF7E4FA20B1B9A003F055
:10AD700027FF012010BDB8A003F022FF0020F9E753
:10AD800010B52A20F6F794FBFFF7B7FE044603F050
:10AD900022FF0D20F6F78CFB10BD10B52A20F6F728
:10ADA00087FBFFF76EFE044603F015FF0D20F6F754
:10ADB0007FFB10BD10B5A948007800283FD1FFF7F0
:10ADC0004EFE01283DD1FFF7E7FDA148007801289C
:10ADD00031D19F48807800282DDD9D48C07800281B
:10ADE00029DD01210420FAF70BFE00209C490860B0
:10ADF00001209A490870FFF780FE18B999489A49CE
:10AE0000086005E092498868FFF740F996490860B4
:10AE10008F480079401C8E49087108799249096869
:10AE2000FFF73CFEFFF785FA002090490860FFF726
:10AE3000C9F8012010BDFFF74CF80020FAE7FFF732
:10AE400048F80020F6E7F8B5054600260027FFF78A
:10AE500006FE012829D12846FFF761FE064628464E
:10AE6000FFF783FE074600F031FC00903146009862
:10AE700000F0F9FCA0B114207D490880FFF7CFF95C
:10AE8000002408E014207A4908800098FFF791F91F
:10AE9000F6F7C5FB641CBC42F4D30020744908805B
:10AEA000F6F7BDFB684600F046FCF6F7B8FB00205D
:10AEB000F6F7FEFA0020F6F7FBFA0020F6F7F8FAAC
:10AEC000F8BD70B50446FFF7CAFD01280CD12A2051
:10AED000F6F7EEFA2046FFF748FE054603F0C8FEF7
:10AEE0000D20F6F7E5FA08E02A20F6F7E1FA30201F
:10AEF000F6F7DEFA0D20F6F7DBFA70BD1CB5FFF7AA
:10AF0000CBF810B300F0E2FB019014205849088000
:10AF1000FFF785F90EE001226946019800F023FC55
:10AF200020B19DF80000F6F7C3FA00E009E0142014
:10AF30004F490880019800F0AEFC45498968884275
:10AF4000E9D300BF01A800F0F6FB1CBD4348007820
:10AF50007047012047490870704770B5044645485E
:10AF60000078002863D0207834285CD160783028BD
:10AF700057D100202070A078352838D008DCA0F107
:10AF8000300005284BD2DFE800F01011152B2F0000
:10AF9000382835D004DC36282CD037283FD12CE097
:10AFA00039282ED046283AD12CE038E0201DFFF772
:10AFB0001CFE34E0207903F0A3FF642100FB01F6BE
:10AFC000607903F09DFF00EB800006EB4006A0795E
:10AFD00003F096FF3044C5B22846FFF72DFC1EE073
:10AFE000201DFFF770FC1AE0FFF77AFE17E0FFF76D
:10AFF00084FD14E0FFF733FD11E0FFF7B3FC0EE032
:10B000000DE00CE000201C4908700220F6F750FA11
:10B010003120F6F74DFA0320F6F74AFA00BF00BFD9
:10B0200000BF00BF00BF00BF00201249087070BD04
:10B0300010B50446114801880088401C0F4A108052
:10B040000F4844540D2C01D1FFF74BFB10BD0000FD
:10B05000384B00202A310D002A300D000401002059
:10B060004000002000C20D0000010020FC00002074
:10B070000E010020070100202C000020F800002015
:10B08000444B00202DE9F84F04464FF0040B0620F6
:10B0900000904FF03F0A00E0641C20783A28FBD172
:10B0A000641C2078642817D1641C641C002507E008
:10B0B00014F8010B303805EB850100EB410085B237
:10B0C00035F026F900682178405C2028F0D0002D6A
:10B0D00001DD05F0FF0B641C20786F280CD1641C87
:10B0E000641C14F8010B303885B2032D03DB072DE7
:10B0F00001DCE8B20090641C2078622814D1641C42
:10B10000641C002507E014F8010B303805EB8501BD
:10B1100000EB410085B235F0FBF800682178405C17
:10B120002028F0D0AA46641CBAF1000F01D1BDE876
:10B13000F88F4EF6602090FBFAF0870080E0002543
:10B1400007E014F8010B303805EB850100EB4100F6
:10B1500085B235F0DDF800682178405C2028F0D019
:10B1600015B1B7FBF5F601E0B7FBFBF64FF00008B1
:10B170002078652816D008DC61281CD062281DD0F4
:10B18000632809D064281CD109E066280DD06728FF
:10B190000ED0702815D115E04FF0010815E04FF0E2
:10B1A000030812E04FF005080FE04FF006080CE02E
:10B1B0004FF0080809E04FF00A0806E04FF00C08CD
:10B1C00003E000BF4FF0000800BF00BF641C207800
:10B1D000232804D108F1010000F0FF08641C207846
:10B1E0002E2802D106EB5606641C35F091F8006853
:10B1F0002178405C202805D12078303800F0FF0904
:10B20000641C01E0DDF8009009F0FF0920782C288B
:10B2100000D1641CB8F1000F0FD0B1B2A9F1040243
:10B2200002EB420208EB8202084B33F81200FAF7F5
:10B2300018FCB0B204F04EFD02E0B0B204F04AFDDA
:10B24000207800287FF47BAF00BF70E71201002058
:10B2500001460020CAB21044C1F307221044C1F3D2
:10B2600007421044C0B270472DE9F0410446250E54
:10B2700024F07F463046FFF7EBFF0746BD4202D081
:10B280000020BDE8F0813046FBE72DE9F0410025C4
:10B29000002409E0E006070E074850F824603078E3
:10B2A000B8400543601CC4B2042CF3D3ED432846D8
:10B2B000FFF7DAFFBDE8F081401604085D487047EB
:10B2C0005D48704770B5FFF7FBFF0446A07808B9EA
:10B2D00000250EE072B6E078255CA078401EA070D4
:10B2E000E178481C00EBD0714910A0EB4101E170FE
:10B2F00062B6284670BD2DE9F0410646FFF7E0FF33
:10B300000446A078022803D1FFF7DCFF054600BF02
:10B3100072B6E178A278881800EBD0714910A0EBE2
:10B320004101CFB2E655A078401CA07062B6BDE8DE
:10B33000F08170B5FFF7C2FF0446FFF7C1FF054675
:10B34000002060802071A870E87032203B4908809E
:10B3500005203B49088070BD49B103785A1C027032
:10B36000052B0BDD052202700122027106E0037835
:10B370005A1E027013B1002202700271704770B53C
:10B38000FFF79CFF0446432006F0E0FB05462946F4
:10B390002046FFF7E1FF207910B360884FF6FF7178
:10B3A000884209DA6188481C608029B924480188EC
:10B3B00022480088FAF755FB608840F2DC51884249
:10B3C00025D12048007800F0020000B34FF49671B8
:10B3D0004FF4FA60FAF745FB0220FFF78CFF16E006
:10B3E0006088032811DD608840F2DC5188420CDA65
:10B3F0001448007800F0010038B132214FF47A602F
:10B40000FAF72FFB0120FFF776FF0020608070BD68
:10B4100029B10C4A127802430A4B1A7004E0094A17
:10B4200012788243074B1A707047044A1080044A0E
:10B43000118070477A0100208001002076010020F1
:10B44000780100207401002010B50121402030F067
:10B45000EAF901212B4831F068FB0021294831F03D
:10B4600009FC0021274831F0CEFD4FF0FF3125487F
:10B4700031F0CBFD012240F25721224831F0F7FB99
:10B4800010BD2DE9F04706464FF00009CA4605E019
:10B49000A6F5803609F101001FFA80F9B6F5803F64
:10B4A000F6D2184831F0CFFD85B2A81987B22C46E4
:10B4B000A04610E04FF0000A08E0124831F0C3FD4A
:10B4C00084B2444501DA4FF0010AA046BAF1000FF8
:10B4D000F3D0AC42F1DB5FEA0900A9F101011FFAE8
:10B4E00081F9E7D1AF4205DA00BF064831F0ABFD84
:10B4F000B842FAD800BF034831F0A5FDB842FAD9E6
:10B50000BDE8F087001800400146E84BB3F800386A
:10B51000CA1A0020E64B9B5C6BB1E44BB3F80038D1
:10B520008B4208D8E14BB3F800381B1D8B4202D97F
:10B53000DE4B03EB42207047DC4AB2F80028811A48
:10B54000DA4AB2F80028824208D8D84AB2F800286D
:10B55000121D824202D90023D54A535470472DE967
:10B56000F04105466F02002403E00021D048015558
:10B57000641C042CF9D30423DA013946CB4833F098
:10B58000A2FA0646C949A1F800582A2E07D100247C
:10B5900003E00121C6480155641C042CF9D3304650
:10B5A000BDE8F08110B504464FF40070A4F8000225
:10B5B0000146204635F07CF910BD2DE9F0410646E4
:10B5C0000F463846FFF7A0FF05460DB12A2407E0D5
:10B5D0003846FFF7C4FF04463846FFF795FF054697
:10B5E00045B14FF400722946304635F0EAF80020A4
:10B5F000A6F800022046BDE8F08170B505460C466D
:10B6000066022046FFF798FF4FF400723146284645
:10B6100033F09AFC70BD0246B1F5007F03D2A2F868
:10B620000012012070470020FCE70146B1F800023B
:10B6300070470146B1F80002C0F5007080B2704753
:10B6400070B504460E4615462046FFF7F2FFA842A5
:10B650000DDBB4F8001208192A46314635F0B1F86E
:10B66000B4F800022844A4F80002012070BD0020B4
:10B67000FCE770B504460E4615462046FFF7D9FF95
:10B68000A8420DDBB4F8000201192A46304635F015
:10B6900098F8B4F800022844A4F80002012070BD14
:10B6A0000020FCE770B504460D46824885420BD267
:10B6B000294604F10800FFF780FF207020782A282F
:10B6C00002D16560012070BD0020FCE770B5002547
:10B6D00000242BE07848005D30BB012076490855F6
:10B6E00004EB440101EBC411744A02EB810101F146
:10B6F0000800FFF757FF4FF0FF3004EB440101EB68
:10B70000C4116E4A02EB810148602A2004EB440117
:10B7100001EBC41102F8210004EB440000EBC4105B
:10B72000114601EB800503E0601CC4B20A2CD1D3A2
:10B7300000BF284670BD0146002010E000EB40022B
:10B7400002EBC0125D4B03EB82020B689A4204D1FC
:10B7500000220A60584B1A5403E0421CD0B20A2857
:10B76000ECD300BF70472DE9F047044688461646E3
:10B77000002528E004F10800FFF75BFF8146B9F1DE
:10B78000000F0DD16068411C2046FFF78BFF10B9F8
:10B790000020BDE8F08704F10800FFF74AFF81466A
:10B7A000701B484501DD484600E0701B87B208EB7E
:10B7B00005013A4604F10800FFF75BFF08B90020D5
:10B7C000E7E7E81985B2B542D4DB0120E1E710B51F
:10B7D000044604F108006168FFF70FFF207020782D
:10B7E0002A2801D1012010BD0020FCE72DE9F047F7
:10B7F00004468846164600252EE004F10800FFF7AF
:10B8000018FF8146B9F1000F13D12046FFF7DFFF83
:10B8100010B90020BDE8F0876068411C2046FFF7A2
:10B8200041FF08B90020F5E704F10800FFF701FF28
:10B830008146701B484501DD484600E0701B87B219
:10B8400008EB05013A4604F10800FFF7F9FE08B9D4
:10B850000020DFE7E81985B2B542CEDB0120D9E749
:10B860000146087870472DE9F04104460D466E0AFE
:10B87000C5F308076068B04207D031462046FFF79D
:10B8800011FF10B90020BDE8F081B9B204F1080041
:10B89000FFF7C1FEF7E710B5044604F10800FFF713
:10B8A000C4FE616800EB412010BD0000A0680020CC
:10B8B000A2700020FFFF7F00946800201C5400202D
:10B8C00030B502466FF000458A4201D9104600E0CB
:10B8D000084603468A4201D2104600E00846044664
:10B8E000181BB0F1004F05D38A4201D8012030BDAA
:10B8F0000020FCE78A4201D30120F8E70020F6E7A8
:10B90000002007E0FF2100EB4002424B03F8221029
:10B91000411C88B21428F5D300213F4A116001214F
:10B920003E4A117070473C480068401C3A49086024
:10B93000704739480068704770B53848007808B9D2
:10B94000FFF7DEFF002420E004EB4400314911F84A
:10B950002000FF2817D004EB44020B4603EB8202C1
:10B9600051682D4A1068FFF7ABFF60B104EB44004B
:10B97000284901EB80008568FF2004EB4401254A3B
:10B9800002F82100A847601C84B2142CDCD370BDDF
:10B9900030B502460B46002121E072B601EB4100B2
:10B9A0001C4C14F82000FF2816D101EB4104194D5E
:10B9B00005F8241001EB41002C4604EB80004260A6
:10B9C00001EB410004EB8000836062B601EB4100B3
:10B9D000104C14F8200030BD62B6481C81B2142906
:10B9E000DBD3FF20F7E710B501460A4672B602EB3B
:10B9F0004200084B13F82000884208D1FF2002EBD8
:10BA00004203044C04F8230062B6012010BD62B664
:10BA10000020FBE7A870002088010020840100209E
:10BA200010B58A082E4B18601B6803EB82032D4C5F
:10BA300023602B4B1B682C4C236001232B4C237061
:10BA400010BD70B504460D462848007808B900209E
:10BA500070BD274831F0F7FA234909680880224869
:10BA60000068847020480068C5701F480068001D89
:10BA70001D490860084600681A490968884203D3CE
:10BA800017480068184908600120E1E70146154899
:10BA90000068814201D900207047081D114A1268D0
:10BAA00090420AD1104800680D4A1268904201D1B4
:10BAB0000020F1E70A480068EEE7081D0A4A12680C
:10BAC000904201D10020E7E7081DE5E70020074983
:10BAD00008700548006870470120044908707047E5
:10BAE0008C0100209001002094010020980100208A
:10BAF0000018004010B502460B4619460020D081C0
:10BB00009081002416E008785B2810D008785D2822
:10BB10000DD008782D280AD008787C2807D008781E
:10BB2000302802DB0878392801DD002010BD601CB8
:10BB300084B2491C0878202802D008780028E2D175
:10BB4000136093601068204450600120EEE770B5E8
:10BB500004460D46A089E189884206DAA089401C86
:10BB6000A081A0892880012070BD02E0A068401C4F
:10BB7000A060A06800785B28F8D0A06800785D28F5
:10BB8000F4D0A06800787C28F0D0D4E90110884275
:10BB900001D10020E8E7A06834F08AFDA081A089E7
:10BBA000288002E0A068401CA060A06800783028CF
:10BBB00003DBA06800783928F4DDA06800782D2820
:10BBC00012D1A068401CA060A06834F071FDE08133
:10BBD00002E0A068401CA060A0680078302803DB69
:10BBE000A06800783928F4DD0120BDE71CB50120EC
:10BBF0008DF8040002208DF8050000208DF8060065
:10BC000001208DF80700182001F0C9FF00901820CE
:10BC100001F0C0FF044669462FF096F902208DF826
:10BC20000700172001F0BBFF0090172001F0B2FFC2
:10BC3000044669462FF088F900208DF804000220A0
:10BC40008DF8050000208DF8060001208DF8070012
:10BC5000192001F0A4FF0090192001F09BFF044679
:10BC600069462FF071F91A2001F099FF00901A200F
:10BC700001F090FF044669462FF066F9152001F0A7
:10BC80008EFF0090152001F085FF044669462FF0D5
:10BC90005BF9162001F083FF0090162001F07AFF77
:10BCA000044669462FF050F90A2004F013F80121E8
:10BCB000182005F01FFF0021172005F01BFF3C2076
:10BCC00004F008F81CBD2DE9F047002600270025E8
:10BCD000A8460120F9F7E7FB01210846FFF798FB8A
:10BCE000F8F7EFF80024FE48C07841280AD1F8F7A9
:10BCF00014F806461EB9FBA002F062FF02E0FCA0A9
:10BD000002F05EFFF648C07842280BD1FEF7A7FE8E
:10BD10000746012F03D1F9A002F052FF02E0FAA07A
:10BD200002F04EFFEE48C07843281BD10020F949AD
:10BD3000086000BFF5F773FCFFF7C4FA8046B8F15E
:10BD4000010F00D101242CB9F248006842F21071B1
:10BD50008842EFD91CB9F0A002F032FF02E0F1A056
:10BD600002F02EFFDE48C07844280CD14FF4167242
:10BD70004FF47A711046F9F799FB0F20F9F75DFB44
:10BD8000EBA002F01DFFD648C07845280FD1002057
:10BD9000F9F789FB00210120FFF73AFBF8F74BFC8C
:10BDA0000024E6A002F00CFFE7A0FFF76BF9CC48F7
:10BDB000C07846282BD10020F9F775FB002500201C
:10BDC000D449086002F083FE814602F004FFCAA055
:10BDD00002F0F6FE00BF02F07AFE1E2800DA01250E
:10BDE0002DB9CC48006842F210718842F3D902F0B4
:10BDF0006EFE814602F0EFFEBFA002F0E1FE1DB92B
:10BE0000DCA002F0DDFE02E0DDA002F0D9FEBDE81C
:10BE1000F08770B50025002406E04FF6FF70DB497F
:10BE200021F81400601C04B2282CF6D3002406E08C
:10BE30004FF6FF70D64921F81400601C04B2B4F527
:10BE4000FA7FF5DD0020F7F775FA0022082142F6A7
:10BE5000A000F7F7C3F80F2207210420F5F7F8FF39
:10BE6000142003F037FF0121462005F043FE012195
:10BE7000452005F03FFE012003F02CFF0021452066
:10BE800005F038FE052003F025FF5420BF49088047
:10BE90004FF6FF7048800021052003F0A6FE3220F7
:10BEA00003F018FF0121452005F024FE07220F2191
:10BEB0000420F5F7CDFF142003F00CFF0020954976
:10BEC0000860B449088000BFF5F7A9FBB1480088B5
:10BED000012803DA8F480068B428F5D98D48006836
:10BEE000B42801D3022506E0A9480088652801D1BD
:10BEF000012500E00325284670BD70B5002500240B
:10BF000006E04FF6FF70A14921F81400601C04B24E
:10BF1000282CF6D3002406E04FF6FF709C4921F848
:10BF20001400601C04B2B4F5FA7FF5DD0020F7F7C9
:10BF300001FA0022082142F6A000F7F74FF8072285
:10BF40000F210420F5F784FF142003F0C3FE012124
:10BF5000462005F0CFFD0121452005F0CBFD002056
:10BF60006C4908608B49088000BFF5F758FB894889
:10BF70000088012804DA67480068B0F5FA6FF4D940
:10BF800064480068B0F5FA6F01D3022548E08048A4
:10BF90000088542843D10F2207210420F5F758FFC9
:10BFA000142003F097FE0125002406E04FF6FF70F1
:10BFB000764921F81400601C04B2282CF6D3002422
:10BFC00006E04FF6FF70724921F81400601C04B2BD
:10BFD000B4F5FA7FF5DD0121462005F08BFD012146
:10BFE000452005F087FD012003F074FE0021452067
:10BFF00005F080FD962003F06DFE65206349088002
:10C000004FF6FF7048800021052003F0EEFD32203E
:10C0100003F060FE0121452005F06CFD00E00325E2
:10C02000284670BD70B50025002406E04FF6FF706D
:10C03000564921F81400601C04B2282CF6D30024C1
:10C0400006E04FF6FF70524921F81400601C04B25C
:10C05000B4F5FA7FF5DD0020F7F76CF9002208212E
:10C0600042F6A000F6F7BAFF0F2207210420F5F7E9
:10C07000EFFE142003F02EFE0121452005F03AFDCD
:10C080000121462005F036FD012003F023FE0021AA
:10C09000462005F02FFD002406E04FF6FF703B49D7
:10C0A00021F81400601C04B2282CF6D3002406E00A
:10C0B0004FF6FF70364921F81400601C04B2B4F545
:10C0C000FA7FF5DD962003F005FE0121452005F0FD
:10C0D00011FD0121462005F00DFD01205CE000006E
:10C0E000741400202A393138415F4641494C0D0013
:10C0F0002A393138415F4F4B0D0000002A39313861
:10C10000425F4F4B0D0000002A393138425F4641F3
:10C11000494C0D00380000202A393138435F464130
:10C12000494C0D002A393138435F4F4B0D00000058
:10C130002A393138445F4F4B0D0000002A3931381D
:10C14000455F4F4B0D0000005553423A643D382C7B
:10C150006F3D352C623D3136303A3136612C313607
:10C16000672C3136612C313661232C63362C6336D3
:10C17000000000002A393138465F4641494C0D0025
:10C180002A393138465F4F4B0D000000F81200206D
:10C19000040800201600002003F09CFD002146202A
:10C1A00005F0A8FC5620FE4908804FF6FF70488035
:10C1B0000121052003F019FD0121462005F09AFC1C
:10C1C0000020F8490860F849088000BFF5F727FA11
:10C1D000F5480088012803DAF2480068B428F5D948
:10C1E000F0480068B42801D3022506E0EF48008833
:10C1F000672801D1012500E00325284670BD70B5F0
:10C200000025002406E04FF6FF70E54921F81400F0
:10C21000601C04B2282CF6D3002406E04FF6FF7011
:10C22000E24921F81400601C04B2B4F5FA7FF5DD90
:10C230000020F7F77FF80022082142F6A000F6F769
:10C24000CDFE0F2207210420F5F702FE142003F093
:10C2500041FD0121462005F04DFC0121452005F05E
:10C2600049FC0020CF490860CF49088000BFF5F79E
:10C27000D6F9CD480088012805DACA48006840F69A
:10C2800054318842F3D9C748006840F65431884297
:10C2900001D302253DE0C5480088562838D1002446
:10C2A00006E04FF6FF70BE4921F81400601C04B28E
:10C2B000282CF6D3002406E04FF6FF70BB4921F886
:10C2C0001400601C04B2B4F5FA7FF5DD01214620AC
:10C2D00005F010FC012003F0FDFC0021462005F0D4
:10C2E00009FC0121452005F005FC6720AC490880C8
:10C2F0004FF6FF7048800121052003F076FC3220C4
:10C3000003F0E8FC0121462005F0F4FB012500E0E4
:10C310000325284670BD70B58CB0002400260E227F
:10C3200006210120F5F794FD142003F0D3FC002032
:10C330004FF4FC6101230246CDE9001019464FF489
:10C34000FA7008F088F800204FF4FD6102230246DD
:10C35000CDE90010014608F07EF800220221944841
:10C3600030F0E6FF00220821914830F0E1FF002282
:10C370004FF400418E4830F0DBFF00224FF40061A3
:10C380008B4830F0D5FF00224FF48071884830F0A0
:10C39000CFFF962003F09EFC01208DF820000220A4
:10C3A0008DF8210003208DF8220004208DF8230051
:10C3B00005208DF8240006208DF8250007208DF833
:10C3C000260008208DF8270000BF04E000200AA9FD
:10C3D0000855601C84B2082CF8DB01203223024689
:10C3E00008A90090082008F0B5F800206D49086001
:10C3F000002506E06F496E4831F05AF90546F5F719
:10C400000EF91DB967480068B428F3D3EDB303AA49
:10C410000021674831F0A5F89DF817008DF8280035
:10C420009DF818008DF829009DF819008DF82A0054
:10C430009DF81A008DF82B009DF81B008DF82C003C
:10C440009DF81C008DF82D009DF81D008DF82E0024
:10C450009DF81E008DF82F009DF8280015281FD18B
:10C460009DF8290016281BD19DF82A00172817D1FE
:10C470009DF82B00182813D19DF82C0019280FD1F6
:10C480009DF82D001A280BD100E00BE09DF82E003E
:10C490001B2805D19DF82F001C2801D1012602E0A0
:10C4A000032600E00226FAF77BFC0122082140481F
:10C4B00030F03EFF0122D1033D4830F039FF012228
:10C4C000D1023B4830F034FF01221102384830F0ED
:10C4D0002FFF30460CB070BD70B58AB00024002626
:10C4E0000E2206210120F5F7B3FC142003F0F2FB25
:10C4F00000204FF4FD6101230246CDE900101946EA
:10C500004FF4FA7007F0A7FF00204FF4FC610223FC
:10C510000246CDE90010014607F09DFF00220221EE
:10C52000234830F005FF00220821214830F000FFA9
:10C5300000224FF400411E4830F0FAFE00224FF472
:10C5400000611B4830F0F4FE00224FF4807118485F
:10C5500030F0EEFE012003F0BDFB00BF04E0002040
:10C5600008A90855601C84B2082CF8DB012003F0F0
:10C57000B1FB00200B490860002506E00D490C487E
:10C5800031F096F80546F5F74AF82DB905480068E8
:10C5900040F654318842F1D3002D78D003AA0BE045
:10C5A000F8120020380000201600002004080020A7
:10C5B00000680040030000120021FE4830F0D1FF67
:10C5C0009DF817008DF820009DF818008DF82100C7
:10C5D0009DF819008DF822009DF81A008DF82300AF
:10C5E0009DF81B008DF824009DF81C008DF8250097
:10C5F0009DF81D008DF826009DF81E008DF827007F
:10C600009DF82000012840D19DF8210002283CD14E
:10C610009DF82200032838D19DF82300042834D146
:10C620009DF82400052830D19DF8250006282CD13E
:10C630009DF82600072828D1012615208DF8200016
:10C6400016208DF8210017208DF8220018208DF873
:10C65000230019208DF824001A208DF825001B20B6
:10C660008DF826001C208DF82700962003F032FB61
:10C6700001203223024608A90090082007F06AFF33
:10C68000322003F027FB03E001E0032600E002264E
:10C69000FAF786FB01220821C64830F049FE012244
:10C6A000D103C44830F044FE0122D102C14830F029
:10C6B0003FFE01221102BF4830F03AFE30460AB078
:10C6C00070BD002070470020704710B588B000246E
:10C6D0003820B9490870052203210846F5F7B8FB50
:10C6E000142003F0F7FAFBF799F9962003F0F2FA19
:10C6F0000820072106220523CDE90432CDE90610E2
:10C700000420032102220123CDE90032CDE90210E9
:10C7100037231A4619460B20FBF709FC0020A749CE
:10C720000880A7490880F4F77AFF0020A54908800F
:10C73000A549086000BFA3480088012802D1002055
:10C740009F490880A0480068B42803D89D48008805
:10C750000028F0D09C480068B42801D3022424E0CB
:10C76000FBF7D7FC9548008909281DD193484089DB
:10C770000A2819D1914880890B2815D18F48C08982
:10C780000C2811D18D48008A0D280DD18B48408A84
:10C790000E2809D18948808A0F2805D18748C08A88
:10C7A000102801D1012400E00324204608B010BD68
:10C7B00010B588B0002437207F4908700522032176
:10C7C0000846F5F745FB142003F084FAFBF726F939
:10C7D000022003F07FFA00207A490880F4F71FFF57
:10C7E0000020794908607549088001E0F4F717FFD7
:10C7F0007548006840F65431884203D87148008873
:10C800000028F3D07048006840F65431884201D3C4
:10C81000022440E0FBF77DFC68480089012839D1FB
:10C8200066484089022835D164488089032831D17F
:10C830006248C08904282DD16048008A052829D182
:10C840005E48408A062825D15C48808A072821D185
:10C850005A48C08A08281DD1962003F03BFA1020C0
:10C860000F210E220D23CDE90432CDE906100C2054
:10C870000B210A220923CDE90032CDE90210382329
:10C880001A4619460B20FBF752FB322003F022FA1E
:10C89000012400E00324204608B010BD70B5002636
:10C8A000FFF7A4F90A2202210846F5F7D1FA14206D
:10C8B00003F010FA0021182005F01CF9142003F0F1
:10C8C00009FA0121182005F015F9322003F002FAC7
:10C8D00000203D490860002500BFF4F7A0FE1920A4
:10C8E00005F034F905461DB937480068B428F4D975
:10C8F00035480468B42C01D302261BE000203249DD
:10C90000086000BFF4F78BFE1A2005F01FF90546FA
:10C910001DB12D480068B428F4D92B480468B42C04
:10C9200001D3022606E00F2C03D3192C01D80126CF
:10C9300000E00326012E01D0304670BD642003F0D4
:10C94000C9F90121172005F0D5F8142003F0C2F928
:10C950000021172005F0CEF8282003F0BBF90020B5
:10C9600019490860012500BFF4F759FE152005F0AC
:10C97000EDF805461DB114480068B428F4D91248F2
:10C980000468B42C01D3022627E000200E49086079
:10C9900000BFF4F744FE162005F0D8F805461DB98F
:10C9A00009480068B428F4D907480468B42C0DD3AA
:10C9B000022612E000680040A80000205403002076
:10C9C000120000201C000020380000200F2C03D390
:10C9D000192C01D8012600E003263046ADE770B5DA
:10C9E0000026FFF703F90A2202210846F5F730FA7C
:10C9F000142003F06FF90020FE490860002500BFF5
:10CA0000F4F70DFE192005F0A1F8054625B9F948FF
:10CA10000068B0F5FA6FF3D9F6480468B4F5FA6F18
:10CA200001D302261BE00020F249086000BFF4F7A2
:10CA3000F6FD1A2005F08AF805461DB1ED4800689C
:10CA4000B428F4D9EB480468B42C01D3022606E0DC
:10CA50000F2C03D3192C01D8012600E00326012E48
:10CA600001D0304670BD642003F034F90021182055
:10CA700005F040F8142003F02DF90121182005F0ED
:10CA800039F8322003F026F90020DA490860012540
:10CA900000BFF4F7C4FD152005F058F805461DB198
:10CAA000D4480068B428F4D9D2480468B42C01D31F
:10CAB00002261BE00020CF49086000BFF4F7AFFD5D
:10CAC000162005F043F805461DB9CA480068B42889
:10CAD000F4D9C8480468B42C01D3022606E00F2C10
:10CAE00003D3192C01D8012600E00326642003F0AB
:10CAF000F1F80121172004F0FDFF142003F0EAF8FB
:10CB00000021172004F0F6FF282003F0E3F8304658
:10CB1000A8E770B50025002406E04FF6FF70B6497F
:10CB200021F81400601C04B2282CF6D3002406E07F
:10CB30004FF6FF70B14921F81400601C04B2B4F53F
:10CB4000FA7FF5DD0120F6F7F5FB0022082142F619
:10CB5000A000F6F743FA092208210520F5F778F935
:10CB6000962003F0B7F8052003F0B4F85420A2494A
:10CB700008804FF6FF7048800021052003F035F84B
:10CB8000322003F0A7F8142003F0A4F800209949FC
:10CB900008609B49088000BFF4F741FD9848008871
:10CBA000012803DA93480068B428F5D99148006851
:10CBB000B42801D3022506E090480088652801D1F9
:10CBC000012500E00325284670BD70B5002500242E
:10CBD00006E04FF6FF70884921F81400601C04B28B
:10CBE000282CF6D3002406E04FF6FF70834921F885
:10CBF0001400601C04B2B4F5FA7FF5DD0120F6F7ED
:10CC000099FB0022082142F6A000F6F7E7F9092275
:10CC100008210520F5F71CF9142003F05BF800202B
:10CC2000744908607649088000BFF4F7F8FC74483E
:10CC30000088012805DA6F48006840F654318842C0
:10CC4000F3D96C480068B0F5FA6F01D3022530E0E3
:10CC50006A48008854282BD1142003F03BF80125A2
:10CC6000002406E04FF6FF70634921F81400601CB1
:10CC700004B2282CF6D3002406E04FF6FF705F497B
:10CC800021F81400601C04B2B4F5FA7FF5DD96209B
:10CC900003F020F86520584908804FF6FF7048805F
:10CCA0000021052002F0A1FF322003F013F800E07C
:10CCB0000325284670BD70B58CB0002400260121E4
:10CCC0002E2004F017FF01212D2004F013FF012274
:10CCD00008210846F5F7BCF8142002F0FBFF0020FD
:10CCE0004FF4FC6101230246CDE9001019462120D2
:10CCF00007F0F5FB00204FF4FD6102230246CDE969
:10CD00000010014607F0EBFB962002F0E3FF002243
:10CD100002213C4830F00CFB00220821394830F059
:10CD200007FB00224FF40041364830F001FB00229F
:10CD30004FF40061334830F0FBFA00224FF4807169
:10CD4000304830F0F5FA01208DF8200002208DF8EF
:10CD5000210003208DF8220004208DF823000520F7
:10CD60008DF8240006208DF8250007208DF8260078
:10CD700008208DF8270004E000200AA90855601C4F
:10CD800084B2082CF8DB01207323024608A9009026
:10CD9000082007F0DFFB002016490860002506E0A8
:10CDA0001949184830F084FC0546F4F738FC1DB9E1
:10CDB00010480068B428F3D3DDB103AA002111485C
:10CDC00030F0CFFB9DF817008DF828009DF8180073
:10CDD0008DF829009DF819008DF82A009DF81A0099
:10CDE0008DF82B009DF81B008DF82C009DF81C0081
:10CDF0000CE039E038000020F81200200408002080
:10CE00001600002000680040030000128DF82D007D
:10CE10009DF81D008DF82E009DF81E008DF82F0046
:10CE20009DF8280015281DD19DF82900162819D134
:10CE30009DF82A00172815D19DF82B00182811D12C
:10CE40009DF82C0019280DD19DF82D001A2809D124
:10CE50009DF82E001B2805D19DF82F001C2801D11C
:10CE6000012602E0032600E00226F9F799FF0122DD
:10CE70000821FE4830F05CFA0122D103FB4830F073
:10CE800057FA0122D102F94830F052FA0122110278
:10CE9000F64830F04DFA30460CB070BD70B58AB02F
:10CEA0000024002601212E2004F024FE01212D2043
:10CEB00004F020FE012208210846F4F7C9FF1420DF
:10CEC00002F008FF00204FF4FD6101230246CDE986
:10CED00000101946212007F002FB00204FF4FC61EE
:10CEE00002230246CDE90010014607F0F8FA0022BD
:10CEF0000221DE4830F01CFA00220821DB4830F025
:10CF000017FA00224FF40041D84830F011FA0022FD
:10CF10004FF40061D54830F00BFA00224FF48071D5
:10CF2000D24830F005FA012002F0D4FE00BF04E040
:10CF3000002008A90855601C84B2082CF8DB0120E9
:10CF400002F0C8FE0020CA490860002506E0C94971
:10CF5000C64830F0ADFB0546F4F761FB2DB9C44877
:10CF6000006840F654318842F1D3002D6AD003AAFC
:10CF70000021BE4830F0F5FA9DF817008DF820002A
:10CF80009DF818008DF821009DF819008DF82200F9
:10CF90009DF81A008DF823009DF81B008DF82400E1
:10CFA0009DF81C008DF825009DF81D008DF82600C9
:10CFB0009DF81E008DF827009DF8200001283FD124
:10CFC0009DF8210002283BD19DF82200032837D18B
:10CFD0009DF82300042833D19DF8240005282FD183
:10CFE0009DF8250006282BD19DF82600072827D17B
:10CFF000012615208DF8200016208DF8210017201D
:10D000008DF8220018208DF8230019208DF82400B7
:10D010001A208DF825001B208DF826001C208DF885
:10D020002700962002F056FE01207323024608A92D
:10D030000090082007F08EFA322002F04BFE02E04A
:10D04000032600E00226F9F7ABFE012208218748FB
:10D0500030F06EF90122D103844830F069F90122E1
:10D06000D102824830F064F9012211027F4830F089
:10D070005FF930460AB070BD70B50025002406E0A7
:10D080004FF6FF707C4921F81400601C04B2282C74
:10D09000F6D3002406E04FF6FF70784921F814001B
:10D0A000601C04B2B4F5FA7FF5DD0220F6F742F910
:10D0B0000022082142F6A000F5F790FF0D220C2176
:10D0C0000620F4F7C5FE142002F004FE052002F04D
:10D0D00001FE5420684908804FF6FF704880002107
:10D0E000052002F082FD322002F0F4FD142002F04F
:10D0F000F1FD00205E4908606149088000BFF4F737
:10D100008EFA5F480088012803DA59480068B4287D
:10D11000F5D957480068B42801D3022506E05748DE
:10D120000088652801D1012500E00325284670BD4F
:10D1300070B50025002406E04FF6FF704E4921F837
:10D140001400601C04B2282CF6D3002406E04FF62D
:10D15000FF704A4921F81400601C04B2B4F5FA7F4C
:10D16000F5DD0220F6F7E6F80022082142F6A000DD
:10D17000F5F734FF0C220D210620F4F769FE142088
:10D1800002F0A8FD00203A4908603D49088000BF30
:10D19000F4F745FA3A480088012804DA3448006870
:10D1A000B0F5FA6FF4D932480068B0F5FA6F01D3E0
:10D1B000022530E03148008854282BD1142002F099
:10D1C00089FD0125002406E04FF6FF702A4921F869
:10D1D0001400601C04B2282CF6D3002406E04FF69D
:10D1E000FF70264921F81400601C04B2B4F5FA7FE0
:10D1F000F5DD962002F06EFD65201F4908804FF690
:10D20000FF7048800021052002F0EFFC322002F080
:10D2100061FD00E00325284670BD70B5012600259C
:10D2200006E04FF6FF70144921F81500681C85B21E
:10D23000282DF6D3002506E04FF6FF700F4921F8A0
:10D240001500681C85B2B5F5FA7FF5DD0020F6F70C
:10D2500071F80022082142F6A000F5F7BFFE012177
:10D26000452004F047FC01200CE00000006800406D
:10D270003800002003000012F812002004080020EB
:10D280001600002002F026FD0021452004F032FCAB
:10D290000121462004F02EFC012442E022B20F219D
:10D2A0000420F4F7D5FD142002F014FD962002F0BE
:10D2B00011FD04F16000FE4908804FF6FF704880C0
:10D2C0000021052002F091FC0F2221B20420F4F786
:10D2D000BFFD142002F0FEFC0020F6490860F6496C
:10D2E000088000BFF4F79BF9F3480088012803DAAF
:10D2F000F0480068B428F5D9EE480068B42801D396
:10D3000002260EE0ED48018804F15000814207D169
:10D31000601C84B2042C01D1A01C84B2012600E060
:10D320000326102C01DA012EB8D0304670BD70B53E
:10D330000126002506E04FF6FF70DD4921F81500B3
:10D34000681C85B2282DF6D3002506E04FF6FF7045
:10D35000DA4921F81500681C85B2B5F5FA7FF5DDCC
:10D360000020F5F7E7FF0022082142F6A000F5F7BC
:10D3700035FE0121462004F0BDFB0121452004F0CB
:10D38000B9FB012002F0A6FC0021452004F0B2FB0D
:10D39000012447E00F2221B20420F4F759FD1420A4
:10D3A00002F098FC0020C3490860C349088000BF10
:10D3B000F4F735F9C0480088012804DABD48006850
:10D3C000B0F5FA6FF4D9BB480068B0F5FA6F01D335
:10D3D000022627E0B948018804F16000814220D18B
:10D3E00022B20F210420F4F733FD142002F072FC66
:10D3F000962002F06FFC04F15000AD4908804FF612
:10D40000FF7048800021052002F0EFFB322002F07F
:10D4100061FC601C84B2042C01D1A01C84B20126E2
:10D4200000E00326102C01DA012EB3D0304670BD87
:10D4300070B58AB00120A2490880A2490870002175
:10D44000084604F057FB0025002403E000204DF8B7
:10D450002400641C0A2CF9D300209B490880002476
:10D4600001F076FF99480079312821D10026FEF796
:10D47000D0FC06464635012E00D0C83501F068FFC5
:10D4800001E0F4F7CCF890480088A842F9D3012EC7
:10D490000CD1FEF7C7FD4DF8240046355DF8240099
:10D4A000012800D0C83501F053FF01E04DF8246099
:10D4B000641C01E0F4F7B3F883480088A842F9D36C
:10D4C0008248807931280BD1FEF725FF4DF82400E2
:10D4D00046355DF82400012800D0C83501F038FF3A
:10D4E000641C01E0F4F79BF877480088A842F9D360
:10D4F0007648007A31280BD1FFF7E7F84DF8240081
:10D5000046355DF82400012800D0C83501F020FF21
:10D51000641C01E0F4F783F86B480088A842F9D353
:10D520006A48807A31280BD1FFF7B8F94DF824000A
:10D5300046355DF82400012800D0C83501F008FF09
:10D54000641C01E0F4F76BF85F480088A842F9D347
:10D550005E48007B31280BD1FFF7DBFA4DF8240041
:10D5600046355DF82400012800D0C83501F0F0FEF2
:10D57000641C01E0F4F753F853480088A842F9D33B
:10D580005248807B31280BD1FFF795FB4DF82400E2
:10D5900046355DF82400012800D0C83501F0D8FEDA
:10D5A000641C01E0F4F73BF847480088A842F9D32F
:10D5B0004648007C31280BD1FFF75EFD4DF8240072
:10D5C00046355DF82400012800D0C83501F0C0FEC2
:10D5D000641C01E0F4F723F83B480088A842F9D323
:10D5E0003A48807C31280BD1FFF76BF84DF82400C6
:10D5F00046355DF82400012800D0C83501F0A8FEAA
:10D60000641C01E0F4F70BF82F480088A842F9D316
:10D610002E48007D31280BD1FFF7FFFD4DF8240087
:10D6200046355DF82400012800D0C83501F090FE91
:10D63000641C27A001F0C4FA002409E0F3F7EFFF0F
:10D6400025A001F0BDFA1DF8240001F08FFB641C39
:10D65000092CF3D321A001F0B3FA00201849088067
:10D66000184908700AB070BD70B58AB0012014491D
:10D670000880144908700021084604F03BFA002590
:10D68000002011490880002403E000204DF8240008
:10D69000641C0A2CF9D3002401F05AFE0B49201D0A
:10D6A000085C31282AD1FEF728FC0646463517E0EB
:10D6B000F812002038000020160000200408002086
:10D6C00002000020510000201000002074140020EF
:10D6D0002A393131000000005F0000000D00000019
:10D6E00001F036FE012E07D1FEF789FD4DF824002A
:10D6F000463501F02DFE01E04DF82460641C052044
:10D7000002F0E8FAF3F78BFF4D488079312806D113
:10D71000FEF7E2FE4DF82400463501F019FE641CC8
:10D72000052002F0D7FAF3F77AFF4548007A31284E
:10D7300006D1FFF73DF84DF82400463501F008FE0C
:10D74000641C052002F0C6FAF3F769FF3C48807AB2
:10D75000312805D1FFF743F94DF8240001F0F8FD19
:10D76000641C052002F0B6FAF3F759FF3448007B39
:10D77000312805D1FFF729FA4DF8240001F0E8FD22
:10D78000641C052002F0A6FAF3F749FF2C48807BC1
:10D79000312805D1FFF782FB4DF8240001F0D8FDB8
:10D7A000641C052002F096FAF3F739FF2448007C48
:10D7B000312805D1FFF7BCFC4DF8240001F0C8FD6D
:10D7C000641C052002F086FAF3F729FF1C48807CD0
:10D7D000312806D1FEF777FF4DF82400463501F0D9
:10D7E000B7FD641C052002F075FAF3F718FF144822
:10D7F000007D312805D1FFF79AFD4DF8240001F096
:10D80000A7FD641C0FA001F0DBF900240AE0F3F788
:10D8100006FFAFF23C1001F0D3F91DF8240001F02F
:10D82000A5FA641C092CF2D3AFF2501001F0C8F92C
:10D83000002006490880064908700AB070BD000043
:10D84000741400202A393132000000000200002048
:10D85000510000205B484088401CB0F5007F01D299
:10D86000002070470120FCE756484188042913DB5B
:10D87000081F544A121D105C4F280DD1C81E105CA1
:10D880004B2809D1881E105C0D2805D1481E105C5C
:10D890000A2801D10120704707291FDBC81F494A08
:10D8A000121D105C452819D1881F105C522815D113
:10D8B000481F105C522811D1081F105C4F280DD151
:10D8C000C81E105C522809D1881E105C0D2805D195
:10D8D000481E105C0A2801D10120DCE70020DAE7AD
:10D8E00038480078704710B5F3F799FE3648FDF7D1
:10D8F000C8FD00203349488001200870F3F78FFEEF
:10D9000032A001F05DF93048FDF7BBFD00202D4944
:10D910000870F3F784FE10BD70B504460020294955
:10D920004880012008702AA001F04AF9207828B127
:10D9300020780D2802D0204601F042F925A001F000
:10D940003FF900251DE04FF47A70FDF79AFDFFF7CF
:10D9500081FF50B1F3F763FE44F62060FDF791FDBF
:10D96000002018490870012070BDFFF77DFF00B14D
:10D9700008E0322D03D1002012490870F4E7681C3A
:10D9800085B2E0E700BF00200E4908700120EBE7F8
:10D9900010B511A0FFF7C0FF10BD00210948428853
:10D9A000001D8154704710B50446FFF753FF38B986
:10D9B000044841884088401C024A5080101D44544D
:10D9C00010BD000098710020A08601002F2F2F00AD
:10D9D00041542A000D00000041542A4144444D0D99
:10D9E0000000000070B5574C574D002057490860A3
:10D9F0000AE0F3F714FE14F8011BC1F1FF005349CC
:10DA00000968084451490860AC42F2D370BD10B5B2
:10DA10004D4800884E4908804B48001D00884D49FC
:10DA20000880FFF7DFFF10BD48480068704738B531
:10DA3000F3F766F84849087000208DF803002520A8
:10DA40008DF8000068462EF002F927208DF80000BE
:10DA500068462EF0FCF834208DF8000068462EF061
:10DA6000F6F826208DF8000068462EF0F0F84720E2
:10DA70008DF8000068462EF0EAF82E208DF80000A0
:10DA800068462EF0E4F81B208DF8000068462EF062
:10DA9000DEF832208DF8000068462EF0D8F80E200F
:10DAA0008DF8000068462EF0D2F80C208DF80000AA
:10DAB00068462EF0CCF840208DF8000068462EF025
:10DAC000C6F842208DF8000068462EF0C0F83620D7
:10DAD0008DF8000068462EF0BAF837208DF8000067
:10DAE00068462EF0B4F818208DF8000068462EF035
:10DAF000AEF828208DF8000068462EF0A8F8122015
:10DB00008DF8000068462EF0A2F82C208DF8000059
:10DB100068462EF09CF831208DF8000068462EF003
:10DB200096F84FF440214FF000602EF0C2F80548FF
:10DB3000446825460146086880F3088800BFA84766
:10DB400038BD000000000C0800FF0F089C010020F9
:10DB5000240000202600002000FF01201CB5012128
:10DB600088032DF071FE0D21022032F00DF9684678
:10DB700032F0C3F84FF40050009000208DF80400FC
:10DB80000C208DF8050001208DF80600684632F063
:10DB90006DF81CBD0146FE4850F831007047014643
:10DBA000FB4800EBC100808870477CB50121084626
:10DBB0002DF006FE012102202DF002FE012104209D
:10DBC0002DF0FEFD012108202DF0FAFD012110208D
:10DBD0002DF0F6FD012120202DF0F2FD0121402045
:10DBE0002DF0EEFD01214FF0C0602DF01CFE012054
:10DBF0008DF8040002208DF8050000208DF8060045
:10DC000001208DF8070000240BE0E24800EBC4007F
:10DC100080880090DF4951F8340069462DF094F96E
:10DC2000641C192CF1D31020FFF7B9FF00900020DD
:10DC30008DF8040002208DF8050000208DF8060004
:10DC40008DF807001020FFF7A5FF054669462DF067
:10DC50007BF901208DF8040002208DF805000020DA
:10DC60008DF806008DF807000120FFF798FF00905F
:10DC70000120FFF78FFF054669462DF065F9022068
:10DC8000FFF78DFF00900220FFF784FF05466946ED
:10DC90002DF05AF90320FFF782FF00900320FFF7D1
:10DCA00079FF054669462DF04FF90420FFF777FF0D
:10DCB00000900420FFF76EFF054669462DF044F9F9
:10DCC00002208DF804008DF8050000208DF8060074
:10DCD0008DF807000520FFF762FF00900520FFF791
:10DCE00059FF054669462DF02FF90620FFF757FF2B
:10DCF00000900620FFF74EFF054669462DF024F9F7
:10DD00000720FFF74CFF00900720FFF743FF054671
:10DD100069462DF019F903208DF8040000208DF8D4
:10DD200007003720FFF73BFF00903720FFF732FF57
:10DD3000054669462DF008F93820FFF730FF0090BE
:10DD40003820FFF727FF054669462DF0FDF83920FA
:10DD5000FFF725FF00903920FFF71CFF05466946B5
:10DD60002DF0F2F83A20FFF71AFF00903A20FFF763
:10DD700011FF054669462DF0E7F83B20FFF70FFF3E
:10DD800000903B20FFF706FF054669462DF0DCF8C2
:10DD900001208DF8040002208DF8050000208DF888
:10DDA00006008DF807004720FFF7F9FE0090472096
:10DDB000FFF7F0FE054669462DF0C6F84820FFF74C
:10DDC000EEFE00904820FFF7E5FE054669462DF07F
:10DDD000BBF801208DF8040002208DF8050000201A
:10DDE0008DF806008DF807004220FFF7D8FE00905E
:10DDF0004220FFF7CFFE054669462DF0A5F8022028
:10DE00008DF804005020FFF7CAFE00905020FFF765
:10DE1000C1FE054669462DF097F800208DF80400F4
:10DE20000820FFF7BCFE00900820FFF7B3FE054670
:10DE300069462DF089F801208DF807003F20FFF793
:10DE4000AEFE00903F20FFF7A5FE054669462DF087
:10DE50007BF84120FFF7A3FE00904120FFF79AFED8
:10DE6000054669462DF070F802208DF80500002067
:10DE70008DF806008DF807008DF804004020FFF7AC
:10DE80008EFE00904020FFF785FE054669462DF086
:10DE90005BF83E20FFF783FE00903E20FFF77AFEFE
:10DEA000054669462DF050F802208DF804003C200C
:10DEB000FFF775FE00903C20FFF76CFE05466946B3
:10DEC0002DF042F801208DF8040002208DF80500A5
:10DED00000208DF806008DF807004C20FFF75FFE4C
:10DEE00000904C20FFF756FE054669462DF02CF8B1
:10DEF0004D20FFF754FE00904D20FFF74BFE0546E6
:10DF000069462DF021F800208DF804000920FFF764
:10DF100046FE00900920FFF73DFE054669462DF0BC
:10DF200013F80A20FFF73BFE00900A20FFF732FEAD
:10DF3000054669462DF008F80B20FFF730FE0090EB
:10DF40000B20FFF727FE054669462CF0FDFF012058
:10DF50008DF8040002208DF8050000208DF80600E1
:10DF60008DF80700FFF71BFE00900020FFF712FE60
:10DF7000054669462CF0E8FF01208DF804000220D8
:10DF80008DF8050000208DF80600012004E0000057
:10DF900054160408DC1804088DF807003020FFF739
:10DFA000FEFD00903020FFF7F5FD054669462CF098
:10DFB000CBFF2D20FFF7F3FD00902D20FFF7EAFDAA
:10DFC000054669462CF0C0FF2E20FFF7E8FD0090C3
:10DFD0002E20FFF7DFFD054669462CF0B5FF2F2008
:10DFE000FFF7DDFD00902F20FFF7D4FD05466946C1
:10DFF0002CF0AAFF02208DF804008DF80500002007
:10E000008DF8060001208DF807003320FFF7C7FDCB
:10E0100000903320FFF7BEFD054669462CF094FFC3
:10E020003420FFF7BCFD00903420FFF7B3FD054618
:10E0300069462CF089FF3320FFF7B1FD012801D19B
:10E04000002071E03320FFF7AAFD022801D1012052
:10E050006AE03320FFF7A3FD042801D1022063E02A
:10E060003320FFF79CFD082801D103205CE033201A
:10E07000FFF795FD102801D1042055E03320FFF76C
:10E080008EFD202801D105204EE03320FFF787FDCB
:10E09000402801D1062047E03320FFF780FD80288B
:10E0A00001D1072040E03320FFF779FDB0F5807FF4
:10E0B00001D1082038E03320FFF771FDB0F5007F73
:10E0C00001D1092030E03320FFF769FDB0F5806F02
:10E0D00001D10A2028E03320FFF761FDB0F5006F81
:10E0E00001D10B2020E03320FFF759FDB0F5805F10
:10E0F00001D10C2018E03320FFF751FDB0F5005F8F
:10E1000001D10D2010E03320FFF749FDB0F5804F1D
:10E1100001D10E2008E03320FFF741FDB0F5004F9C
:10E1200001D10F2000E0FF2005463320FFF732FD2C
:10E130000646092229462CF08AFF3420FFF72FFDDE
:10E14000012801D1002071E03420FFF728FD0228CA
:10E1500001D101206AE03420FFF721FD042801D11C
:10E16000022063E03420FFF71AFD082801D10320C4
:10E170005CE03420FFF713FD102801D1042055E0A6
:10E180003420FFF70CFD202801D105204EE034207B
:10E19000FFF705FD402801D1062047E03420FFF7B6
:10E1A000FEFC802801D1072040E03420FFF7F7FC77
:10E1B000B0F5807F01D1082038E03420FFF7EFFC74
:10E1C000B0F5007F01D1092030E03420FFF7E7FCF3
:10E1D000B0F5806F01D10A2028E03420FFF7DFFC82
:10E1E000B0F5006F01D10B2020E03420FFF7D7FC01
:10E1F000B0F5805F01D10C2018E03420FFF7CFFC90
:10E20000B0F5005F01D10D2010E03420FFF7C7FC0E
:10E21000B0F5804F01D10E2008E03420FFF7BFFC9D
:10E22000B0F5004F01D10F2000E0FF20054634205B
:10E23000FFF7B0FC0646092229462CF008FF002013
:10E240008DF8040002208DF8050000208DF80600EE
:10E2500001208DF807003520FFF7A1FC0090352044
:10E26000FFF798FC054669462CF06EFE3620FFF756
:10E2700096FC00903620FFF78DFC054669462CF091
:10E2800063FE3120FFF78BFC00903120FFF782FC0A
:10E29000054669462CF058FE3220FFF780FC0090BE
:10E2A0003220FFF777FC054669462CF04DFEFFF75C
:10E2B00055FC7CBD70477CB500208DF80400022021
:10E2C0008DF8050000208DF8060001208DF807006C
:10E2D0003120FFF764FC00903120FFF75BFC04461F
:10E2E00069462CF031FE3220FFF759FC00903220B5
:10E2F000FFF750FC044669462CF026FE02208DF8FC
:10E3000004008DF8050000208DF8060001208DF82E
:10E3100007003520FFF743FC00903520FFF73AFC5B
:10E32000044669462CF010FE3620FFF738FC0090BA
:10E330003620FFF72FFC044669462CF005FE3520F9
:10E34000FFF72DFC012801D1002071E03520FFF7F7
:10E3500026FC022801D101206AE03520FFF71FFCCE
:10E36000042801D1022063E03520FFF718FC0828BB
:10E3700001D103205CE03520FFF711FC102801D10A
:10E38000042055E03520FFF70AFC202801D10520A4
:10E390004EE03520FFF703FC402801D1062047E07E
:10E3A0003520FFF7FCFB802801D1072040E0352015
:10E3B000FFF7F5FBB0F5807F01D1082038E035206C
:10E3C000FFF7EDFBB0F5007F01D1092030E03520EB
:10E3D000FFF7E5FBB0F5806F01D10A2028E035207A
:10E3E000FFF7DDFBB0F5006F01D10B2020E03520F9
:10E3F000FFF7D5FBB0F5805F01D10C2018E0352088
:10E40000FFF7CDFBB0F5005F01D10D2010E0352006
:10E41000FFF7C5FBB0F5804F01D10E2008E0352095
:10E42000FFF7BDFBB0F5004F01D10F2000E0FF204A
:10E4300004463520FFF7AEFB0546092221462CF0A5
:10E4400006FE3620FFF7ABFB012801D1002071E06A
:10E450003620FFF7A4FB022801D101206AE0362014
:10E46000FFF79DFB042801D1022063E03620FFF76F
:10E4700096FB082801D103205CE03620FFF78FFBD4
:10E48000102801D1042055E03620FFF788FB202812
:10E4900001D105204EE03620FFF781FB402801D155
:10E4A000062047E03620FFF77AFB802801D10720BD
:10E4B00040E03620FFF773FBB0F5807F01D10820E4
:10E4C00038E03620FFF76BFBB0F5007F01D1092063
:10E4D00030E03620FFF763FBB0F5806F01D10A20F2
:10E4E00028E03620FFF75BFBB0F5006F01D10B2071
:10E4F00020E03620FFF753FBB0F5805F01D10C2000
:10E5000018E03620FFF74BFBB0F5005F01D10D207E
:10E5100010E03620FFF743FBB0F5804F01D10E200D
:10E5200008E03620FFF73BFBB0F5004F01D10F208C
:10E5300000E0FF2004463620FFF72CFB05460922A9
:10E5400021462CF084FD7CBD7CB500208DF80400B4
:10E5500002208DF8050000208DF8060001208DF8BE
:10E5600007003520FFF71BFB00903520FFF712FB5B
:10E57000044669462CF0E8FC3620FFF710FB0090BB
:10E580003620FFF707FB044669462CF0DDFC02202D
:10E590008DF804008DF8050000208DF8060001209C
:10E5A0008DF807003120FFF7FAFA00903120FFF7CD
:10E5B000F1FA044669462CF0C7FC3220FFF7EFFA67
:10E5C00000903220FFF7E6FA044669462CF0BCFCC6
:10E5D0003120FFF7E4FA012801D1002071E0312059
:10E5E000FFF7DDFA022801D101206AE03120FFF7B0
:10E5F000D6FA042801D1022063E03120FFF7CFFAD8
:10E60000082801D103205CE03120FFF7C8FA102868
:10E6100001D1042055E03120FFF7C1FA202801D1B3
:10E6200005204EE03120FFF7BAFA402801D106203C
:10E6300047E03120FFF7B3FA802801D1072040E0FE
:10E640003120FFF7ACFAB0F5807F01D1082038E027
:10E650003120FFF7A4FAB0F5007F01D1092030E0A6
:10E660003120FFF79CFAB0F5806F01D10A2028E035
:10E670003120FFF794FAB0F5006F01D10B2020E0B4
:10E680003120FFF78CFAB0F5805F01D10C2018E043
:10E690003120FFF784FAB0F5005F01D10D2010E0C2
:10E6A0003120FFF77CFAB0F5804F01D10E2008E051
:10E6B0003120FFF774FAB0F5004F01D10F2000E0D0
:10E6C000FF2004463120FFF765FA0546092221465E
:10E6D0002CF0BDFC3220FFF762FA012801D10020A6
:10E6E00071E03220FFF75BFA022801D101206AE0D5
:10E6F0003220FFF754FA042801D1022063E03220CF
:10E70000FFF74DFA082801D103205CE03220FFF723
:10E7100046FA102801D1042055E03220FFF73FFAD5
:10E72000202801D105204EE03220FFF738FA40289A
:10E7300001D1062047E03220FFF731FA802801D1CD
:10E74000072040E03220FFF72AFAB0F5807F01D1A0
:10E75000082038E03220FFF722FAB0F5007F01D11F
:10E76000092030E03220FFF71AFAB0F5806F01D1AE
:10E770000A2028E03220FFF712FAB0F5006F01D12D
:10E780000B2020E03220FFF70AFAB0F5805F01D1BC
:10E790000C2018E03220FFF702FAB0F5005F01D13B
:10E7A0000D2010E03220FFF7FAF9B0F5804F01D1CB
:10E7B0000E2008E03220FFF7F2F9B0F5004F01D14A
:10E7C0000F2000E0FF2004463220FFF7E3F9054662
:10E7D000092221462CF03BFC7CBD92B072B602208F
:10E7E0008DF8450000208DF8460001208DF8470087
:10E7F0008DF844000F20FFF7D2F910900F20FFF79B
:10E80000C9F9044610A92CF09FFB00208DF84400A4
:10E810000E20FFF7C4F910900E20FFF7BBF9044655
:10E8200010A92CF091FB00208DF844000D20FFF77B
:10E83000B6F910900D20FFF7ADF9044610A92CF0A1
:10E8400083FB01208DF844000C20FFF7A8F91090FD
:10E850000C20FFF79FF9044610A92CF075FB00214E
:10E8600053482CF0FFFC02208DF8450000208DF865
:10E87000460001208DF847008DF844001420FFF772
:10E880008EF910901420FFF785F9044610A92CF09A
:10E890005BFB00208DF844001320FFF780F91090F7
:10E8A0001320FFF777F9044610A92CF04DFB002048
:10E8B0008DF844001220FFF772F910901220FFF734
:10E8C00069F9044610A92CF03FFB01208DF84400A3
:10E8D0001120FFF764F910901120FFF75BF904464F
:10E8E00010A92CF031FB002132482CF0BBFC32483F
:10E8F000416A006ACDE90E012F48C1688068CDE900
:10E900000C012D488038416F006FCDE90A012A497A
:10E910008039D1E91A01CDE9080127498039D1E9C7
:10E920001E01CDE906012448C1698069CDE90401D1
:10E9300021498039D1E91801CDE902011E48416918
:10E940000069CDE9000131E0F2F769FEBDF82C1055
:10E950000A982CF04AFB0446BDF83C1022460E985B
:10E960002CF061FBBDF8241008982CF03EFB044607
:10E97000BDF8341022460C982CF055FBBDF814104D
:10E9800004982CF032FB0446BDF81C102246069871
:10E990002CF049FBBDF8041000982CF026FB04462F
:10E9A000BDF80C10224602982CF03DFBCCE700008D
:10E9B0000010014000480040D416040800B58BB098
:10E9C00000207C4908700A2048700120087100204E
:10E9D00088710B217748C17101218172002075492E
:10E9E00008730E217348417301210174022072499A
:10E9F0000880098801EB41016E4A02F811000121EB
:10EA0000C0012CF021FF07A831F071FA07A831F0FE
:10EA100038FA01A831F071FA00208DF80900019050
:10EA200001A9664831F03EFA0121644831F06FFADD
:10EA3000012240F20521614831F07FFA0BB000BDA0
:10EA400010B55D48008800EB40005A4911F81000ED
:10EA5000022830D100205849098801EB4101554A6C
:10EA600002F8110054480088401C032190FBF1F289
:10EA700001FB1200504908800846008800EB400066
:10EA80004C4911F81000B0B901204B49098801EB3D
:10EA90004101484A02F811004748008800EB400055
:10EAA00002EB4000417800230122444831F0ADFAE6
:10EAB000424831F052FA10BD10B572B63D48448854
:10EAC00062B6204600F06EF8243080B210BD10B55A
:10EAD00072B63848048962B6204600F063F810BD6B
:10EAE00010B572B63348C48962B6204600F05AF8B1
:10EAF00010BD10B5FFF7E0FF044640F24C408442E1
:10EB000001DA012010BDB4F5C86F05DD40F6340010
:10EB1000844201DA0120F5E70020F3E710B5FFF7A2
:10EB2000CBFFB0F5C86F01DD012010BD0020FCE770
:10EB300070B52149098801EB41011E4A02EB4101F0
:10EB4000097981B11C49098801EB410102EB4101BE
:10EB500048800021184A128802EB4202154B03EB51
:10EB60004202117115E0144C248804EB4404114D49
:10EB700005EB4404648804EB44010346CC18A20866
:10EB80000D4D2D8805EB45050A4E06EB45056A80BF
:10EB900000BF0221084A128802EB4202054B03F82B
:10EBA000121070BD01464FF4507001FB00F2C2F329
:10EBB0008F2070479C730020A0010020002001409E
:10EBC00010B5044603E014F8010BF2F771FC20784D
:10EBD0000028F8D110BD2DE9F04186B0064642F27A
:10EBE000107096FBF0F0019040F2712101984843BB
:10EBF000A6EB00144FF47A70B4FBF0F00290029888
:10EC000000EB4001C1EBC010A4EBC0046420B4FBD6
:10EC1000F0F00390039800EBC00101EB0010A4EBAF
:10EC200080040A20B4FBF0F00490049800EB80000C
:10EC3000A4EB400005904FF00008012513E05DF8BB
:10EC4000250018B9059818B9052D01D14FF0010814
:10EC5000B8F1010F06D11DF825003030C7B2384693
:10EC6000F2F726FC6D1C062DE9DB06B0BDE8F0814D
:10EC70002DE9F0418CB00646FA48B6FBF0F0029060
:10EC8000F94902984843A6EB4024F848B4FBF0F059
:10EC90000390F74903984843A4EB0024F548B4FBDC
:10ECA000F0F00490F44904984843A4EBC014F348EE
:10ECB000B4FBF0F0059043F6095105984843A4EBE6
:10ECC0008014EF48B4FBF0F0069040F6354106980A
:10ECD0004843A4EB401442F21070B4FBF0F00790EC
:10ECE00040F2712107984843A4EB00144FF47A7066
:10ECF000B4FBF0F00890089800EB4001C1EBC010A5
:10ED0000A4EBC0046420B4FBF0F00990099800EB78
:10ED1000C00101EB0010A4EB80040A20B4FBF0F06A
:10ED20000A900A9800EB8000A4EB40000B904FF093
:10ED30000008012515E001A850F8250018B90B9826
:10ED400018B90A2D01D14FF00108B8F1010F07D110
:10ED500001A810F825003030C7B23846F2F7A8FBFA
:10ED60006D1C0B2DE7DB0CB0BDE8F08170B50546DE
:10ED70002C09092C03DC04F13000C4B202E004F1D8
:10ED80003700C4B22046F2F793FB05F00F04092CBC
:10ED900003DC04F13000C4B202E004F13700C4B275
:10EDA0002046F2F785FB70BD70B505462C0B092C8B
:10EDB00003DC04F13000C4B202E004F13700C4B255
:10EDC0002046F2F775FBC5F30324092C03DC04F19C
:10EDD0003000C4B202E004F13700C4B22046F2F7BA
:10EDE00067FBC5F30314092C03DC04F13000C4B243
:10EDF00002E004F13700C4B22046F2F759FB05F0F7
:10EE00000F04092C03DC04F13000C4B202E004F169
:10EE10003700C4B22046F2F74BFB70BD70B5054613
:10EE20002C0F092C03DC04F13000C4B202E004F121
:10EE30003700C4B22046F2F73BFBC5F30364092C4C
:10EE400003DC04F13000C4B202E004F13700C4B2C4
:10EE50002046F2F72DFBC5F30354092C03DC04F123
:10EE60003000C4B202E004F13700C4B22046F2F729
:10EE70001FFBC5F30344092C03DC04F13000C4B2CA
:10EE800002E004F13700C4B22046F2F711FBC5F3EB
:10EE90000334092C03DC04F13000C4B202E004F1B5
:10EEA0003700C4B22046F2F703FBC5F30324092C54
:10EEB00003DC04F13000C4B202E004F13700C4B254
:10EEC0002046F2F7F5FAC5F30314092C03DC04F12C
:10EED0003000C4B202E004F13700C4B22046F2F7B9
:10EEE000E7FA05F00F04092C03DC04F13000C4B28A
:10EEF00002E004F13700C4B22046F2F7D9FA70BD3F
:10EF00000146302905DB392903DCA1F13000C0B20C
:10EF10007047612905DB662903DCA1F15700C0B207
:10EF2000F6E7412905DB462903DCA1F13700C0B231
:10EF3000EEE73020ECE72DE9F04105460E46174696
:10EF40002A20F2F7B5FA002414E0F2F768FB482F04
:10EF500001D0682F03D1285DFFF708FF02E0285D8C
:10EF6000FFF739FE701EA04202DD2020F2F7A0FA62
:10EF7000601C84B2B442E8DBBDE8F0812DE9FC41BD
:10EF800004460020019001A9204602F037FA054608
:10EF9000BDF804000444BDF80400002861D0022D2F
:10EFA00040D003DC3DB1012D6FD10BE00A2D15D00F
:10EFB0000B2D7ED12AE003F075F832A0FFF700FE9A
:10EFC000BDE8FC8114F8011B39B1204603F080F83C
:10EFD00018B12CA0FFF7F4FDF2E76BE014F8011B69
:10EFE00099B101A9204602F009FA0646BDF80400CD
:10EFF0000444621C14461146B0B203F08DF818B1F7
:10F0000020A0FFF7DDFDDBE700BF53E014F8011B94
:10F0100039B1204603F0A0F818B11AA0FFF7D0FDCF
:10F02000CEE747E014F8011B71B3012601A9204681
:10F0300002F0E4F90746BDF80400044427B1012FAB
:10F0400008D0022F28D121E000208DF800008DF893
:10F05000010023E001208DF8000000208DF8010060
:10F060001CE028E000CA9A3B65CD1D0000E1F505D3
:10F07000E1F50500809698002D31010040420F0017
:10F08000A08601002A310D0012E012E001208DF867
:10F0900000008DF8010001E0002600BF00BF36B17E
:10F0A0000748008818B1684603F075F888E700BF84
:10F0B00000E000BF00BF03A0FFF782FD00BF7FE7B5
:10F0C000020000202A300D0010B504460121452021
:10F0D00002F010FD0121462002F00CFD012000F09D
:10F0E000F9FD0021462002F005FD152C7CD2DFE859
:10F0F00004F0AF0B1117AFAF1D23292F353B41474C
:10F100004D53596A7C8D9E00002201210420F2F7A4
:10F110009FFEA3E0002202210420F2F799FE9DE069
:10F12000002203210420F2F793FE97E0002206213B
:10F130000420F2F78DFE91E0002207210420F2F76F
:10F1400087FE8BE0002208210420F2F781FE85E093
:10F15000002209210420F2F77BFE7FE000220A2131
:10F160000420F2F775FE79E000220B210420F2F76B
:10F170006FFE73E000220C210420F2F769FE6DE0BF
:10F1800000220D210420F2F763FE67E000220E2129
:10F190000420F2F75DFE61E000220F210420F2F767
:10F1A00057FE5BE00F220D210420F2F751FE0121F2
:10F1B000452002F09FFC012000F08CFD002145203D
:10F1C00002F098FC4AE00F220C210420F2F740FEE6
:10F1D0000121452002F08EFC012000F07BFD002182
:10F1E000452002F087FC39E032E00F220B21042099
:10F1F000F2F72EFE0121452002F07CFC012000F0F8
:10F2000069FD0021452002F075FC27E00F2207214F
:10F210000420F2F71DFE0121452002F06BFC0120C5
:10F2200000F058FD0021452002F064FC16E00222A7
:10F2300003210420F2F70CFE0121452002F05AFCC4
:10F24000012000F047FD0021452002F053FC05E0BD
:10F25000002207210420F2F7FBFD00BF00BF64205D
:10F2600000F038FD10BD70B505460C460121452063
:10F2700002F040FC0121462002F03CFC012000F09D
:10F2800029FD0121452002F035FC012000F022FD7E
:10F290000021452002F02EFC0121462002F02AFC2C
:10F2A000012000F017FD0021462002F023FC1CB9CC
:10F2B0000121452002F01EFC224629460420F2F7D7
:10F2C000C7FD642000F006FD70BD10B50020F4F706
:10F2D0002CF80020F4F72EF8002208214FF4964075
:10F2E000F3F77CFE0121462002F004FC01214520B9
:10F2F00002F000FC012000F0EDFC0021452002F0AE
:10F30000F9FB0D220C210420F2F7A2FD0A2000F0E7
:10F31000E1FC0020E3490860E3490880FF20E3495D
:10F320000880E3490880E349088000BFF2F777F9D5
:10F33000DD480088012803DADA4800680528F5D995
:10F34000D8480068052801D3002010BD0120FCE743
:10F3500010B5002211461046F2F77AFD10BD70B5C7
:10F3600004460D460020F3F7E0FF0020F3F7E2FF2C
:10F37000002208214FF49640F3F730FE0121462089
:10F3800002F0B8FB0121452002F0B4FB012000F09F
:10F39000A1FC0021452002F0ADFB2A4621460420B5
:10F3A000F2F756FD0A2000F095FC0020BD490860E8
:10F3B000BD490880FF20BD490880BD490880BD497E
:10F3C000088000BFF2F72BF9B7480088012803DA5C
:10F3D000B44800680528F5D9B2480068052803D369
:10F3E000FFF7B6FF002070BDFFF7B2FF0120FAE77C
:10F3F00070B5054601240020F3F797FF0020F3F7CE
:10F4000099FF002208214FF49640F3F7E7FD012110
:10F41000462002F06FFB0121452002F06BFB01202A
:10F4200000F058FC0021452002F064FB092208216D
:10F430000420F2F70DFD022000F04CFC0020994959
:10F44000086099490880FF209849088098490880F9
:10F450009849088000BFF2F7E2F893480088012835
:10F4600003DA904800680328F5D98E48006803281D
:10F4700001D3002402E0FFF76BFF01241CBB0E2226
:10F480000D210420F2F7E4FC022000F023FC002010
:10F490008449086084490880FF20844908808449A1
:10F4A00008808449088000BFF2F7B9F87E480088D8
:10F4B000012803DA7B4800680328F5D979480068F9
:10F4C000032801D3002402E0FFF742FF02242CBBF3
:10F4D000032D27DB082203210420F2F7B9FC0220C8
:10F4E00000F0F8FB00206F4908606F490880FF209A
:10F4F0006E4908806E4908806E49088000BFF2F7A7
:10F500008EF869480088012803DA664800680328F5
:10F51000F5D964480068032801D3002402E0FFF70E
:10F5200017FF03242CBB042D27DB08220121042014
:10F53000F2F78EFC022000F0CDFB00205949086054
:10F5400059490880FF20594908805949088059497C
:10F55000088000BFF2F763F853480088012803DAF7
:10F56000504800680328F5D94E480068032801D3A5
:10F57000002402E0FFF7ECFE0424204670BD10B525
:10F5800001204D49088000204C49088000220821B4
:10F590004FF49640F3F722FD49A0FFF711FB00223C
:10F5A00011460420F2F754FC0020F3F7C3FE0121BA
:10F5B000452002F09FFA012000F08CFB002145203D
:10F5C00002F098FA0121462002F094FA012436E074
:10F5D00022B221B20420F2F73BFC052000F07AFBB6
:10F5E00000203B4908803049088055202F49088079
:10F5F0002F4908802F49088000BFF2F710F82A48E9
:10F600000088012803DA324800880228F5DD3048F6
:10F610000088022806DB0120284908802DA0FFF77A
:10F62000CFFA02E02DA0FFF7CBFAA0B2FFF7D3FA92
:10F630000D20F1F73DFF032C00D1A41C641C0F2CFE
:10F64000C6D91E48008810B926A0FFF7B9FA0020D5
:10F650001949088010BD10B50620F3F76BFE012094
:10F6600000F038FB022200210620F2F7F1FB032014
:10F6700000F030FB0021202002F03CFA012000F0D5
:10F6800029FB0121202002F035FA032000F022FBA3
:10F690000E2206210120F2F7DBFB052000F01AFB09
:10F6A00010BD000038000020160000200444004077
:10F6B00004140140044C004002000020120000200D
:10F6C0000D546573742072656C61793A0D00000009
:10F6D0001000002046656C3A20000000204F4B3A95
:10F6E000200000002A4F4B0D0000000070B5FE48BE
:10F6F000048850250020FD49088000BFF1F78FFFE6
:10F70000F9480088001B80B2502803DD0120F84929
:10F71000088003E0F54800880128EFDB00BF70BDDA
:10F720002DE9F05F0646894600244FF004084FF0AB
:10F73000200A002500BFF1F772FFEE4A08F101012F
:10F74000505CFFF7DDFB8346EA4911F80800FFF73C
:10F75000D7FB0BEB0010C7B2484600F0BBFAE648F7
:10F760000780E6480780E64807802846691C0DB2F6
:10F77000E4490F540B2E08D1B8F1040F01D13C46D7
:10F7800010E084EA070004460CE0052E02D184EA6A
:10F7900007000446082E03D00A2E01D0FFF7A6FF6B
:10F7A000E01984B2D34908F1020011F800A0401C0E
:10F7B0000FFA80F8BAF1000FBDD10C2E76D2DFE837
:10F7C00006F006071628476676C7898AA9B6CEE0EE
:10F7D000484600F07FFAE0B2C7490880C749088070
:10F7E000C7490880C7494C55FFF780FFBFE0E4B226
:10F7F000484600F06FFAC4F58070BF490880BF49E1
:10F800000880BF4908806042BE494855FFF76EFF37
:10F81000ADE0484600F05EFA2012B7490880B749CB
:10F820000880B749088022122846691C0DB2B549E4
:10F830000A54484600F04EFAE0B2AF490880AF499A
:10F840000880AF490880AF494C55FFF74FFF8EE065
:10F85000484600F03FFAE0B2A7490880A74908806F
:10F86000A74908802846691C0DB2A6490C54484691
:10F8700000F030FA2012A0490880A0490880A04971
:10F88000088020129F494855FFF730FF6FE0484637
:10F8900000F020FAE0B29849088098490880984919
:10F8A000088098494C55FFF721FF60E050E0E4B232
:10F8B000484600F00FFAC4F1FF008F4908808F49D5
:10F8C00008808F490880C4F1FF008E494855FFF732
:10F8D0000DFF4CE04BE087494879FFF711FB834669
:10F8E00084490879FFF70CFB0BEB0010201A84B257
:10F8F000E4B2484600F0EEF9C4F580707E49088015
:10F900007E4908807E49088060427E494855FFF75D
:10F91000EDFE2CE0484600F0DDF9E0B276490880C3
:10F92000764908807649088076494C551FE048465C
:10F9300000F0D0F984F0FF006F4908806F4908801B
:10F940006F490880E0436F494855FFF7CFFE0EE04E
:10F95000484600F0BFF9E0B267490880674908806F
:10F960006749088067494C55FFF7C0FE00BF00BFDC
:10F9700065490D806348007800F08000802804D13C
:10F98000604880786149088002E000205F49088073
:10F99000BDE8F09F2DE9FF4F81B0824699460E9E4B
:10F9A0002020009000240025DDF8088000BFF1F73A
:10F9B00036FE08F101011AF80100FFF7A1FA8346AB
:10F9C0001AF80800FFF79CFA0BEB0017B0B200F032
:10F9D00081F94948078049480780494807802846F7
:10F9E0006D1C48490F54B9F1050F02D184EA070094
:10F9F0000446B9F1080F01D0FFF778FE3C4408F146
:10FA000002001AF80000009008F1030803988045EE
:10FA100005D2B8F5787F02D200980028C7D1B9F195
:10FA20000A0F75D2DFE809F005061527477D8CBE61
:10FA30009FA0C6E0B0B200F04DF9E0B22E490880B8
:10FA40002E4908802E4908802E494C55FFF74EFE5E
:10FA5000B7E0E4B2B0B200F03DF9C4F580702649D9
:10FA60000880264908802649088060422549485573
:10FA7000FFF73CFEA5E0B0B200F02CF9C4F30F2074
:10FA80001D4908801D4908801D490880C4F30722CC
:10FA900028466D1C1B490A54B0B200F01BF9E0B2B5
:10FAA00015490880154908801549088015494C55A5
:10FAB000FFF71CFE85E0B0B200F00CF9E0B20E4991
:10FAC00008800E4908800E49088028466D1C0D49A3
:10FAD0000C54B0B200F0FEF8C4F30F2006490880C1
:10FAE00006490880064914E0100000201600002096
:10FAF000120000207414002004440040041401404B
:10FB0000044C004048130020360000203200002042
:10FB100048E00880C4F307205F494855FFF7E6FD39
:10FB20004FE0B0B200F0D6F8E0B25C4908805C4922
:10FB300008805C49088058494C55FFF7D7FD40E0E4
:10FB4000E4B2B0B200F0C6F8C4F1FF005349088037
:10FB50005349088053490880C4F1FF004E49485575
:10FB6000FFF7C4FD2DE02CE04F494879FFF7C8F9B5
:10FB700083464D490879FFF7C3F90BEB0010241AAF
:10FB8000E4B2B0B200F0A6F8C4F580704349088032
:10FB9000434908804349088060423F494855FFF780
:10FBA000A5FD0EE0B0B200F095F8A0B23B49088088
:10FBB0003B4908803B49088037494C55FFF796FD83
:10FBC00000BF00BF39490D803348007800F0800045
:10FBD000802804D1304880783549088002E0002030
:10FBE0003349088005B0BDE8F08F70B505460E4674
:10FBF000002400BFF1F713FD15B1A8B200F06AF8B8
:10FC00002C4810F81400254908802549088025490A
:10FC10000880284810F814001F490855012E01D10A
:10FC2000FFF764FD601C04B2224830F814004FF660
:10FC3000FF71884201D0282CDCDB1C490C8016485F
:10FC4000007800F08000802804D11348807818499B
:10FC5000088002E000201649088070BD70B5044697
:10FC60000D46002600BFF1F7DAFC14B1A0B200F097
:10FC700031F83046761C0849085C08490880084974
:10FC8000088008490880012D01D1FFF72FFD0748A2
:10FC900000888642E7DD70BD481300200444004020
:10FCA00004140140044C004074140020360000206D
:10FCB00032000020F812002070B504461348058871
:10FCC00000BFF1F7ACFC11480088401B80B2A04295
:10FCD000F7DB70BD70B504460D48056800BFF1F74D
:10FCE0009EFC0B480068411B601C8142F7D370BD2D
:10FCF00070B50446162004FB00F500BFF1F78FFC39
:10FD00002800A5F10105F9D170BD00001000002008
:10FD10003800002070B504460025002600E0641C71
:10FD200020782028FBD020785F28F8D002E0681CDB
:10FD300085B2641C2CB12078302802DB2078392869
:10FD4000F5DDFBF7A2FA06463046FEF791FF0D20DF
:10FD5000F1F7AEFB70BDF7484078313809280FD273
:10FD6000DFE800F005060708090A0B0C0D0007E0A4
:10FD700006E005E004E003E002E001E000E000BF8F
:10FD800000BF7047EB484078312804D0322803D0B8
:10FD9000332803D101E001E000E000BF00BF70475D
:10FDA00010B5E4484078302874D1E248807838288B
:10FDB00057D009DCA0F13000082830D2DFE800F08D
:10FDC0001530393A3B3C3F4843286ED006DC392891
:10FDD0004AD041284BD0422821D17EE0612847D02B
:10FDE00062287BD06328F7D182E0F3F796FF80B1D9
:10FDF000F3F753FF30B10120CF490870CFA0FEF7D1
:10FE0000DFFE0CE00020CC490870CDA0FEF7D8FE44
:10FE100005E00020C8490870C9A0FEF7D1FE68E0DF
:10FE2000F3F77BFF20B1F3F738FF08B1FBF766F873
:10FE30005FE05EE05DE05CE0FAF7A2FF59E0BD48FC
:10FE4000001D30F035FCC4B22046FBF73AF850E014
:10FE5000B848001D30F02CFCC4B22046FAF7F3FF7E
:10FE600047E0FAF79AFF44E0FAF777FF41E000BF76
:10FE7000FAF7F5FD0446012C18D1F3F721FF50B134
:10FE8000B0A0FEF79DFE0120FEF7A5FEAEA0FEF796
:10FE900097FE21E02FE0ABA0FEF792FE0420FEF7D4
:10FEA0009AFEA9A0FEF78CFE16E020E0022C0AD1F3
:10FEB000A4A0FEF785FE0220FEF78DFEA2A0FEF7AD
:10FEC0007FFE09E00AE09FA0FEF77AFE0020FEF721
:10FED00082FE9DA0FEF774FE0BE000BF9548001D5A
:10FEE00030F0E6FB84B22046F9F7BAFF01E000BF2C
:10FEF00000BF00BF10BD00BFFCE710B58D484078C3
:10FF00003138092872D2DFE800F0053D5B859FB7E4
:10FF1000CFE7F40087488078382829D009DCA0F1A1
:10FF2000300008282CD2DFE800F015181B1C1D201B
:10FF30002122432822D006DC39281AD0412819D0A2
:10FF400042281DD118E0612815D0622815D06328F9
:10FF500016D114E025F0DEFB12E025F0D4FF0FE00F
:10FF60000EE00DE026F0CCFB0AE009E008E007E037
:10FF700006E005E000BF03E000BF01E000BF00BFF6
:10FF800000BF10BD6B48807830380A2816D2DFE8F1
:10FF900000F005080B0C0F101112131426F0F5FCDD
:10FFA0000CE020F0F3FC09E008E026F0D3FE05E0C9
:10FFB00004E003E002E001E000E000BF00BFE0E792
:10FFC0005C48807836281DD008DCA0F13000062877
:10FFD0001ED2DFE800F0111213141516392814D0C0
:10FFE00005DC37280FD0382812D10DE0F9E0412880
:10FFF0000CD061280CD10AE00AE009E008E007E033
:020000040801F1
:1000000006E005E004E003E002E001E000BF00BF1D
:1000100000BFB6E74748807830380A2812D2DFE8B8
:1000200000F005060708090A0B0C0D0E0AE009E0AE
:1000300008E007E006E005E004E003E002E0FFF787
:100040009EFA00BF00BF9CE73A48807830380A2803
:1000500010D2DFE800F005060708090A0B0C0D0EA8
:1000600008E007E006E005E004E003E002E001E06C
:1000700000E000BF00BF84E72E48807830380A28AF
:1000800010D2DFE800F005060708090A0B0C0D0E78
:1000900008E007E006E005E004E003E002E001E03C
:1000A00000E000BF00BF6CE72248807830380A28A3
:1000B00010D2DFE800F005060708090A0B0C0D0E48
:1000C00008E007E006E005E004E003E002E001E00C
:1000D00000E000BF00BF54E71648807830380A2897
:1000E00011D2DFE800F0050708090A0B0C0D0E0F0E
:1000F00009E00AE007E006E005E004E003E002E0D2
:1001000001E000E000BF00BF3BE70A4880783038DC
:10011000092864D2DFE800F00506071E1F202A2BFD
:1001200062005CE05BE0FFF7D0F878B127F03DFAC1
:100130000FE00000741400202C0000202A310D0074
:100140002A300D002A0000000D000000FCA0FEF780
:1001500037FD44E043E042E0FFF7B7F810B127F085
:10016000CAF802E0F6A0FEF72BFD38E037E0FFF713
:10017000ACF870B3F448407D30280BD1F248807C55
:10018000332803D14120F04908711AE03020EE49AC
:10019000087116E0EC48407D312803D13420EA494B
:1001A00008710EE0E848407D342803D14520E64937
:1001B000087106E0E448407D332802D14420E2493A
:1001C00008713020E04988713320C87126F0C2FDE3
:1001D00003E0FFE7DAA0FEF7F3FC00E000BF00BF9A
:1001E000CFE600BFCDE670B58EB0D7484078362850
:1001F00078D008DCA0F13100052874D2DFE800F0E7
:1002000010D4EFEEED0039286ED004DC37286CD026
:10021000382868D17DE3412868D06128F9D1EEE320
:10022000C948807842286FD00EDCA0F13000122837
:1002300046D2DFE800F02246494A4D5C5F6A6D70A5
:10024000B6B6B6B6B6B6B67D622876D00CDC452812
:100250006CD004DC43287ED0442831D184E0462889
:1002600075D06128F9D164E0632875D064287CD00A
:1002700065286FD06628F0D18DE0B349087CFEF781
:100280003FFE0646B049C87BFEF73AFE06EB001477
:10029000AD49487BFEF734FE0646AB49087BFEF7C6
:1002A0002FFE06EB001000EB8000400005B200209E
:1002B0004FF47A73224629460090022014F076F912
:1002C0006FE024F0B4FC6CE06BE018F0BBFF68E07A
:1002D00001204FF4E1630522322100900B2014F03D
:1002E00065F95EE06BE2F1E347E3D8E2C9E302F0CF
:1002F00055FA56E001204FF4E163052232210090C7
:10030000092014F053F94CE016E002F031FF48E008
:1003100019F0A2F945E001204FF448730522282185
:100320000090002014F042F93BE006E027E012E0E4
:1003300000BF15F0FDFA34E000BF01204FF4487310
:10034000052228210090032014F030F929E021E053
:1003500002E00AE014E000BF01234FF448720521D7
:10036000282016F0E5F91CE000BF01204FF4487387
:10037000052228210090082014F018F911E000BF90
:1003800001204FF448730522282100900A2014F020
:100390000DF906E000BF01220021084619F031FDE9
:1003A00000BF00BF0EB070BD67488078382843D0CA
:1003B00009DCA0F1300008284CD2DFE800F0181B5F
:1003C0001E212427313A432842D009DC392836D06F
:1003D000412837D042283DD136E0B4E1E4E03BE0AB
:1003E000612830D0622830D0632833D131E01AF050
:1003F00043F92FE003F0C3F82CE010F0EDF829E00A
:1004000018F0C7FA26E003F095FA23E001204FF434
:100410004873052228210090104614F0C7F819E00F
:1004200001204FF4487305222821009014F0BEF8F3
:1004300010E00FF083FB0DE016F058FF0AE017F014
:1004400030F907E000BF05E000BF1EF061FE01E0EB
:1004500000BF00BF00BFA5E73B48807837282ED0FB
:1004600009DCA0F13000072816D2DFE800F01316EF
:10047000191C1F222500422868D006DC38281FD00E
:10048000392820D0412807D12BE061282AD06228C2
:1004900002D15CE00EF002FF84E00FF0DDF981E0B4
:1004A0000EF02AFD7EE017F04DFB7BE020F007F810
:1004B00078E020F029FB75E01FF0D3FE72E071E0D8
:1004C0000FF0A4FE6EE00020F2F734FF0F220721A8
:1004D0000420F1F7BDFC04228A21012010F00AFD5E
:1004E00060E000BF0020F2F725FF1749C87DFEF746
:1004F00007FD44B21449887DFEF702FD45B221464E
:100500002846FEF7B0FE1049087DFEF7F9FC0646C6
:100510000D49C87CFEF7F4FC06EB00140A49487C40
:10052000FEF7EEFC06460849087CFEF7E9FC06EB00
:10053000001504222146284610F0DCFC32E005E0DC
:100540002A393939390D20007414002000BFFD49C3
:10055000C87DFEF7D5FC0446FA49887DFEF7D0FC3D
:100560000546224629460520F1F772FCF549087D2B
:10057000FEF7C6FC0646F349C87CFEF7C1FC06EB55
:100580000014F049487CFEF7BBFC0646ED49087CA8
:10059000FEF7B6FC06EB001505222146284610F0B2
:1005A000A9FC00BF00BFFDE6E648807839286FD07F
:1005B0000ADCA0F1300009281DD2DFE800F01A1D86
:1005C0002124273D47565900452871D008DC412891
:1005D00079D0422878D043286DD044280BD1A1E0AF
:1005E000622872D0632868D0642867D0652802D159
:1005F0009DE020F003FEA4E0002020F034FCA0E009
:1006000017F00FFE9DE01BF0EAFA9AE0CD48C078A3
:100610004D2807D10220FEF7EBFE18B10020C94992
:100620000871487101204FF4E163052232210090E6
:10063000002013F0BBFF84E001204FF44873052233
:1006400064210090002013F0B1FF7AE0BD48C0782B
:100650004D2807D10220FEF7CBFE18B10020B94982
:10066000487288721CF0BAFD6BE01CF025FB68E054
:10067000B448C0784D2807D10220FEF7B9FE18B162
:100680000020B049C87108721CF0DCF859E0FFE79F
:100690002FF03EFE0068AB49C979405C20280ED19E
:1006A000A849C879FEF72CFC04461AF0EEF909E0D7
:1006B0003CE008E008E01EE007E01DE033E0002039
:1006C0001AF0E3F93DE03CE000BF9E48C0784D28B9
:1006D00007D10220FEF78CFE18B10020994908715D
:1006E000487101204FF4E163052232210090062079
:1006F00013F05CFF25E000BF9248C0784D2807D179
:100700000220FEF775FE18B100208E49087148716D
:1007100001204FF4E163052232210090072013F0FD
:1007200045FF0EE000BF21F0D5FB0AE000BF01202D
:100730004FF4E1630246322100900C2013F036FFA3
:1007400000BF00BF2EE67F488078362822D008DC24
:10075000A0F13000062830D2DFE800F010131415A5
:100760001619392821D004DC372817D0382824D18D
:1007700018E041281CD061281FD11AE0FDF757F975
:100780001BE01AE019E018E01DF08FFC15E003F003
:10079000EDF812E001201EF00DFF0EE000201EF02B
:1007A00009FF0AE001F0F2FD07E002F03EFA04E082
:1007B00000BF02201EF0FEFE00BF00BFF2E5614850
:1007C0008078422851D00EDCA0F13000122864D28B
:1007D000DFE800F02225282B2E33373B3F436363AD
:1007E000636363636346622840D00CDC45284BD0CA
:1007F00004DC43283ED044284FD13FE0462848D06F
:1008000061284AD12DE0632835D0642837D0652887
:100810003BD0662841D13DE022F0C9FB3DE022F00B
:100820003DFE3AE023F048F837E021F0DFFE34E007
:100830000021084629F04CF92FE0002028F047FE5F
:100840002BE0002008F0BBFF27E0012006F039FB79
:1008500023E0002006F035FB1FE00AF002FD1CE05B
:1008600000BF022006F02DFB17E000BF022008F0B9
:10087000A6FF12E000BF03F083FF0EE000BF0121DE
:10088000002029F025F908E000BF032006F019FB3D
:1008900003E000BF0DF007F800BF00BF82E5294864
:1008A000807838282BD009DCA0F1300008282ED21F
:1008B000DFE800F015181F2021222324432824D02C
:1008C00006DC39281CD041281BD042281FD11AE051
:1008D000612817D0622817D0632818D116E023F0BA
:1008E000FEF914E001A826F0BAFF01A827F02DFBBD
:1008F0000DE00CE00BE00AE009E008E007E006E0AC
:1009000005E000BF03E000BF01E000BF00BF00BF83
:1009100048E50C488078382825D009DCA0F1300063
:10092000082828D2DFE800F01718191A1B1C1D1E12
:1009300043281ED008DC392816D0412815D042287B
:1009400019D114E07414002061280FD062280FD050
:10095000632810D10EE00EE00DE00CE00BE00AE0A1
:1009600009E008E007E006E005E000BF03E000BFA3
:1009700001E000BF00BF00BF14E5F94880783828C7
:1009800025D009DCA0F13000082878D2DFE800F09B
:100990001718191A1B1C1D1E462820D008DC3928E0
:1009A00016D0412815D0422815D0432867D114E02D
:1009B00061280FD062280FD0632860D10EE05EE07E
:1009C0005DE05CE05BE05AE059E058E057E056E05B
:1009D00055E000BF53E000BF51E000BF4FE0E049E9
:1009E0000879FEF78DFA012801D1092416E0DC49C7
:1009F0000879FEF785FA022802D10A240EE041E0C8
:100A0000D7490879FEF77CFA032801D10B2405E0C9
:100A100000243020D249087188710872D049087AC0
:100A2000FEF76EFA0546CE498879FEF769FA064662
:100A30002A4631462046F1F70BFA2A20F0F738FD16
:100A4000C7490879FEF75CFA0446FEF7C4F820208F
:100A5000F0F72EFDC2498879FEF752FA0446FEF7F8
:100A6000BAF82020F0F724FDBD49087AFEF748FACD
:100A70000446FEF7B0F80D20F0F71AFD00BF00BFE6
:100A800090E400BFB6488078422845D00EDCA0F143
:100A90003000122868D2DFE800F02326292C2F32FC
:100AA0003337383C676767676767673D622834D0CC
:100AB0000DDC452836D004DC43282FD0442853D100
:100AC0002EE0462830D061284ED124E04EE0632845
:100AD00025D0642825D0652825D0662844D124E077
:100AE0001EF0B3F840E020F051FF3DE029F04BFA52
:100AF0003AE029F09CFE37E02AF056F834E033E083
:100B0000002008F05CFE2FE02EE0002006F0D9F96E
:100B10002AE029E000BF27E000BF25E000BF23E076
:100B200000BF21E000BF1FE000BF8D4800793128E1
:100B300007D10120F3F78DF8AFF60020FEF740F85B
:100B400011E087480079322806D10220F3F781F8B6
:100B500084A0FEF735F806E00020F3F77AF8AFF648
:100B60002020FEF72DF800BF00BF1BE400BF19E4F2
:100B700070B57B484078313809286ED2DFE800F044
:100B800005726D6D6D8AA2E5EF0075488078382892
:100B90005BD009DCA0F13000082861D2DFE800F06A
:100BA0001516191C25263E50432857D006DC392837
:100BB0004ED041284DD0422852D14CE0612849D036
:100BC000622849D063284BD149E049E0FCF730FC6A
:100BD00046E0FCF749FD43E063A0FDF7F1FF642028
:100BE000FFF778F8FDF7F9FD3AE039E063A0FDF78B
:100BF000E7FF6B486B490860BFF34F8F6A48006896
:100C000000F4E06069490843001D67490860BFF3CC
:100C10004F8F40F6B830FFF75DF821E0504800797B
:100C2000302806D10020F0F7CBFC61A0FDF7C8FF0B
:100C300005E065A0FDF7C4FF0120F0F7C1FC0FE05F
:100C40004748C01CFFF766F80AE0FBF73CF807E0EE
:100C500006E000BF04E000BF02E030E200BF00BFDA
:100C600000BF70BD3E48807830380A2810D2DFE8D7
:100C700000F005060708090A0B0C0D0E08E007E056
:100C800006E005E004E003E002E001E000E000BF70
:100C900000BFE6E73248807830380A2810D2DFE813
:100CA00000F005060708090A0B0C0D0E08E007E026
:100CB00006E005E004E003E002E001E000E000BF40
:100CC00000BFCEE72648807830380A283BD2DFE8DC
:100CD00000F005080B0E27282B2F3439F2F7DDFF23
:100CE00031E0F3F71AF82EE0F3F71FF82BE01C4978
:100CF0000879FEF705F9642100FB01F618494879E7
:100D0000FEF7FEF800EB800006EB400614498879F8
:100D1000FEF7F6F8304445022846F3F752F812E0A1
:100D200011E0F2F7CDFF0EE001202D4908700AE036
:100D300001210420F4F764FE05E001210820F4F706
:100D40005FFE00E000BF00BF8BE7054880784128C8
:100D50006FD04EDCA0F130000A286BD242E0FBE0FD
:100D6000741400202A320D00557361727431203CD6
:100D70002D3E20557361727433210D00456E7465EC
:100D800072696E6720426F6F74204C6F6164657288
:100D90002E2E200D42796520627965210D0000001C
:100DA000EFBEADDEF0FF00200CED00E00000FA0524
:100DB0002A576972656C65737320636F6D2064696F
:100DC0007361626C65640D002A576972656C6573A6
:100DD0007320636F6D20656E61626C65640D000049
:100DE00051000020DFE800F01A304C52679EA2A6A6
:100DF000AAAB61287AD008DC422878D0432877D083
:100E0000442876D0452815D1A2E0622872D0632804
:100E100071D0642870D06528F5D19AE0A948C078CF
:100E200058B1A848001D2FF043FCC6B2042E02DBC7
:100E300017E785E08EE0354602E0EFF761FE0546F4
:100E4000284600F0CDF985E0FAF740FE044612E0AE
:100E50002188080AF0F72CFB2078F0F729FBA0780E
:100E6000F0F726FBE078F0F723FB2046FAF70EFEBA
:100E70000446F0F7D4FB002CEAD1FAF72DFE69E026
:100E8000FCF731FD90A0FDF79BFE63E08D48C07834
:100E900010B900208B4908718A48001DFCF73CFD01
:100EA00028B1FCF77AFD0546FDF78AFE02E08BA02B
:100EB000FDF786FE4EE0FCF716FD8FA0FCF72CFD3B
:100EC00048B3FCF76AFD054628462FF010FC1F28A2
:100ED0001DD9132229468AA02FF028FCB8B98DA06D
:100EE000FDF76EFE133505F10C060AE029E029E056
:100EF0002AE02BE027E028E029E015F8010BF0F7C5
:100F0000D7FAB542F9D30D20F0F7D2FA02E083A068
:100F1000FDF756FE02E089A0FDF752FE8EA0FCF719
:100F2000FBFC17E08EA0FDF74BFE13E094A0FDF74D
:100F300047FE0FE08AA0FDF743FE0BE00AE009E060
:100F400000BF07E000BF05E000BF03E000BF01E015
:100F500000BF00BF00BFB2E05A488078412879D076
:100F60000ADCA0F130000A281ED2DFE800F01A1EC9
:100F7000222D2E3198999A9B61286CD008DC42284A
:100F80006AD0432869D0442868D045280CD192E023
:100F900062286FD063286ED064286DD06528F5D1A3
:100FA0008AE06FA0FDF70CFE87E06DA0FDF708FE5C
:100FB00083E0F2F7B2FE18B178A0FDF701FE02E07F
:100FC0007BA0FDF7FDFD78E077E0FBF77AFB74E0AE
:100FD0000120F4F768FA3B4800793038092858D2E4
:100FE000DFE800F005090D1115191D21250000206D
:100FF000F4F759FA51E00120F4F71FFA4DE002200E
:10100000F4F71BFA49E00420F4F717FA45E008204A
:10101000F4F713FA41E01020F4F70FFA3DE0202036
:10102000F4F70BFA39E00020F4F707FA35E0002571
:10103000012600206449088000BF2846F4F7FDF926
:101040005020FEF747FE55B9681CC5B2681CC5B2F2
:10105000012609E027E027E027E028E029E016B193
:101060006806050E00E06D10202D08DD102526B95C
:10107000012003E01AE01BE01CE000200646524875
:1010800000880028D9D000204F490880F4F70BFAD7
:1010900003E04EA0FDF794FD00BF00BF0DE00CE0A3
:1010A0000BE00AE009E000BF07E000BF05E000BF79
:1010B00003E000BF01E000BF00BF00BFD1E500BFFB
:1010C00000BFCEE574140020456E746572696E67CA
:1010D000204154206D6F64650D0000002A4E6F2082
:1010E000726573706F6E73652066726F6D206D6FC1
:1010F00064756C650D00000041494C42413F0000A1
:1011000041542A41494C42413F0D0D0A2A41494C64
:1011100042413A004254204D41432000496E7661DD
:101120006C696420726573706F6E73652066726F90
:101130006D206D6F64756C650D0000004E6F207240
:101140006573706F6E73652066726F6D206D6F646E
:10115000756C650D000000004144444D0000000026
:10116000436D64206F6E6C7920696D706C656D6580
:101170006E74656420696E2077656173792B0D004C
:101180005553424820646576696365206E6F74200C
:10119000636F6E6E65637465640D000053442D6368
:1011A00061726420696E7365727465640D0000007D
:1011B00053442D63617264206E6F7420696E736591
:1011C000727465640D0000000A000020496E7661AB
:1011D0006C696420636F6D6D616E64210D000000A9
:1011E0005649087070472DE9F341044636E02078EF
:1011F00025282FD1641C2078632814D064280BD0B4
:10120000732802D0782820D116E0019820C80190D8
:101210002846FDF7D5FC1CE0019840C801903046F7
:10122000FDF726FD15E0019810F8041BCFB20190E0
:101230003846F0F73DF90CE0019810F8041BCFB2E6
:1012400001903846FDF7EAFD03E02078F0F730F929
:1012500000BF02E02078F0F72BF9641C207800280A
:10126000C5D1BDE8FC810FB4F8B505460C4633483E
:101270000078E0B131480078EFF73DFC064609A858
:1012800000902846FDF79CFC2DA0FDF799FCA0B22C
:10129000FDF7A1FC2BA0FDF793FC00990898FFF740
:1012A000A2FF002000903046EFF725FC00BF00BFF2
:1012B000FEE70FB4F8B505460C462048007810B993
:1012C000F8BC5DF814FB1D480078EFF714FC0646E7
:1012D00009A800902846FDF773FC19A0FDF770FCE3
:1012E000A0B2FDF778FC17A0FDF76AFC00990898FA
:1012F000FFF779FF002000903046EFF7FCFB00BFBE
:1013000000BFDDE70FB438B50C48007810B938BC21
:101310005DF814FB09480078EFF7EDFB044605A8DB
:10132000009000990498FFF75EFF0020009020468F
:10133000EFF7E1FB00BF00BFE9E70000A2010020DA
:101340002028000029203A00F0B502460C46002073
:10135000012100251678302E07D15678782E02D03C
:101360005678582E01D1921C0125002315E01678DD
:10137000302E02DB1678392E0BDD1678412E02DB7B
:101380001678462E05DD1678612E04DB1678662E5B
:1013900001DC5B1C00E002E0521C002AE7D100BF28
:1013A00024B10DB19E1C00E01E46268021E0521E95
:1013B0001678302E07DB1678392E04DC1678303E8E
:1013C00006FB010014E01678412E07DB1678462E46
:1013D00004DC1678373E06FB010009E01678612E22
:1013E00006DB1678662E03DC1678573E06FB0100F6
:1013F00009011E00A3F10103D9D1F0BDF0B50246E9
:101400000B4600240125002610782D2801D1012645
:10141000521C002109E01078302804DB10783928AC
:1014200001DC491C00E002E0521C002AF3D100BF9D
:1014300023B10EB1481C00E0084618800DE0521E92
:101440001078302806DB1078392803DC1078303823
:1014500000FB054405EB850045000800A1F10101F2
:10146000EDD127460EB17842F0BD2046FCE72DE9CC
:10147000F04F89B006460C46174614224FA104A827
:101480002FF0E4F94FF000090025AA46AB460A2CDC
:1014900006D0102C04D00020387009B0BDE8F08FC1
:1014A0002EB930222846691CCDB23A5438E00A2CB5
:1014B00006D1002E04DA4FF0010BC6F1000800E05F
:1014C000B0460EE0B8FBF4F004FB1080C5B204A8EF
:1014D000425D4846411C01F0FF0901A90A54B8FBCE
:1014E000F4F8B8F1000FEDD1BBF1000F06D02D22BA
:1014F0004846411C01F0FF0901A90A54A9F1010065
:1015000000F0FF0A002509E001A810F80A0078554C
:10151000681CC5B2AAF1010000F0FF0A4D45F3DBDB
:1015200000222846691CCDB23A5400BFB5E7F8B591
:1015300004460D461746002614E069462046FFF78C
:1015400003FF05F8010BBDF80000022800D00EE0F3
:10155000701C86B2A078202803D0A0785F2800D025
:1015600005E0E41CBE4202DA20780028E5D100BF85
:101570003046F8BD30B502460020002305E012F8E1
:10158000015B2C18E0B25C1CA3B28B42F7DB30BDD0
:101590000146302903DB392901DC0120704761292C
:1015A00003DB662901DC0120F8E7412903DB46293A
:1015B00001DC0120F2E70020F0E700003031323397
:1015C000343536373839414243444546000000003F
:1015D00002461078802803D1D0780880101D70470B
:1015E000107800F0C000802805D1107800F03F008E
:1015F0000880D01CF3E7107818B9D0780880101D47
:10160000EDE7107800F0C00028B9107800F03F0036
:101610000880501CE3E70020088000BFDFE7024697
:101620001078012804DB1078401E0880901C704759
:101630000020088000BFFAE70146487870474170F3
:1016400070474A1C02707047014602230A46012077
:101650001070022070472DE9F04104460D461646F1
:101660002F4614B1012C0BD105E031463846FFF767
:10167000D6FFBDE8F08131463846FFF7A9FFF8E70D
:1016800000BF00BF0020F4E770B504460D462E46AB
:101690001CB93046FFF7D0FF70BD0020FCE72DE9F4
:1016A000F04104460D4616462F461CB931463846D1
:1016B000FFF7C5FFBDE8F08170B504460D461CB9C3
:1016C0002846FFF7C1FF70BD0020FCE72DE9F0417F
:1016D00004460D4616462F461CB931463846FFF7DC
:1016E000B0FFBDE8F081002101807047F0B58BB0FC
:1016F00005460E46282201A93046FFF718FF87B29B
:10170000002406E001A8015DA81C20F81410601C4C
:1017100084B2BC42F6DB2F800BB0F0BD30B503467F
:101720000C461888904201DC188808B9002030BDAA
:10173000012A04D12088FF2801D10020F7E70021E9
:101740000AE0981C30F8110034F81150A84201D07A
:101750000020ECE7481C81B218888842F1DC0120A7
:10176000E5E7000000203049A1F80208A1F80008D0
:1017700081F8050881F8040870472B4981F80408AE
:1017800070472DE9F041284C94F8050860B3B4F88F
:101790000008051904F50068002084F80508B4F86D
:1017A000020800B3002616E015F8017B1E4890F8E9
:1017B0000408012803D13846FDF7D8FA02E038467C
:1017C000FDF709FA2020EFF773FE00BF454500D36F
:1017D0002546701C86B2B4F80208B042E4DC002052
:1017E000A4F8020800BF00BFBDE8F08170B505464F
:1017F0000D4C012084F80508B4F80208B0F5006F1C
:1018000001D3FFF7BEFF72B6B4F80008B4F80218AF
:101810000844C0F30A06A555B4F80208401CA4F811
:10182000020862B670BD0000AE73002010B503461A
:10183000AC4CAD48007858B12146002206E048681B
:10184000984201D1084610BD521C1031802AF6D3AF
:101850000020F8E7A349002008E04FF0FF3201EB39
:1018600000135A6001EB00131A60401C8028F4D367
:10187000704710B59B4CFFF7EDFF002084F803087C
:101880009A49087001209849087010BD95490020B8
:1018900007E0002201EB00131A7301EB0013DA7268
:1018A000401C8028F5D370472DE9F04107460E46CD
:1018B0008C4D8D48007808B9FFF7DBFF3046FFF705
:1018C000B5FFC8B9002415E072B605EB04104068F6
:1018D000401C68B905EB0410076005EB0410466076
:1018E000002005EB0411887262B60120BDE8F0818A
:1018F00062B6641C802CE7D30020F7E710B50346DE
:10190000784A002112E072B602EB0110406898425A
:101910000AD14FF0FF3002EB0114606002EB0114BA
:10192000206062B6012010BD62B6491C8029EAD34E
:101930000020F8E7F0B502460B466A4C4FF0FF3145
:101940000D4600200DE004EB00167668761C3EB1D3
:1019500004EB001CDCF80460F74331403D4000BF5D
:10196000401C8028EFD3116041EA05061E60F0BDDF
:1019700070B505462846FFF759FF04460CB12046CE
:1019800070BD0020FCE770B506460D46554C564824
:10199000007808B9FFF76DFFA4F8006884F80258D2
:1019A000012084F8030870BDF8B504460E461746BA
:1019B0004C4DE07A20F00100E07295F80308A8B1E0
:1019C000B5F80008002811DDB5F80008B8420DD8B8
:1019D000B5F80018491E88B2315C95F8022891428A
:1019E00003D1E17A41F00101E17200BFE07A20F019
:1019F0000E00E072032F1FD36946304609F052F8FB
:101A0000C8B19DF80000212804D0232807D07828E9
:101A10000FD109E0E07A40F00200E0720AE0E07ADB
:101A200040F00400E07205E0E07A40F00800E07267
:101A300000E000BF00BF00BFF8BD002172B62B4818
:101A4000007858B90120294A107062B628494FF62B
:101A5000FF700880012088700846704762B6002039
:101A6000FBE70246002172B62048007860B90120E9
:101A70001E4B187062B61E494FF6FF70088000209A
:101A80008870CA700846704762B60020FBE710B540
:101A90000146144A0888401C08800888802801D123
:101AA000002010BD0888802801D9002008800FE0A0
:101AB0000B8802EB031043685B1C33B18B781BB9B6
:101AC000CB78847AA34200D1EBE70888401C0880D9
:101AD00008888028ECD30020E3E700210160034A56
:101AE00011707047B47B0020A4010020AA010020DF
:101AF000A60100202DE9F04105460C465CB12846C0
:101B0000FCF74DF806462846FCF744F807463146F0
:101B100029F085FA0AE02846FCF741F806462846EF
:101B2000FCF738F80746314629F07BFABDE8F0812A
:101B300070B504462046FCF732F805462046FCF70F
:101B400029F80646294629F075FA70BD70B5044695
:101B50002046FCF724F805462046FCF71BF806460D
:101B6000294629F042FA08B1012070BD0020FCE7A7
:101B70000021C180018141808180704710B50446F9
:101B8000601EFE4951F8200028B9204600F0E0F917
:101B900008B9002010BD601EF84951F82000F9E78F
:101BA0000246108920B102F10B030B60012070473F
:101BB0000020FCE770B506460C46206880B120681E
:101BC00000F005FA2168891C4518318906F10B00DF
:101BD0000844A84203D929462160012070BD00BFF6
:101BE0000020FBE7024639B1138902F10B001844CB
:101BF000884201D9002070470120FCE710B500247D
